:020000040000FA
:06000000BAEFE6F0120069
:06100000BAEFE6F0120059
:0610080016EF7EF012005D
:06101800EEEF7DF0120076
:06102A00140057CE010086
:10103000B1070000010000000BCE0100890500008F
:101040004C00000009CE0100AA07000002000000C9
:1010500006CE0100970700000300000039C9010017
:10106000B00700000100000004CE0100A807000046
:1010700002000000A7740000AF070000010000009C
:10108000F7CD01006C0700000D000000F5CD010058
:10109000A607000002000000F2CD0100FD050000DF
:1010A00003000000D3CD0100AE07000001000000E6
:1010B000F0CD0100A407000002000000E7CD010010
:1010C0008E07000009000000C33A0100AD070000D0
:1010D00001000000E5CD0100A207000002000000B1
:1010E000E1CD01003C0F000004000000DECD010056
:1010F000FD03000003000000DCCD0100A00700009C
:1011000002000000DACD01009E070000020000008E
:0C111000D8CD01009A070000020000008A
:04111C004D50465399
:1011200002010C00465EE6CD863AAC76FFFFE67221
:10113000EC46FFFFA663865BE6B4666A2801000002
:1011400090010000050000003EE14A4B0000000055
:1011500000003001000095010000050000003EE1A4
:101160004A4B000000000000390100009A01000015
:10117000030000003EE14A4B000000000000440173
:1011800000009D0100004D4000003EF9B94B0000F9
:101190000000020050010000EA410000700300005E
:1011A0003EF9B94B000000000000510100005A4513
:1011B0000000030000003EE14A4B00000000000078
:1011C0005D0100005D450000C61A00008F015D4E04
:1011D00000000000020068010000236000005803C6
:1011E00000008F015D4E000000000000690100005A
:1011F0007B630000050000003EE14A4B0000000058
:1012000000007101000080630000030000003EE167
:101210004A4B0000000000007C01000083630000D6
:10122000030000003EE14A4B00000000000088017E
:10123000000086630000050000003EE14A4B00000C
:10124000000000006164632E636769006175746863
:101250002E63676900636F6E6669672E6367690056
:10126000636F6E6669672E68746D6C0000636F6EE5
:10127000666967322E63676900696E6465782E68F7
:10128000746D6C00006C63642E636769006D6F643D
:101290006966792E636769006D6F64696679322EBD
:1012A000636769006E74702E636769002531300DC5
:1012B0000A2530350D0A2530323C21444F4354591C
:1012C00050452068746D6C205055424C4943202293
:1012D0002D2F2F5733432F2F445444205848544D1B
:1012E0004C20312E30205374726963742F2F454E79
:1012F000222022687474703A2F2F7777772E7733F5
:101300002E6F72672F54522F7868746D6C312F4492
:1013100054442F7868746D6C312D737472696374E2
:101320002E647464223E0D0A3C68746D6C20786DE6
:101330006C6E733D22687474703A2F2F7777772E16
:1013400077332E6F72672F313939392F7868746D82
:101350006C223E0D0A3C686561643E0D0A20203C0B
:101360006D65746120687474702D65717569763D62
:1013700022436F6E74656E742D54797065222063FC
:101380006F6E74656E743D22746578742F68746D29
:101390006C3B20636861727365743D536869667461
:1013A0005F4A4953223E0D0A20203C6D657461203E
:1013B000687474702D65717569763D22707261670D
:1013C0006D612220636F6E74656E743D226E6F2DA9
:1013D000636163686522202F3E0D0A20203C6D6505
:1013E000746120687474702D65717569763D22632F
:1013F000616368652D636F6E74726F6C2220636F1A
:101400006E74656E743D226E6F2D63616368652234
:10141000202F3E0D0A20203C7469746C653E5049B3
:10142000432D4E494320436F6E6669677572617440
:10143000696F6E3C2F7469746C653E0D0A3C736372
:1014400072697074206C616E67756167653D224AD0
:10145000617661536372697074223E0D0A3C212DDE
:101460002D0D0A66756E6374696F6E20436865633F
:101470006B436F6E6669726D287061727473290DAB
:101480000A7B0D0A2069662028646F63756D656E9E
:10149000742E61757468662E7073312E76616C756A
:1014A0006520213D20646F63756D656E742E6175D6
:1014B0007468662E7073322E76616C756520290D06
:1014C0000A207B0D0A2020616C6572742822526507
:1014D000747279205B4E65772050617373776F72F9
:1014E000645D206F72205B436F6E6669726D205081
:1014F000617373776F72645D206669656C642E2218
:10150000293B0D0A202072657475726E2066616C2D
:1015100073653B0D0A207D0D0A20656C73650D0A0D
:10152000207B0D0A202072657475726E20747275AE
:10153000653B0D0A207D0D0A7D0D0A2D2D3E0D0AFD
:101540003C2F7363726970743E0D0A0D0A3C73631D
:1015500072697074206C616E67756167653D224ABF
:10156000617661536372697074223E0D0A3C212DCD
:101570002D0D0A66756E6374696F6E20496E69740D
:10158000436F6E6669726D287061727473290D0AFB
:101590007B0D0A206D79526574203D20636F6E6665
:1015A00069726D2822446F20796F7520696E6974A5
:1015B00069616C697A6520746869732073657474F5
:1015C000696E67203F22290D0A2069662028206D58
:1015D00079526574203D3D207472756520290D0A8D
:1015E000207B0D0A202070617274732E666F726DFD
:1015F0002E7375626D697428293B0D0A207D0D0AD2
:101600007D0D0A2D2D3E0D0A3C2F73637269707497
:101610003E0D0A3C2F686561643E0D0A3C626F64B2
:10162000793E0D0A3C666F6E742073697A653D22BF
:101630002B32223E3C7370616E207374796C653D71
:1016400022666F6E742D7765696768743A20626FE1
:101650006C643B223E0D0A436F6E6669677572616A
:1016600074696F6E3C2F7370616E3E3C6272202F06
:101670003E0D0A3C2F666F6E743E0D0A3C68722068
:101680002F3E0D0A3C666F726D206D6574686F6445
:101690003D22706F73742220616374696F6E3D2206
:1016A000636F6E6669672E636769223E0D0A2020AC
:1016B0003C68333E4E6574776F726B3C2F68333EE7
:1016C0000D0A20203C68353E81A6836C83628367C7
:1016D000838F815B834E8AD68C5782CC83708389BB
:1016E0008381815B835E82F095CF8D588CE382CDC0
:1016F0008141838A835A8362836782B582C489BAAF
:1017000082B382A281423C2F68353E0D0A20203CE4
:10171000646C3E0D0A202020203C64643E0D0A20AB
:1017200020202020203C7461626C6520626F72640E
:1017300065723D2231223E0D0A20202020202020EB
:10174000203C74626F64793E0D0A20202020202006
:10175000202020203C74723E0D0A202020202020D2
:101760002020202020203C74643E266E6273703B53
:101770004D41432041646472657373266E627370D9
:101780003B3C2F74643E0D0A202020202020202086
:10179000202020203C74643E266E6273703B7E6382
:1017A0006F6E6669675F6D616328297E0D0A202070
:1017B000202020202020202020203C2F74643E0D5B
:1017C0000A202020202020202020203C2F74723E40
:1017D0000D0A202020202020202020203C74723E52
:1017E0000D0A2020202020202020202020203C74B2
:1017F000643E266E6273703B49502041646472659A
:101800007373266E6273703B3C2F74643E0D0A2026
:1018100020202020202020202020203C74643E3CDA
:10182000696E707574206D61786C656E6774683D63
:1018300022313522206E616D653D2269702220764D
:10184000616C75653D227E636F6E6669675F697066
:1018500028297E22202F3E266E6273703B0D0A20BF
:101860002020202020202020202020202020204454
:101870004843503C696E707574206E616D653D2201
:10188000646863702220747970653D2263686563C3
:101890006B626F7822207E646863705F737728299B
:1018A0007E202F3E3C2F74643E0D0A2020202020F5
:1018B00020202020203C2F74723E0D0A2020202062
:1018C0002020202020203C74723E0D0A2020202061
:1018D00020202020202020203C74643E266E62734D
:1018E000703B4E6574204D61736B266E6273703B66
:1018F0003C2F74643E0D0A20202020202020202030
:101900002020203C74643E3C696E707574206D61CB
:10191000786C656E6774683D22313522206E616D8A
:10192000653D22737562222076616C75653D227E6D
:10193000636F6E6669675F7375626E657428297E72
:1019400022202F3E3C2F74643E0D0A2020202020B0
:1019500020202020203C2F74723E0D0A20202020C1
:101960002020202020203C74723E0D0A20202020C0
:1019700020202020202020203C74643E266E6273AC
:10198000703B47617465776179266E6273703B3C8A
:101990002F74643E0D0A20202020202020202020AB
:1019A00020203C74643E3C696E707574206D6178D3
:1019B0006C656E6774683D22313522206E616D65FD
:1019C0003D226777222076616C75653D227E636FCC
:1019D0006E6669675F677728297E22202F3E3C2F3D
:1019E00074643E0D0A202020202020202020203C4E
:1019F0002F74723E0D0A202020202020202020203D
:101A00003C74723E0D0A202020202020202020201F
:101A100020203C74643E266E6273703B444E53201B
:101A200073657276657220285072696D61727929CA
:101A3000266E6273703B3C2F74643E0D0A2020209A
:101A40002020202020202020203C74643E3C696E11
:101A5000707574206D61786C656E6774683D2231B5
:101A60003522206E616D653D22646E7331222076D1
:101A7000616C75653D227E636F6E6669675F646E3B
:101A8000733128297E22202F3E3C2F74643E0D0A9C
:101A9000202020202020202020203C2F74723E0D6A
:101AA0000A202020202020202020203C74723E0D7F
:101AB0000A2020202020202020202020203C746488
:101AC0003E266E6273703B444E532073657276659A
:101AD0007220285365636F6E6461727929266E6285
:101AE00073703B3C2F74643E0D0A20202020202080
:101AF0002020202020203C74643E3C696E70757468
:101B0000206D61786C656E6774683D2231352220E6
:101B10006E616D653D22646E7332222076616C7554
:101B2000653D227E636F6E6669675F646E733228FF
:101B3000297E22202F3E3C2F74643E0D0A20202057
:101B4000202020202020203C2F74723E0D0A2020CF
:101B500020202020202020203C74723E0D0A2020CE
:101B6000202020202020202020203C74643E266E4F
:101B70006273703B4854545020506F72743A23265D
:101B80006E6273703B3C2F74643E0D0A202020204F
:101B900020202020202020203C74643E3C696E7070
:101BA0007574206D61786C656E6774683D223522AE
:101BB000206E616D653D226874222076616C7565CA
:101BC0003D227E636F6E6669675F69705F706F72DA
:101BD000742830297E2220747970653D22746578DE
:101BE00074222F3E3C2F74643E0D0A2020202020BA
:101BF00020202020203C2F74723E0D0A202020201F
:101C00002020202020203C74723E0D0A202020201D
:101C100020202020202020203C74643E266E627309
:101C2000703B4C434420506F72743A23266E6273AB
:101C3000703B3C2F74643E0D0A2020202020202081
:101C400020202020203C74643E3C696E7075742016
:101C50006D61786C656E6774683D223522206E6117
:101C60006D653D226C74222076616C75653D227E27
:101C7000636F6E6669675F69705F706F7274283139
:101C8000297E2220747970653D2274657874222F34
:101C90003E0D0A202020202020202020202020204F
:101CA000202020266E6273703B5443503C696E7056
:101CB0007574206E616D653D2274637031222074ED
:101CC0007970653D22636865636B626F7822207E60
:101CD0007463705F73772830297E202F3E3C2F7409
:101CE000643E0D0A202020202020202020203C2F90
:101CF00074723E0D0A202020202020202020203C2D
:101D000074723E0D0A202020202020202020202038
:101D1000203C74643E266E6273703B506172616C4D
:101D20006C656C20506F72743A23266E6273703B40
:101D30003C2F74643E0D0A202020202020202020EB
:101D40002020203C74643E3C696E707574206D6187
:101D5000786C656E6774683D223522206E616D6512
:101D60003D227075222076616C75653D227E636F21
:101D70006E6669675F69705F706F72742832297E62
:101D80002220747970653D2274657874222F3E0D8F
:101D90000A20202020202020202020202020202059
:101DA00020266E6273703B5443503C696E707574AC
:101DB000206E616D653D22746370322220747970EB
:101DC000653D22636865636B626F7822207E746371
:101DD000705F73772831297E202F3E3C2F74643E3C
:101DE0000D0A202020202020202020203C2F74724B
:101DF0003E0D0A202020202020202020203C74722C
:101E00003E0D0A2020202020202020202020203CC1
:101E100074643E266E6273703B53657269616C2018
:101E2000506F72743A23266E6273703B3C2F746459
:101E30003E0D0A2020202020202020202020203C91
:101E400074643E3C696E707574206D61786C656E6B
:101E50006774683D223522206E616D653D22737581
:101E6000222076616C75653D227E636F6E666967C0
:101E70005F69705F706F72742833297E22207479D5
:101E800070653D2274657874222F3E0D0A20202053
:101E900020202020202020202020202020266E62AC
:101EA00073703B5443503C696E707574206E616D65
:101EB000653D22746370332220747970653D22631E
:101EC0006865636B626F7822207E7463705F7377DE
:101ED0002832297E202F3E3C2F74643E0D0A20209C
:101EE00020202020202020203C2F74723E0D0A202C
:101EF0002020202020202020203C74723E0D0A202B
:101F000020202020202020202020203C74643E26F9
:101F10006E6273703B43444320506F72743A2326C1
:101F20006E6273703B3C2F74643E0D0A20202020AB
:101F300020202020202020203C74643E3C696E70CC
:101F40007574206D61786C656E6774683D2235220A
:101F5000206E616D653D226375222076616C75652A
:101F60003D227E636F6E6669675F69705F706F7236
:101F7000742834297E2220747970653D2274657836
:101F800074222F3E0D0A20202020202020202020F7
:101F9000202020202020266E6273703B5443503C4A
:101FA000696E707574206E616D653D227463703466
:101FB0002220747970653D22636865636B626F7877
:101FC00022207E7463705F73772833297E202F3E32
:101FD0003C2F74643E0D0A20202020202020202049
:101FE000203C2F74723E0D0A20202020202020202B
:101FF00020203C74723E0D0A20202020202020202A
:10200000202020203C74643E203C2F74643E0D0A46
:102010002020202020202020202020203C74643EEE
:102020003C696E707574206E616D653D2243665328
:1020300076222076616C75653D225361766522209B
:10204000747970653D227375626D697422202F3E2C
:102050003C696E7075742076616C75653D224465CF
:102060006661756C742220747970653D22627574A6
:10207000746F6E22206F6E436C69636B3D22496EF4
:102080006974436F6E6669726D287468697329227A
:102090002F3E3C2F74643E0D0A202020202020205B
:1020A0002020203C2F74723E0D0A2020202020206A
:1020B00020203C2F74626F64793E0D0A202020207E
:1020C00020203C2F7461626C653E0D0A2020202088
:1020D0003C2F64643E0D0A20203C2F646C3E0D0AA8
:1020E0003C2F666F726D3E0D0A3C666F726D206DFF
:1020F0006574686F643D22706F737422206163742D
:10210000696F6E3D226D6F64696679322E6367690F
:10211000223E0D0A20203C68333E446967697461A1
:102120006C20506F727420446972656374696F6EBD
:102130003C2F68333E0D0A20203C646C3E0D0A2083
:102140002020203C64643E0D0A2020202020203CDA
:102150007461626C6520626F726465723D22312227
:102160003E0D0A20202020202020203C74626F6435
:10217000793E0D0A202020202020202020203C74A1
:10218000723E0D0A20202020202020202020202008
:102190003C74643E266E6273703B44696769746187
:1021A0006C20506F727420446972656374696F6E3D
:1021B000202330266E6273703B3C2F74643E0D0A00
:1021C0002020202020202020202020203C74643E3D
:1021D0000D0A2020202020202020202020203C69C3
:1021E0006E707574206E616D653D227064302220C2
:1021F00076616C75653D22494E2220747970653D8B
:1022000022726164696F22207E6469725F6368650F
:10221000636B656428302C54525545297E202F3E2F
:10222000494E5055540D0A202020202020202020E7
:102230002020203C696E707574206E616D653D22B2
:10224000706430222076616C75653D224F555422B2
:1022500020747970653D22726164696F22207E640A
:1022600069725F636865636B656428302C46414C16
:102270005345297E202F3E4F55545055540D0A206A
:1022800020202020202020202020203C2F74643E6D
:102290000D0A202020202020202020203C2F747296
:1022A0003E0D0A202020202020202020203C747277
:1022B0003E0D0A2020202020202020202020203C0D
:1022C00074643E266E6273703B4469676974616C26
:1022D00020506F7274266E6273703B44697265633E
:1022E00074696F6E202331266E6273703B3C2F74CD
:1022F000643E0D0A202020202020202020202020A5
:102300003C74643E3C696E707574206E616D653D11
:1023100022706431222076616C75653D22494E221F
:1023200020747970653D22726164696F22207E6439
:1023300069725F636865636B656428312C5452551C
:1023400045297E202F3E494E5055540D0A2020200D
:102350002020202020202020203C696E70757420D1
:102360006E616D653D22706431222076616C756509
:102370003D224F55542220747970653D227261646C
:10238000696F22207E6469725F636865636B656450
:1023900028312C46414C5345297E202F3E4F555421
:1023A0005055543C2F74643E0D0A202020202020DC
:1023B000202020203C2F74723E0D0A202020202057
:1023C00020202020203C74723E0D0A202020202056
:1023D000202020202020203C74643E266E627370F2
:1023E0003B4469676974616C20506F7274266E6239
:1023F00073703B446972656374696F6E2023322683
:102400006E6273703B3C2F74643E0D0A20202020C6
:1024100020202020202020203C74643E3C696E70E7
:102420007574206E616D653D227064322220766184
:102430006C75653D22494E2220747970653D22728B
:102440006164696F22207E6469725F636865636B93
:10245000656428322C54525545297E202F3E494E22
:102460005055540D0A2020202020202020202020FC
:10247000203C696E707574206E616D653D227064DC
:1024800032222076616C75653D224F5554222074AE
:102490007970653D22726164696F22207E64697281
:1024A0005F636865636B656428322C46414C534515
:1024B000297E202F3E4F55545055543C2F74643E76
:1024C0000D0A202020202020202020203C2F747264
:1024D0003E0D0A202020202020202020203C747245
:1024E0003E0D0A2020202020202020202020203CDB
:1024F00074643E266E6273703B4469676974616CF4
:1025000020506F7274266E6273703B44697265630B
:1025100074696F6E202333266E6273703B3C2F7498
:10252000643E0D0A20202020202020202020202072
:102530003C74643E3C696E707574206E616D653DDF
:1025400022706433222076616C75653D22494E22EB
:1025500020747970653D22726164696F22207E6407
:1025600069725F636865636B656428332C545255E8
:1025700045297E202F3E494E5055540D0A202020DB
:102580002020202020202020203C696E707574209F
:102590006E616D653D22706433222076616C7565D5
:1025A0003D224F55542220747970653D227261643A
:1025B000696F22207E6469725F636865636B65641E
:1025C00028332C46414C5345297E202F3E4F5554ED
:1025D0005055543C2F74643E0D0A202020202020AA
:1025E000202020203C2F74723E0D0A202020202025
:1025F00020202020203C74723E0D0A202020202024
:10260000202020202020203C74643E266E627370BF
:102610003B4469676974616C20506F7274266E6206
:1026200073703B446972656374696F6E202334264E
:102630006E6273703B3C2F74643E0D0A2020202094
:1026400020202020202020203C74643E3C696E70B5
:102650007574206E616D653D227064342220766150
:102660006C75653D22494E2220747970653D227259
:102670006164696F22207E6469725F636865636B61
:10268000656428342C54525545297E202F3E494EEE
:102690005055540D0A2020202020202020202020CA
:1026A000203C696E707574206E616D653D227064AA
:1026B00034222076616C75653D224F55542220747A
:1026C0007970653D22726164696F22207E6469724F
:1026D0005F636865636B656428342C46414C5345E1
:1026E000297E202F3E4F55545055543C2F74643E44
:1026F0000D0A202020202020202020203C2F747232
:102700003E0D0A202020202020202020203C747212
:102710003E0D0A2020202020202020202020203CA8
:1027200074643E266E6273703B4469676974616CC1
:1027300020506F7274266E6273703B4469726563D9
:1027400074696F6E202335266E6273703B3C2F7464
:10275000643E0D0A20202020202020202020202040
:102760003C74643E3C696E707574206E616D653DAD
:1027700022706435222076616C75653D22494E22B7
:1027800020747970653D22726164696F22207E64D5
:1027900069725F636865636B656428352C545255B4
:1027A00045297E202F3E494E5055540D0A202020A9
:1027B0002020202020202020203C696E707574206D
:1027C0006E616D653D22706435222076616C7565A1
:1027D0003D224F55542220747970653D2272616408
:1027E000696F22207E6469725F636865636B6564EC
:1027F00028352C46414C5345297E202F3E4F5554B9
:102800005055543C2F74643E0D0A20202020202077
:10281000202020203C2F74723E0D0A2020202020F2
:1028200020202020203C74723E0D0A2020202020F1
:10283000202020202020203C74643E266E6273708D
:102840003B4469676974616C20506F7274266E62D4
:1028500073703B446972656374696F6E202336261A
:102860006E6273703B3C2F74643E0D0A2020202062
:1028700020202020202020203C74643E3C696E7083
:102880007574206E616D653D22706436222076611C
:102890006C75653D22494E2220747970653D227227
:1028A0006164696F22207E6469725F636865636B2F
:1028B000656428362C54525545297E202F3E494EBA
:1028C0005055540D0A202020202020202020202098
:1028D000203C696E707574206E616D653D22706478
:1028E00036222076616C75653D224F555422207446
:1028F0007970653D22726164696F22207E6469721D
:102900005F636865636B656428362C46414C5345AC
:10291000297E202F3E4F55545055543C2F74643E11
:102920000D0A202020202020202020203C2F7472FF
:102930003E0D0A202020202020202020203C7472E0
:102940003E0D0A2020202020202020202020203C76
:1029500074643E266E6273703B4469676974616C8F
:1029600020506F7274266E6273703B4469726563A7
:1029700074696F6E202337266E6273703B3C2F7430
:10298000643E0D0A2020202020202020202020200E
:102990003C74643E3C696E707574206E616D653D7B
:1029A00022706437222076616C75653D22494E2283
:1029B00020747970653D22726164696F22207E64A3
:1029C00069725F636865636B656428372C54525580
:1029D00045297E202F3E494E5055540D0A20202077
:1029E0002020202020202020203C696E707574203B
:1029F0006E616D653D22706437222076616C75656D
:102A00003D224F55542220747970653D22726164D5
:102A1000696F22207E6469725F636865636B6564B9
:102A200028372C46414C5345297E202F3E4F555484
:102A30005055543C2F74643E0D0A20202020202045
:102A4000202020203C2F74723E0D0A2020202020C0
:102A500020202020203C74723E0D0A2020202020BF
:102A6000202020202020203C74643E266E6273705B
:102A70003B4469676974616C20506F7274266E62A2
:102A800073703B446972656374696F6E2023383CD0
:102A90002F74643E0D0A202020202020202020209A
:102AA00020203C74643E3C696E707574206E616DCC
:102AB000653D22706438222076616C75653D22493F
:102AC0004E2220747970653D22726164696F222004
:102AD0007E6469725F636865636B656428382C5433
:102AE000525545297E202F3E494E5055540D0A20FF
:102AF00020202020202020202020203C696E70757E
:102B000074206E616D653D22706438222076616CA0
:102B100075653D224F55542220747970653D2272AF
:102B20006164696F22207E6469725F636865636BAC
:102B3000656428382C46414C5345297E202F3E4F52
:102B400055545055543C2F74643E0D0A20202020CB
:102B50002020202020203C2F74723E0D0A202020AF
:102B6000202020202020203C74723E0D0A202020AE
:102B70002020202020202020203C74643E266E62ED
:102B800073703B4469676974616C20506F7274267E
:102B90006E6273703B446972656374696F6E202363
:102BA00039266E6273703B3C2F74643E0D0A202000
:102BB000202020202020202020203C74643E3C69DE
:102BC0006E707574206E616D653D227064392220CF
:102BD00076616C75653D22494E2220747970653DA1
:102BE00022726164696F22207E6469725F63686526
:102BF000636B656428392C54525545297E202F3E3D
:102C0000494E5055540D0A202020202020202020FD
:102C10002020203C696E707574206E616D653D22C8
:102C2000706439222076616C75653D224F555422BF
:102C300020747970653D22726164696F22207E6420
:102C400069725F636865636B656428392C46414C23
:102C50005345297E202F3E4F55545055543C2F74D8
:102C6000643E0D0A202020202020202020203C2F00
:102C700074723E0D0A202020202020202020203C9D
:102C800074723E0D0A2020202020202020202020A9
:102C9000203C74643E266E6273703B4469676974BD
:102CA000616C20506F7274266E6273703B4469725F
:102CB000656374696F6E20233130266E6273703BDA
:102CC0003C2F74643E0D0A2020202020202020204C
:102CD0002020203C74643E3C696E707574206E61E7
:102CE0006D653D2270643130222076616C75653DE2
:102CF00022494E2220747970653D22726164696FA9
:102D000022207E6469725F636865636B6564283145
:102D1000302C54525545297E202F3E494E50555453
:102D20000D0A2020202020202020202020203C6967
:102D30006E707574206E616D653D22706431302255
:102D40002076616C75653D224F5554222074797050
:102D5000653D22726164696F22207E6469725F63DF
:102D60006865636B65642831302C46414C534529B6
:102D70007E202F3E4F55545055543C2F74643E0DC9
:102D80000A202020202020202020203C2F74723E6A
:102D90000D0A202020202020202020203C74723E7C
:102DA0000D0A2020202020202020202020203C74DC
:102DB000643E266E6273703B4469676974616C207F
:102DC000506F7274266E6273703B446972656374EF
:102DD000696F6E202331313C2F74643E0D0A202030
:102DE000202020202020202020203C74643E3C69AC
:102DF0006E707574206E616D653D22706431312294
:102E00002076616C75653D22494E2220747970658B
:102E10003D22726164696F22207E6469725F63681B
:102E200065636B65642831312C54525545297E20E9
:102E30002F3E494E5055540D0A202020202020209E
:102E400020202020203C696E707574206E616D65B5
:102E50003D2270643131222076616C75653D224FD0
:102E600055542220747970653D22726164696F2225
:102E7000207E6469725F636865636B6564283131C5
:102E80002C46414C5345297E202F3E4F55545055DA
:102E9000543C2F74643E0D0A202020202020202046
:102EA00020203C2F74723E0D0A202020202020205C
:102EB0002020203C74723E0D0A202020202020205B
:102EC00020202020203C74643E266E6273703B44B8
:102ED00069676974616C20506F7274266E627370DA
:102EE0003B446972656374696F6E202331323C2FF5
:102EF00074643E0D0A202020202020202020202045
:102F0000203C74643E3C696E707574206E616D6522
:102F10003D2270643132222076616C75653D224914
:102F20004E2220747970653D22726164696F22209F
:102F30007E6469725F636865636B65642831322CF7
:102F400054525545297E202F3E494E5055540D0A66
:102F50002020202020202020202020203C696E706E
:102F60007574206E616D653D227064313222207669
:102F7000616C75653D224F55542220747970653D12
:102F800022726164696F22207E6469725F63686582
:102F9000636B65642831322C46414C5345297E20B1
:102FA0002F3E4F55545055543C2F74643E0D0A200B
:102FB0002020202020202020203C2F74723E0D0A4B
:102FC000202020202020202020203C74723E0D0A4A
:102FD0002020202020202020202020203C74643E1F
:102FE000266E6273703B4469676974616C20506F30
:102FF0007274266E6273703B446972656374696FA4
:103000006E202331333C2F74643E0D0A2020202093
:1030100020202020202020203C74643E3C696E70DB
:103020007574206E616D653D2270643133222076A7
:10303000616C75653D22494E2220747970653D2290
:10304000726164696F22207E6469725F6368656380
:103050006B65642831332C54525545297E202F3E10
:10306000494E5055540D0A20202020202020202099
:103070002020203C696E707574206E616D653D2264
:1030800070643133222076616C75653D224F555452
:103090002220747970653D22726164696F22207EFE
:1030A0006469725F636865636B65642831332C46BD
:1030B000414C5345297E202F3E4F55545055543C8A
:1030C0002F74643E0D0A2020202020202020202064
:1030D0003C2F74723E0D0A2020202020202020202A
:1030E000203C74723E0D0A20202020202020202029
:1030F0002020203C74643E266E6273703B446967F6
:103100006974616C20506F7274266E6273703B44F8
:103110006972656374696F6E202331343C2F746467
:103120003E0D0A2020202020202020202020203C8E
:1031300074643E3C696E707574206E616D653D22ED
:1031400070643134222076616C75653D22494E22CF
:1031500020747970653D22726164696F22207E64FB
:1031600069725F636865636B65642831342C5452FF
:103170005545297E202F3E494E5055540D0A20209A
:10318000202020202020202020203C696E70757493
:10319000206E616D653D2270643134222076616C51
:1031A00075653D224F55542220747970653D227219
:1031B0006164696F22207E6469725F636865636B16
:1031C00065642831342C46414C5345297E202F3EDE
:1031D0004F55545055543C2F74643E0D0A20202006
:1031E000202020202020203C2F74723E0D0A202019
:1031F00020202020202020203C74723E0D0A202018
:10320000202020202020202020203C74643E266E98
:103210006273703B4469676974616C20506F7274AB
:10322000266E6273703B446972656374696F6E20C9
:103230002331353C2F74643E0D0A202020202020AD
:103240002020202020203C74643E3C696E70757400
:10325000206E616D653D2270643135222076616C8F
:1032600075653D22494E2220747970653D22726158
:1032700064696F22207E6469725F636865636B6551
:10328000642831352C54525545297E202F3E494E15
:103290005055540D0A2020202020202020202020BE
:1032A000203C696E707574206E616D653D2270649E
:1032B0003135222076616C75653D224F55542220B0
:1032C000747970653D22726164696F22207E646941
:1032D000725F636865636B65642831352C46414CC9
:1032E0005345297E202F3E4F55545055543C2F7442
:1032F000643E0D0A202020202020202020203C2F6A
:1033000074723E0D0A202020202020202020203C06
:1033100074723E0D0A202020202020202020202012
:10332000203C74643E203C2F74643E0D0A20202013
:103330002020202020202020203C74643E3C696E08
:10334000707574206E616D653D2250645376222045
:1033500076616C75653D22536176652220747970C3
:10336000653D227375626D697422202F3E3C696E43
:103370007075742076616C75653D22446566617573
:103380006C742220747970653D22627574746F6E5E
:1033900022206F6E436C69636B3D22496E697443F2
:1033A0006F6E6669726D287468697329222F3E3CBE
:1033B0002F74643E0D0A2020202020202020202071
:1033C0003C2F74723E0D0A20202020202020203C1B
:1033D0002F74626F64793E0D0A2020202020203C4B
:1033E0002F7461626C653E0D0A202020203C2F6402
:1033F000643E0D0A20203C2F646C3E0D0A3C2F6673
:103400006F726D3E0D0A3C666F726D206D6574685B
:103410006F643D22706F73742220616374696F6EF4
:103420003D22636F6E666967322E636769223E0DC7
:103430000A20203C68333E492F4F20506F72742081
:103440004E616D653C2F68333E0D0A20203C646C54
:103450003E0D0A202020203C64643E0D0A202020DE
:103460002020203C7461626C6520626F726465721A
:103470003D2231223E0D0A20202020202020203C09
:1034800074626F64793E0D0A2020202020202020C5
:1034900020203C74723E0D0A202020202020202075
:1034A000202020203C74643E266E6273703B416E87
:1034B000616C6F6720506F7274204E616D652023C0
:1034C00030266E6273703B3C2F74643E0D0A2020E0
:1034D000202020202020202020203C74643E3C69B5
:1034E0006E707574206D61786C656E6774683D22CE
:1034F0007E4765744D61784C656E677468506F7275
:10350000744E616D6528297E22206E616D653D22B5
:10351000706E30222076616C75653D227E506F7230
:10352000744E616D652830297E22202F3E3C2F7419
:10353000643E0D0A202020202020202020203C2F27
:1035400074723E0D0A202020202020202020203CC4
:1035500074723E0D0A2020202020202020202020D0
:10356000203C74643E266E6273703B416E616C6FEA
:103570006720506F7274204E616D65202331266E76
:103580006273703B3C2F74643E0D0A202020202083
:10359000202020202020203C74643E3C696E707501
:1035A00074206D61786C656E6774683D227E476536
:1035B000744D61784C656E677468506F72744E61BB
:1035C0006D6528297E22206E616D653D22706E3109
:1035D000222076616C75653D227E506F72744E615B
:1035E0006D652831297E22202F3E3C2F74643E0DCC
:1035F0000A202020202020202020203C2F74723EF2
:103600000D0A202020202020202020203C74723E03
:103610000D0A2020202020202020202020203C7463
:10362000643E266E6273703B416E616C6F67205022
:103630006F7274204E616D65202332266E62737046
:103640003B3C2F74643E0D0A2020202020202020A7
:10365000202020203C74643E3C696E707574206D9F
:1036600061786C656E6774683D227E4765744D6154
:10367000784C656E677468506F72744E616D652822
:10368000297E22206E616D653D22706E3222207689
:10369000616C75653D227E506F72744E616D652858
:1036A00032297E22202F3E3C2F74643E0D0A2020BA
:1036B00020202020202020203C2F74723E0D0A2044
:1036C0002020202020202020203C74723E0D0A2043
:1036D00020202020202020202020203C74643E2612
:1036E0006E6273703B416E616C6F6720506F7274D5
:1036F000204E616D65202333266E6273703B3C2F34
:1037000074643E0D0A20202020202020202020202C
:10371000203C74643E3C696E707574206D61786CF9
:10372000656E6774683D227E4765744D61784C65AF
:103730006E677468506F72744E616D6528297E22C1
:10374000206E616D653D22706E33222076616C754E
:10375000653D227E506F72744E616D652833297EFF
:1037600022202F3E3C2F74643E0D0A202020202072
:1037700020202020203C2F74723E0D0A2020202083
:103780002020202020203C74723E0D0A2020202082
:1037900020202020202020203C74643E266E62736E
:1037A000703B416E616C6F6720506F7274204E6188
:1037B0006D65202334266E6273703B3C2F74643E2B
:1037C0000D0A2020202020202020202020203C74B2
:1037D000643E3C696E707574206D61786C656E67CF
:1037E00074683D227E4765744D61784C656E6774E0
:1037F00068506F72744E616D6528297E22206E615B
:103800006D653D22706E34222076616C75653D22B7
:103810007E506F72744E616D652834297E22202F90
:103820003E3C2F74643E0D0A2020202020202020C2
:1038300020203C2F74723E0D0A20202020202020C2
:103840002020203C74723E0D0A20202020202020C1
:1038500020202020203C74643E266E6273703B4121
:103860006E616C6F6720506F7274204E616D6520C1
:103870002335266E6273703B3C2F74643E0D0A2024
:1038800020202020202020202020203C74643E3C4A
:10389000696E707574206D61786C656E6774683DD3
:1038A000227E4765744D61784C656E677468506F11
:1038B00072744E616D6528297E22206E616D653DB2
:1038C00022706E35222076616C75653D227E506FC8
:1038D00072744E616D652835297E22202F3E3C2F63
:1038E00074643E0D0A202020202020202020203C2F
:1038F0002F74723E0D0A202020202020202020201E
:103900003C74723E0D0A2020202020202020202000
:1039100020203C74643E266E6273703B416E616C85
:103920006F6720506F7274204E616D6520233626BC
:103930006E6273703B3C2F74643E0D0A2020202081
:1039400020202020202020203C74643E3C696E70A2
:103950007574206D61786C656E6774683D227E4772
:1039600065744D61784C656E677468506F72744E03
:10397000616D6528297E22206E616D653D22706E25
:1039800036222076616C75653D227E506F72744ED2
:10399000616D652836297E22202F3E3C2F74643EBF
:1039A0000D0A202020202020202020203C2F74726F
:1039B0003E0D0A202020202020202020203C747250
:1039C0003E0D0A2020202020202020202020203CE6
:1039D00074643E266E6273703B416E616C6F67204B
:1039E000506F7274204E616D65202337266E6273AE
:1039F000703B3C2F74643E0D0A20202020202020A4
:103A000020202020203C74643E3C696E7075742038
:103A10006D61786C656E6774683D227E4765744D94
:103A200061784C656E677468506F72744E616D6535
:103A300028297E22206E616D653D22706E3722201E
:103A400076616C75653D227E506F72744E616D6556
:103A50002837297E22202F3E3C2F74643E0D0A20F9
:103A60002020202020202020203C2F74723E0D0A90
:103A7000202020202020202020203C74723E0D0A8F
:103A80002020202020202020202020203C74643E64
:103A9000266E6273703B4469676974616C20506F75
:103AA0007274204E616D65202330266E6273703B08
:103AB0003C2F74643E0D0A2020202020202020204E
:103AC0002020203C74643E3C696E707574206D61EA
:103AD000786C656E6774683D227E4765744D6178C9
:103AE0004C656E677468506F72744E616D652829FD
:103AF0007E22206E616D653D22706E3822207661D7
:103B00006C75653D227E506F72744E616D6528380C
:103B1000297E22202F3E3C2F74643E0D0A20202057
:103B2000202020202020203C2F74723E0D0A2020CF
:103B300020202020202020203C74723E0D0A2020CE
:103B4000202020202020202020203C74643E266E4F
:103B50006273703B4469676974616C20506F727462
:103B6000204E616D65202331266E6273703B3C2FC1
:103B700074643E0D0A2020202020202020202020B8
:103B8000203C74643E3C696E707574206D61786C85
:103B9000656E6774683D227E4765744D61784C653B
:103BA0006E677468506F72744E616D6528297E224D
:103BB000206E616D653D22706E39222076616C75D4
:103BC000653D227E506F72744E616D652839297E85
:103BD00022202F3E3C2F74643E0D0A2020202020FE
:103BE00020202020203C2F74723E0D0A202020200F
:103BF0002020202020203C74723E0D0A202020200E
:103C000020202020202020203C74643E266E6273F9
:103C1000703B4469676974616C20506F7274204E08
:103C2000616D65202332266E6273703B3C2F746495
:103C30003E0D0A2020202020202020202020203C73
:103C400074643E3C696E707574206D61786C656E4D
:103C50006774683D227E4765744D61784C656E6778
:103C60007468506F72744E616D6528297E22206ED3
:103C7000616D653D22706E3130222076616C756514
:103C80003D227E506F72744E616D65283130297E01
:103C900022202F3E3C2F74643E0D0A20202020203D
:103CA00020202020203C2F74723E0D0A202020204E
:103CB0002020202020203C74723E0D0A202020204D
:103CC00020202020202020203C74643E266E627339
:103CD000703B4469676974616C20506F7274204E48
:103CE000616D65202333266E6273703B3C2F7464D4
:103CF0003E0D0A2020202020202020202020203CB3
:103D000074643E3C696E707574206D61786C656E8C
:103D10006774683D227E4765744D61784C656E67B7
:103D20007468506F72744E616D6528297E22206E12
:103D3000616D653D22706E3131222076616C756552
:103D40003D227E506F72744E616D65283131297E3F
:103D500022202F3E3C2F74643E0D0A20202020207C
:103D600020202020203C2F74723E0D0A202020208D
:103D70002020202020203C74723E0D0A202020208C
:103D800020202020202020203C74643E266E627378
:103D9000703B4469676974616C20506F7274204E87
:103DA000616D65202334266E6273703B3C2F746412
:103DB0003E0D0A2020202020202020202020203CF2
:103DC00074643E3C696E707574206D61786C656ECC
:103DD0006774683D227E4765744D61784C656E67F7
:103DE0007468506F72744E616D6528297E22206E52
:103DF000616D653D22706E3132222076616C756591
:103E00003D227E506F72744E616D65283132297E7D
:103E100022202F3E3C2F74643E0D0A2020202020BB
:103E200020202020203C2F74723E0D0A20202020CC
:103E30002020202020203C74723E0D0A20202020CB
:103E400020202020202020203C74643E266E6273B7
:103E5000703B4469676974616C20506F7274204EC6
:103E6000616D65202335266E6273703B3C2F746450
:103E70003E0D0A2020202020202020202020203C31
:103E800074643E3C696E707574206D61786C656E0B
:103E90006774683D227E4765744D61784C656E6736
:103EA0007468506F72744E616D6528297E22206E91
:103EB000616D653D22706E3133222076616C7565CF
:103EC0003D227E506F72744E616D65283133297EBC
:103ED00022202F3E3C2F74643E0D0A2020202020FB
:103EE00020202020203C2F74723E0D0A202020200C
:103EF0002020202020203C74723E0D0A202020200B
:103F000020202020202020203C74643E266E6273F6
:103F1000703B4469676974616C20506F7274204E05
:103F2000616D65202336266E6273703B3C2F74648E
:103F30003E0D0A2020202020202020202020203C70
:103F400074643E3C696E707574206D61786C656E4A
:103F50006774683D227E4765744D61784C656E6775
:103F60007468506F72744E616D6528297E22206ED0
:103F7000616D653D22706E3134222076616C75650D
:103F80003D227E506F72744E616D65283134297EFA
:103F900022202F3E3C2F74643E0D0A20202020203A
:103FA00020202020203C2F74723E0D0A202020204B
:103FB0002020202020203C74723E0D0A202020204A
:103FC00020202020202020203C74643E266E627336
:103FD000703B4469676974616C20506F7274204E45
:103FE000616D65202337266E6273703B3C2F7464CD
:103FF0003E0D0A2020202020202020202020203CB0
:1040000074643E3C696E707574206D61786C656E89
:104010006774683D227E4765744D61784C656E67B4
:104020007468506F72744E616D6528297E22206E0F
:10403000616D653D22706E3135222076616C75654B
:104040003D227E506F72744E616D65283135297E38
:1040500022202F3E3C2F74643E0D0A202020202079
:1040600020202020203C2F74723E0D0A202020208A
:104070002020202020203C74723E0D0A2020202089
:1040800020202020202020203C74643E266E627375
:10409000703B4469676974616C20506F7274204E84
:1040A000616D65202338266E6273703B3C2F74640B
:1040B0003E0D0A2020202020202020202020203CEF
:1040C00074643E3C696E707574206D61786C656EC9
:1040D0006774683D227E4765744D61784C656E67F4
:1040E0007468506F72744E616D6528297E22206E4F
:1040F000616D653D22706E3136222076616C75658A
:104100003D227E506F72744E616D65283136297E76
:1041100022202F3E3C2F74643E0D0A2020202020B8
:1041200020202020203C2F74723E0D0A20202020C9
:104130002020202020203C74723E0D0A20202020C8
:1041400020202020202020203C74643E266E6273B4
:10415000703B4469676974616C20506F7274204EC3
:10416000616D65202339266E6273703B3C2F746449
:104170003E0D0A2020202020202020202020203C2E
:1041800074643E3C696E707574206D61786C656E08
:104190006774683D227E4765744D61784C656E6733
:1041A0007468506F72744E616D6528297E22206E8E
:1041B000616D653D22706E3137222076616C7565C8
:1041C0003D227E506F72744E616D65283137297EB5
:1041D00022202F3E3C2F74643E0D0A2020202020F8
:1041E00020202020203C2F74723E0D0A2020202009
:1041F0002020202020203C74723E0D0A2020202008
:1042000020202020202020203C74643E266E6273F3
:10421000703B4469676974616C20506F7274204E02
:10422000616D6520233130266E6273703B3C2F74C4
:10423000643E0D0A20202020202020202020202045
:104240003C74643E3C696E707574206D61786C6579
:104250006E6774683D227E4765744D61784C656E6B
:10426000677468506F72744E616D6528297E2220D4
:104270006E616D653D22706E3138222076616C75FD
:10428000653D227E506F72744E616D65283138290C
:104290007E22202F3E3C2F74643E0D0A20202020D9
:1042A0002020202020203C2F74723E0D0A20202048
:1042B000202020202020203C74723E0D0A20202047
:1042C0002020202020202020203C74643E266E6286
:1042D00073703B4469676974616C20506F7274201D
:1042E0004E616D6520233131266E6273703B3C2F29
:1042F00074643E0D0A202020202020202020202031
:10430000203C74643E3C696E707574206D61786CFD
:10431000656E6774683D227E4765744D61784C65B3
:104320006E677468506F72744E616D6528297E22C5
:10433000206E616D653D22706E3139222076616C90
:1043400075653D227E506F72744E616D65283139FE
:10435000297E22202F3E3C2F74643E0D0A2020200F
:10436000202020202020203C2F74723E0D0A202087
:1043700020202020202020203C74723E0D0A202086
:10438000202020202020202020203C74643E266E07
:104390006273703B4469676974616C20506F72741A
:1043A000204E616D6520233132266E6273703B3C76
:1043B0002F74643E0D0A2020202020202020202061
:1043C00020203C74643E3C696E707574206D617889
:1043D0006C656E6774683D227E4765744D61784CEC
:1043E000656E677468506F72744E616D6528297EC2
:1043F00022206E616D653D22706E32302220766122
:104400006C75653D227E506F72744E616D65283209
:1044100030297E22202F3E3C2F74643E0D0A20203E
:1044200020202020202020203C2F74723E0D0A20C6
:104430002020202020202020203C74723E0D0A20C5
:1044400020202020202020202020203C74643E2694
:104450006E6273703B4469676974616C20506F725F
:1044600074204E616D6520233133266E6273703B7C
:104470003C2F74643E0D0A20202020202020202084
:104480002020203C74643E3C696E707574206D6120
:10449000786C656E6774683D227E4765744D6178FF
:1044A0004C656E677468506F72744E616D65282933
:1044B0007E22206E616D653D22706E323122207643
:1044C000616C75653D227E506F72744E616D65281A
:1044D0003231297E22202F3E3C2F74643E0D0A206B
:1044E0002020202020202020203C2F74723E0D0A06
:1044F000202020202020202020203C74723E0D0A05
:104500002020202020202020202020203C74643ED9
:10451000266E6273703B4469676974616C20506FEA
:104520007274204E616D6520233134266E62737083
:104530003B3C2F74643E0D0A2020202020202020A8
:10454000202020203C74643E3C696E707574206DA0
:1045500061786C656E6774683D227E4765744D6155
:10456000784C656E677468506F72744E616D652823
:10457000297E22206E616D653D22706E32322220CE
:1045800076616C75653D227E506F72744E616D650B
:10459000283232297E22202F3E3C2F74643E0D0AA1
:1045A000202020202020202020203C2F74723E0D2F
:1045B0000A202020202020202020203C74723E0D44
:1045C0000A2020202020202020202020203C74644D
:1045D0003E266E6273703B4469676974616C20505B
:1045E0006F7274204E616D6520233135266E6273C3
:1045F000703B3C2F74643E0D0A2020202020202098
:1046000020202020203C74643E3C696E707574202C
:104610006D61786C656E6774683D227E4765744D88
:1046200061784C656E677468506F72744E616D6529
:1046300028297E22206E616D653D22706E32332204
:104640002076616C75653D227E506F72744E616D8F
:1046500065283233297E22202F3E3C2F74643E0D84
:104660000A202020202020202020203C2F74723E71
:104670000D0A202020202020202020203C74723E83
:104680000D0A2020202020202020202020203C74E3
:10469000643E203C2F74643E0D0A20202020202000
:1046A0002020202020203C74643E3C696E7075748C
:1046B000206E616D653D22506E5376222076616CCE
:1046C00075653D22536176652220747970653D22BF
:1046D0007375626D697422202F3E3C696E7075742B
:1046E0002076616C75653D2244656661756C742247
:1046F00020747970653D22627574746F6E22206F2C
:104700006E436C69636B3D22496E6974436F6E66DC
:1047100069726D287468697329222F3E3C2F746476
:104720003E0D0A202020202020202020203C2F7415
:10473000723E0D0A20202020202020203C2F746271
:104740006F64793E0D0A2020202020203C2F7461C8
:10475000626C653E0D0A202020203C2F64643E0DD3
:104760000A20203C2F646C3E0D0A3C2F666F726D50
:104770003E0D0A0D0A3C666F726D206E616D653DDF
:104780002261646322206D6574686F643D22706FDE
:1047900073742220616374696F6E3D226164632EBD
:1047A000636769223E0D0A20203C68333E412F4456
:1047B00020436F6E766572746572205365747469F8
:1047C0006E673C2F68333E0D0A20203C646C3E0D22
:1047D0000A202020203C64643E0D0A202020202056
:1047E000203C7461626C6520626F726465723D2268
:1047F00031223E0D0A20202020202020203C7462FF
:104800006F64793E0D0A20202020202020202020C7
:104810003C74723E0D0A20202020202020202020E1
:1048200020203C74643E266E6273703B56524546AF
:104830002B266E6273703B3C2F74643E0D0A202061
:10484000202020202020202020203C74643E0D0ABF
:104850002020202020202020202020203C696E7055
:104860007574206E616D653D22767230222076610E
:104870006C75653D22494E2220747970653D227227
:104880006164696F22207E767265665F6368656326
:104890006B656428302C54525545297E202F3E41AB
:1048A0005644440D0A2020202020202020202020B3
:1048B000203C696E707574206E616D653D22767264
:1048C00030222076616C75653D224F55542220744C
:1048D0007970653D22726164696F22207E7672650F
:1048E000665F636865636B656428302C46414C5392
:1048F00045297E202F3E565265664558542B0D0A99
:104900002020202020202020202020203C2F7464E4
:104910003E0D0A202020202020202020203C2F7423
:10492000723E0D0A202020202020202020203C74D0
:10493000723E0D0A20202020202020202020202030
:104940003C74643E266E6273703B565245462D3C65
:104950002F74643E0D0A20202020202020202020BB
:1049600020203C74643E0D0A20202020202020209E
:10497000202020203C696E707574206E616D653D4D
:1049800022767231222076616C75653D22494E2275
:1049900020747970653D22726164696F22207E7691
:1049A0007265665F636865636B656428312C545279
:1049B0005545297E202F3E415653530D0A20202075
:1049C0002020202020202020203C696E707574203B
:1049D0006E616D653D22767231222076616C75655F
:1049E0003D224F55542220747970653D22726164D6
:1049F000696F22207E767265665F636865636B65AA
:104A00006428312C46414C5345297E202F3E565276
:104A100065664558542D0D0A202020202020202096
:104A2000202020203C2F74643E0D0A2020202020CE
:104A300020202020203C2F74723E0D0A20202020B0
:104A40002020202020203C74723E0D0A20202020AF
:104A500020202020202020203C74643E203C2F7405
:104A6000643E0D0A2020202020202020202020200D
:104A70003C74643E3C696E707574206E616D653D7A
:104A80002261645376222076616C75653D22536104
:104A900076652220747970653D227375626D697444
:104AA000222F3E3C696E7075742076616C75653D91
:104AB0002244656661756C742220747970653D22AC
:104AC000627574746F6E22206F6E436C69636B3D08
:104AD00022496E6974436F6E6669726D28746869E5
:104AE0007329222F3E3C2F74643E0D0A2020202083
:104AF0002020202020203C2F74723E0D0A202020F0
:104B000020202020203C2F74626F64793E0D0A2003
:104B100020202020203C2F7461626C653E0D0A200D
:104B20002020203C2F64643E0D0A20203C2F646C22
:104B30003E0D0A3C2F666F726D3E0D0A0D0A3C66F3
:104B40006F726D206E616D653D22617574686622BD
:104B5000206D6574686F643D22706F7374222061EC
:104B60006374696F6E3D22617574682E6367692294
:104B7000206F6E5375626D69743D22436865636B87
:104B8000436F6E6669726D287468697329223E0DE1
:104B90000A20203C68333E57656220536572766573
:104BA000722041757468656E7469636174696F6EB3
:104BB0002053657474696E673C2F68333E0D0A207C
:104BC000203C646C3E0D0A202020203C64643E0D95
:104BD0000A2020202020203C7461626C6520626FD6
:104BE000726465723D2231223E0D0A202020202071
:104BF0002020203C74626F64793E0D0A2020202022
:104C00002020202020203C74723E0D0A20202020ED
:104C100020202020202020203C74643E266E6273D9
:104C2000703B5573652041757468656E7469636186
:104C300074696F6E266E6273703B3C2F74643E0D18
:104C40000A2020202020202020202020203C7464C6
:104C50003E3C696E707574206E616D653D226168C1
:104C60002220747970653D22636865636B626F789A
:104C700022207E617574685F6F6E6F666628297E7C
:104C80002F3E3C2F74643E0D0A202020202020203F
:104C90002020203C2F74723E0D0A2020202020204E
:104CA000202020203C74723E0D0A2020202020204D
:104CB0002020202020203C74643E266E6273703BCE
:104CC0004E6F772050617373776F7264266E6273D4
:104CD000703B3C2F74643E0D0A20202020202020B1
:104CE00020202020203C74643E3C696E7075742046
:104CF0006D61786C656E6774683D227E4765744DA2
:104D000061784C656E6774684175746828297E22E5
:104D1000206E616D653D22707330222076616C7566
:104D2000653D227E50617373776F72642832297EED
:104D30002220747970653D2270617373776F72649D
:104D400022202F3E3C2F74643E0D0A20202020207C
:104D500020202020203C2F74723E0D0A202020208D
:104D60002020202020203C74723E0D0A202020208C
:104D700020202020202020203C74643E266E627378
:104D8000703B4E65772050617373776F7264266E47
:104D90006273703B3C2F74643E0D0A20202020205B
:104DA000202020202020203C74643E3C696E7075D9
:104DB00074206D61786C656E6774683D227E47650E
:104DC000744D61784C656E67746841757468282904
:104DD0007E22206E616D653D2270733122207661E6
:104DE0006C75653D227E50617373776F72642830F5
:104DF000297E2220747970653D2270617373776F0C
:104E0000726422202F3E3C2F74643E0D0A20202025
:104E1000202020202020203C2F74723E0D0A2020CC
:104E200020202020202020203C74723E0D0A2020CB
:104E3000202020202020202020203C74643E266E4C
:104E40006273703B436F6E6669726D20506173735D
:104E5000776F7264266E6273703B3C2F74643E0DF4
:104E60000A2020202020202020202020203C7464A4
:104E70003E3C696E707574206D61786C656E677408
:104E8000683D227E4765744D61784C656E67746835
:104E90004175746828297E22206E616D653D2270FF
:104EA0007332222076616C75653D227E506173738A
:104EB000776F72642831297E2220747970653D22D3
:104EC00070617373776F726422202F3E3C2F74647D
:104ED0003E0D0A202020202020202020203C2F745E
:104EE000723E0D0A202020202020202020203C740B
:104EF000723E0D0A2020202020202020202020206B
:104F00003C74643E266E6273703B7E5061737377AF
:104F10006F7264526573756C7428297E266E627395
:104F2000703B3C2F74643E0D0A202020202020205E
:104F300020202020203C74643E3C696E70757420F3
:104F40006E616D653D2241685376222076616C75F5
:104F5000653D22536176652220747970653D227328
:104F600075626D6974222F3E3C696E70757420768F
:104F7000616C75653D2244656661756C74222074B0
:104F80007970653D22627574746F6E22206F6E4376
:104F90006C69636B3D22496E6974436F6E6669721A
:104FA0006D287468697329222F3E3C2F74643E0D6E
:104FB0000A202020202020202020203C2F74723E18
:104FC0000D0A20202020202020203C2F74626F64B6
:104FD000793E0D0A2020202020203C2F7461626C35
:104FE000653E0D0A202020203C2F64643E0D0A20DF
:104FF000203C2F646C3E0D0A3C2F666F726D3E0D97
:105000000A0D0A3C666F726D206E616D653D226E01
:10501000747022206D6574686F643D22706F7374C4
:105020002220616374696F6E3D226E74702E636717
:1050300069223E0D0A20203C68333E4E54502053D6
:10504000657474696E673C2F68333E0D0A20203CFE
:10505000646C3E0D0A202020203C64643E0D0A2032
:1050600020202020203C7461626C6520626F726495
:1050700065723D2231223E0D0A2020202020202072
:10508000203C74626F64793E0D0A2020202020208D
:10509000202020203C74723E0D0A20202020202059
:1050A0002020202020203C74643E266E6273703BDA
:1050B0004E545020736572766572266E6273703B33
:1050C0003C2F74643E0D0A20202020202020202028
:1050D0002020203C74643E3C696E707574206D61C4
:1050E000786C656E6774683D227E4765744D6178A3
:1050F0004C656E6774684E545028297E22206E617C
:105100006D653D226E7470222076616C75653D225E
:105110007E4E545073657276657228297E22207403
:105120007970653D227465787422202F3E3C2F747F
:10513000643E0D0A202020202020202020203C2F0B
:1051400074723E0D0A202020202020202020203CA8
:1051500074723E0D0A2020202020202020202020B4
:10516000203C74643E203C2F74643E0D0A202020B5
:105170002020202020202020203C74643E3C696EAA
:10518000707574206E616D653D226E7453762220B9
:1051900076616C75653D2253617665222074797065
:1051A000653D227375626D6974222F3E3C696E7095
:1051B00075742076616C75653D2244656661756C19
:1051C000742220747970653D22627574746F6E224A
:1051D000206F6E436C69636B3D22496E6974436F47
:1051E0006E6669726D287468697329222F3E3C2FA0
:1051F00074643E0D0A202020202020202020203C06
:105200002F74723E0D0A20202020202020203C2FC9
:1052100074626F64793E0D0A2020202020203C2FEC
:105220007461626C653E0D0A202020203C2F64646E
:105230003E0D0A20203C2F646C3E0D0A20203C6865
:1052400072202F3E3C6272202F3E0D0A3C2F666F6B
:10525000726D3E0D0A3C666F726D206D6574686FED
:10526000643D226765742220616374696F6E3D221C
:10527000636F6E6669672E636769223E0D0A2020A0
:105280003C68333E3C2F68333E0D0A20203C646C62
:105290003E0D0A202020203C64643E203C696E7054
:1052A00075742076616C75653D22476F746F204977
:1052B0006E646578205061676522206E616D653D82
:1052C00022676F5F696E6465782220747970653D2E
:1052D000227375626D697422202F3E3C2F64643EF8
:1052E0000D0A20203C2F646C3E0D0A3C2F666F7225
:1052F0006D3E0D0A3C2F626F64793E0D0A3C2F68AB
:10530000746D6C3E0D0AE5040000000000008D0580
:10531000000001000000DD0500000200000076062C
:105320000000030000001407000004000000BD0797
:105330000000050000006A080000060000000909DE
:10534000000007000000B609000008000000160A6F
:10535000000009000000B40A00000A000000140B5D
:1053600000000B000000B00B00000C000000100C4F
:1053700000000D000000A90C00000E000000090D47
:1053800000000F0000004F0F000010000000A50FEC
:105390000000110000007510000012000000CB108A
:1053A0000000130000008D11000014000000E31144
:1053B000000015000000A512000016000000FB12FE
:1053C000000017000000BD130000180000001314B7
:1053D000000019000000D51400001A0000002B1571
:1053E00000001B000000ED1500001C00000043162B
:1053F00000001D000000051700001E0000005B17E4
:1054000000001F00000017180000200000006D18A9
:105410000000210000002F19000022000000851963
:10542000000023000000491A000024000000A11A17
:10543000000025000000601B000026000000B81BD3
:10544000000027000000771C000028000000CF1C8F
:105450000000290000008E1D00002A000000E61D4B
:1054600000002B000000A51E00002C000000FD1E07
:1054700000002D000000BC1F00002E0000001420C2
:1054800000002F00000037220000300000006322DF
:10549000000031000000F422000030000000202352
:1054A000000032000000B123000030000000DD23C6
:1054B0000000330000006E240000300000009A2439
:1054C0000000340000002B250000300000005725AC
:1054D000000035000000E825000030000000142620
:1054E000000036000000A526000030000000D12694
:1054F00000003700000062270000300000008E2707
:1055000000003800000020280000300000004C2877
:10551000000039000000DE280000300000000A29E9
:1055200000003A0000009C29000030000000C9295A
:1055300000003B0000005C2A000030000000892AC7
:1055400000003C0000001C2B000030000000492B34
:1055500000003D000000DC2B000030000000092CA2
:1055600000003E0000009C2C000030000000C92C10
:1055700000003F0000005C2D000030000000892D7D
:105580000000400000001C2E000030000000492EEA
:10559000000041000000DC2E000030000000092F58
:1055A0000000420000009D2F000030000000CA2FC4
:1055B0000000430000005E300000300000008B302F
:1055C0000000440000001F310000300000004C319A
:1055D000000045000000E0310000300000000D3206
:1055E000000046000000A132000030000000CE3272
:1055F00000004700000062330000300000008F33DD
:10560000000048000000CD350000490000002336AE
:1056100000004A000000E53600004B0000003B3768
:1056200000004C000000B93900004D000000423A73
:1056300000004E0000006A3A00004F000000043BEA
:1056400000004E0000002C3B000050000000CA3B50
:1056500000004E000000F23B000051000000513CF1
:10566000000052000000303E000053000000573E92
:105670000000540000002530363C21444F4354596B
:1056800050452048544D4C205055424C494320220F
:105690002D2F2F5733432F2F4454442048544D4C23
:1056A00020342E3031205472616E736974696F6ECC
:1056B000616C2F2F454E223E0A3C68746D6C206C45
:1056C000616E673D226A61223E0A093C6865616439
:1056D0003E0A09093C6D65746120687474702D651B
:1056E000717569763D22436F6E74656E742D5479C1
:1056F00070652220636F6E74656E743D22746578E8
:10570000742F68746D6C3B20636861727365743DBF
:1057100053686966745F4A4953223E0A09093C6D21
:1057200065746120687474702D65717569763D22A9
:10573000707261676D612220636F6E74656E743D77
:10574000226E6F2D6361636865223E0A09093C6D14
:1057500065746120687474702D65717569763D2279
:1057600063616368652D636F6E74726F6C22206372
:105770006F6E74656E743D226E6F2D636163686534
:10578000223E0A09093C7469746C653E5049432DF8
:105790004E494320504943204E6574776F726B2009
:1057A000496E7465726661636520436172643C2F63
:1057B0007469746C653E0A0A09093C736372697006
:1057C00074206C616E67756167653D224A61766120
:1057D000536372697074223E0A0909093C212D2D18
:1057E0000A09090966756E6374696F6E20496E69EE
:1057F00074436F6D6669726D287061727473290AE3
:105800000909097B0A0909096D79526574203D204F
:10581000636F6E6669726D2822446F20796F752000
:10582000696E697469616C697A652074686973204E
:1058300073657474696E67203F22290A0909096932
:10584000662028206D79526574203D3D2074727564
:105850006520290A0909097B0A090909706172741E
:10586000732E666F726D2E7375626D697428293B95
:105870000A0909097D0A0909097D0A0909092D2D65
:105880003E0A09093C2F7363726970743E0A093C31
:105890002F686561643E0A0A093C626F64793E0ABA
:1058A00009093C666F6E742073697A653D222B325C
:1058B000223E0A09093C7370616E207374796C652D
:1058C0003D22666F6E742D7765696768743A206251
:1058D0006F6C643B223E5049432D4E49433C2F732D
:1058E00070616E3E3C62723E3C62723E0A09095033
:1058F000494331384638374A3530204E6574776F22
:10590000726B20496E7465726661636520436172D3
:10591000642056657273696F6E207E426F61726497
:1059200056657273696F6E28297E3C2F666F6E74A0
:105930003E0A09093C68723E0A09093C68333E493F
:105940002F4F20506F7274733C2F68333E0A090941
:105950003C646C3E0A09093C64643E0A09093C64E3
:105960006976207374796C653D22746578742D6155
:105970006C69676E3A2063656E7465723B223E3CCB
:105980002F6469763E0A09093C666F726D206D6569
:1059900074686F643D2267657420222061637469B6
:1059A0006F6E3D226D6F646966792E636769223E72
:1059B000203C62723E0A09093C68343E506F7274A2
:1059C0002D313C2F68343E0A09093C7461626C65D4
:1059D00020626F726465723D2231223E0A09093CE1
:1059E00074626F64793E0A09093C74723E0A0909BF
:1059F0003C7464207374796C653D22746578742DF1
:105A0000616C69676E3A2063656E7465723B223E15
:105A1000506F72743C2F74643E0A09093C74642010
:105A20007374796C653D22746578742D616C696757
:105A30006E3A2063656E7465723B223E56616C75EA
:105A4000653C2F74643E0A09093C2F74723E0A09B2
:105A5000093C74723E0A09093C74643E266E627306
:105A6000703B7E506F72744E616D652830297E26C2
:105A70006E6273703B5B7E416E616C6F675452491E
:105A8000532830297E5D266E6273703B3C2F746410
:105A90003E0A09093C7464207374796C653D227474
:105AA0006578742D616C69676E3A207269676874F5
:105AB0003B223E266E6273703B7E416E616C6F6767
:105AC000496E7075742830297E266E6273703B3C77
:105AD0002F74643E0A09093C2F74723E0A09093C7E
:105AE00074723E0A09093C74643E266E6273703B10
:105AF0007E506F72744E616D652831297E266E620C
:105B000073703B5B7E416E616C6F675452495328E2
:105B100031297E5D266E6273703B3C2F74643E0AB1
:105B200009093C7464207374796C653D227465784E
:105B3000742D616C69676E3A2072696768743B22E4
:105B40003E266E6273703B7E416E616C6F67496E7C
:105B50007075742831297E266E6273703B3C2F74F9
:105B6000643E0A09093C2F74723E0A09093C7472AA
:105B70003E0A09093C74643E266E6273703B7E5097
:105B80006F72744E616D652832297E266E62737065
:105B90003B5B7E416E616C6F6754524953283229DA
:105BA0007E5D266E6273703B3C2F74643E0A090969
:105BB0003C7464207374796C653D22746578742D2F
:105BC000616C69676E3A2072696768743B223E2691
:105BD0006E6273703B7E416E616C6F67496E70756B
:105BE000742832297E266E6273703B3C2F74643EAB
:105BF0000A09093C2F74723E0A09093C74723E0A74
:105C000009093C74643E266E6273703B7E506F726D
:105C1000744E616D652833297E266E6273703B5B1E
:105C20007E416E616C6F67545249532833297E5D03
:105C3000266E6273703B3C2F74643E0A09093C7403
:105C400064207374796C653D22746578742D616C81
:105C500069676E3A2072696768743B223E266E62FD
:105C600073703B7E416E616C6F67496E707574280E
:105C700033297E266E6273703B3C2F74643E0A09A2
:105C8000093C2F74723E0A09093C74723E0A0909E4
:105C90003C74643E266E6273703B7E506F72744E2D
:105CA000616D652838297E266E6273703B5B7E4489
:105CB00069676974616C545249532830297E5D26A6
:105CC0006E6273703B3C2F74643E0A09093C746435
:105CD0003E266E6273703B7E4469676974616C50E6
:105CE0004F525428302C54525545297E0A09093CFC
:105CF000696E707574207E4469676974616C53774E
:105D000044697361626C65642830297E206E616D20
:105D1000653D225030222076616C75653D227E44BF
:105D200069676974616C504F525428302C46414C5D
:105D30005345297E2220747970653D227375626D0A
:105D40006974223E3C2F74643E0A09093C2F747228
:105D50003E0A09093C74723E0A09093C74643E26F5
:105D60006E6273703B7E506F72744E616D65283940
:105D7000297E266E6273703B5B7E4469676974613D
:105D80006C545249532831297E5D266E6273703BF4
:105D90003C2F74643E0A09093C74643E266E6273AB
:105DA000703B7E4469676974616C504F525428316E
:105DB0002C54525545297E0A09093C696E70757448
:105DC000207E4469676974616C53774469736162CA
:105DD0006C65642831297E206E616D653D225031ED
:105DE000222076616C75653D227E44696769746125
:105DF0006C504F525428312C46414C5345297E2239
:105E000020747970653D227375626D6974223E3C21
:105E10002F74643E0A09093C2F74723E0A09093C3A
:105E200074723E0A09093C74643E266E6273703BCC
:105E30007E506F72744E616D65283130297E266EFA
:105E40006273703B5B7E4469676974616C5452494C
:105E5000532832297E5D266E6273703B3C2F74643A
:105E60003E0A09093C74643E266E6273703B7E44B0
:105E700069676974616C504F525428322C545255E2
:105E800045297E0A09093C696E707574207E446953
:105E9000676974616C537744697361626C656428E7
:105EA00032297E206E616D653D225032222076615E
:105EB0006C75653D227E4469676974616C504F5210
:105EC0005428322C46414C5345297E222074797047
:105ED000653D227375626D6974223E3C2F74643E89
:105EE0000A09093C2F74723E0A09093C74723E0A81
:105EF00009093C74643E266E6273703B7E506F727B
:105F0000744E616D65283131297E266E6273703B57
:105F10005B7E4469676974616C5452495328332924
:105F20007E5D266E6273703B3C2F74643E0A0909E5
:105F30003C74643E266E6273703B7E44696769748C
:105F4000616C504F525428332C54525545297E0AC7
:105F500009093C696E707574207E446967697461D3
:105F60006C537744697361626C65642833297E20C1
:105F70006E616D653D225033222076616C75653D02
:105F8000227E4469676974616C504F525428332CE7
:105F900046414C5345297E2220747970653D227319
:105FA00075626D6974223E3C2F74643E0A09093C97
:105FB0002F74723E0A09093C74723E0A09093C7446
:105FC000643E266E6273703B7E506F72744E616DDC
:105FD00065283132297E266E6273703B5B7E446990
:105FE000676974616C545249532834297E5D266E6A
:105FF0006273703B3C2F74643E0A09093C74643E32
:10600000266E6273703B7E4469676974616C504FA1
:10601000525428342C54525545297E0A09093C69AA
:106020006E707574207E4469676974616C5377443F
:10603000697361626C65642834297E206E616D65C8
:106040003D225034222076616C75653D227E446984
:10605000676974616C504F525428342C46414C533C
:1060600045297E2220747970653D227375626D69C1
:1060700074223E3C2F74643E0A09093C2F74723E20
:106080000A09093C74723E0A09093C74643E266E92
:106090006273703B7E506F72744E616D6528313350
:1060A000297E266E6273703B5B7E4469676974610A
:1060B0006C545249532835297E5D266E6273703BBD
:1060C0003C2F74643E0A09093C74643E266E627378
:1060D000703B7E4469676974616C504F5254283537
:1060E0002C54525545297E0A09093C696E70757415
:1060F000207E4469676974616C5377446973616297
:106100006C65642835297E206E616D653D225035B1
:10611000222076616C75653D227E446967697461F1
:106120006C504F525428352C46414C5345297E2201
:1061300020747970653D227375626D6974223E3CEE
:106140002F74643E0A09093C2F74723E0A09093C07
:1061500074723E0A09093C74643E266E6273703B99
:106160007E506F72744E616D65283134297E266EC3
:106170006273703B5B7E4469676974616C54524919
:10618000532836297E5D266E6273703B3C2F746403
:106190003E0A09093C74643E266E6273703B7E447D
:1061A00069676974616C504F525428362C545255AB
:1061B00045297E0A09093C696E707574207E446920
:1061C000676974616C537744697361626C656428B4
:1061D00036297E206E616D653D2250362220766123
:1061E0006C75653D227E4469676974616C504F52DD
:1061F0005428362C46414C5345297E222074797010
:10620000653D227375626D6974223E3C2F74643E55
:106210000A09093C2F74723E0A09093C74723E0A4D
:1062200009093C74643E266E6273703B7E506F7247
:10623000744E616D65283135297E266E6273703B20
:106240005B7E4469676974616C54524953283729ED
:106250007E5D266E6273703B3C2F74643E0A0909B2
:106260003C74643E266E6273703B7E446967697459
:10627000616C504F525428372C54525545297E0A90
:1062800009093C696E707574207E446967697461A0
:106290006C537744697361626C65642837297E208A
:1062A0006E616D653D225037222076616C75653DCB
:1062B000227E4469676974616C504F525428372CB0
:1062C00046414C5345297E2220747970653D2273E6
:1062D00075626D6974223E3C2F74643E0A09093C64
:1062E0002F74723E0A09093C74723E0A09093C7413
:1062F000643E203C2F74643E0A09093C74643E3CB1
:10630000696E7075742076616C75653D2252656C9E
:106310006F616422206E616D653D2252454C4F4194
:10632000442220747970653D227375626D69742210
:106330003E3C2F74643E0A09093C2F74723E0A09E0
:10634000093C2F74626F64793E0A09093C2F74611D
:10635000626C653E0A09093C2F666F726D3E0A0940
:10636000093C2F64643E0A09093C64643E0A090939
:106370003C646976207374796C653D227465787429
:106380002D616C69676E3A2063656E7465723B229D
:106390003E3C2F6469763E0A0909203C666F726DA7
:1063A000206D6574686F643D2267657420222061EA
:1063B0006374696F6E3D226D6F646966792E6367E1
:1063C00069223E3C62723E0A09093C68343E506FC5
:1063D00072742D323C2F68343E0A09093C746162A4
:1063E0006C6520626F726465723D2231223E0A093B
:1063F000093C74626F64793E0A09093C74723E0A72
:1064000009093C7464207374796C653D2274657865
:10641000742D616C69676E3A2063656E7465723BBA
:10642000223E506F72743C2F74643E0A09093C741A
:1064300064207374796C653D22746578742D616C89
:1064400069676E3A2063656E7465723B223E5661E1
:106450006C75653C2F74643E0A09093C2F74723ECA
:106460000A09093C74723E0A09093C74643E266EAE
:106470006273703B7E506F72744E616D6528342973
:106480007E266E6273703B5B7E416E616C6F6754FB
:106490005249532834297E5D266E6273703B3C2F2F
:1064A00074643E0A09093C7464207374796C653D18
:1064B00022746578742D616C69676E3A2072696721
:1064C00068743B223E266E6273703B7E416E616C47
:1064D0006F67496E7075742834297E266E627370FA
:1064E0003B3C2F74643E0A09093C2F74723E0A0932
:1064F000093C74723E0A09093C74643E266E62735C
:10650000703B7E506F72744E616D652835297E2612
:106510006E6273703B5B7E416E616C6F6754524973
:10652000532835297E5D266E6273703B3C2F746460
:106530003E0A09093C7464207374796C653D2274C9
:106540006578742D616C69676E3A2072696768744A
:106550003B223E266E6273703B7E416E616C6F67BC
:10656000496E7075742835297E266E6273703B3CC7
:106570002F74643E0A09093C2F74723E0A09093CD3
:1065800074723E0A09093C74643E266E6273703B65
:106590007E506F72744E616D652836297E266E625C
:1065A00073703B5B7E416E616C6F67545249532838
:1065B00036297E5D266E6273703B3C2F74643E0A02
:1065C00009093C7464207374796C653D22746578A4
:1065D000742D616C69676E3A2072696768743B223A
:1065E0003E266E6273703B7E416E616C6F67496ED2
:1065F0007075742836297E266E6273703B3C2F744A
:10660000643E0A09093C2F74723E0A09093C7472FF
:106610003E0A09093C74643E266E6273703B7E50EC
:106620006F72744E616D652837297E266E627370B5
:106630003B5B7E416E616C6F67545249532837292A
:106640007E5D266E6273703B3C2F74643E0A0909BE
:106650003C7464207374796C653D22746578742D84
:10666000616C69676E3A2072696768743B223E26E6
:106670006E6273703B7E416E616C6F67496E7075C0
:10668000742837297E266E6273703B3C2F74643EFB
:106690000A09093C2F74723E0A09093C74723E0AC9
:1066A00009093C74643E266E6273703B7E506F72C3
:1066B000744E616D65283136297E266E6273703B9B
:1066C0005B7E4469676974616C5452495328382968
:1066D0007E5D266E6273703B3C2F74643E0A09092E
:1066E0003C74643E266E6273703B7E4469676974D5
:1066F000616C504F525428382C54525545297E0A0B
:1067000009093C696E707574207E4469676974611B
:106710006C537744697361626C65642838297E2004
:106720006E616D653D225038222076616C75653D45
:10673000227E4469676974616C504F525428382C2A
:1067400046414C5345297E2220747970653D227361
:1067500075626D6974223E3C2F74643E0A09093CDF
:106760002F74723E0A09093C74723E0A09093C748E
:10677000643E266E6273703B7E506F72744E616D24
:1067800065283137297E266E6273703B5B7E4469D3
:10679000676974616C545249532839297E5D266EAD
:1067A0006273703B3C2F74643E0A09093C74643E7A
:1067B000266E6273703B7E4469676974616C504FEA
:1067C000525428392C54525545297E0A09093C69EE
:1067D0006E707574207E4469676974616C53774488
:1067E000697361626C65642839297E206E616D650C
:1067F0003D225039222076616C75653D227E4469C8
:10680000676974616C504F525428392C46414C537F
:1068100045297E2220747970653D227375626D6909
:1068200074223E3C2F74643E0A09093C2F74723E68
:106830000A09093C74723E0A09093C74643E266EDA
:106840006273703B7E506F72744E616D6528313893
:10685000297E266E6273703B5B7E44696769746152
:106860006C54524953283130297E5D266E62737014
:106870003B3C2F74643E0A09093C74643E266E62F8
:1068800073703B7E4469676974616C504F52542841
:1068900031302C54525545297E0A09093C696E70E5
:1068A0007574207E4469676974616C5377446973B9
:1068B00061626C6564283130297E206E616D653DB2
:1068C00022503130222076616C75653D227E44690C
:1068D000676974616C504F52542831302C46414CDA
:1068E0005345297E2220747970653D227375626D4F
:1068F0006974223E3C2F74643E0A09093C2F74726D
:106900003E0A09093C74723E0A09093C74643E2639
:106910006E6273703B7E506F72744E616D6528318C
:1069200039297E266E6273703B5B7E4469676974A9
:10693000616C54524953283131297E5D266E627351
:10694000703B3C2F74643E0A09093C74643E266E19
:106950006273703B7E4469676974616C504F525436
:106960002831312C54525545297E0A09093C696E5B
:10697000707574207E4469676974616C53774469EB
:106980007361626C6564283131297E206E616D65AA
:106990003D22503131222076616C75653D227E4466
:1069A00069676974616C504F52542831312C4641EB
:1069B0004C5345297E2220747970653D227375629F
:1069C0006D6974223E3C2F74643E0A09093C2F74A1
:1069D000723E0A09093C74723E0A09093C74643E1D
:1069E000266E6273703B7E506F72744E616D6528C7
:1069F0003230297E266E6273703B5B7E4469676924
:106A000074616C54524953283132297E5D266E627E
:106A100073703B3C2F74643E0A09093C74643E2643
:106A20006E6273703B7E4469676974616C504F524B
:106A3000542831322C54525545297E0A09093C69A3
:106A40006E707574207E4469676974616C53774415
:106A5000697361626C6564283132297E206E616DD4
:106A6000653D22503132222076616C75653D227E73
:106A70004469676974616C504F52542831322C4616
:106A8000414C5345297E2220747970653D227375EF
:106A9000626D6974223E3C2F74643E0A09093C2FE2
:106AA00074723E0A09093C74723E0A09093C746416
:106AB0003E266E6273703B7E506F72744E616D65E0
:106AC000283231297E266E6273703B5B7E44696793
:106AD0006974616C54524953283133297E5D266EA6
:106AE0006273703B3C2F74643E0A09093C74643E37
:106AF000266E6273703B7E4469676974616C504FA7
:106B000052542831332C54525545297E0A09093CE8
:106B1000696E707574207E4469676974616C53771F
:106B200044697361626C6564283133297E206E612B
:106B30006D653D22503133222076616C75653D22B2
:106B40007E4469676974616C504F52542831332C0C
:106B500046414C5345297E2220747970653D22734D
:106B600075626D6974223E3C2F74643E0A09093CCB
:106B70002F74723E0A09093C74723E0A09093C747A
:106B8000643E266E6273703B7E506F72744E616D10
:106B900065283232297E266E6273703B5B7E4469C3
:106BA000676974616C54524953283134297E5D26DB
:106BB0006E6273703B3C2F74643E0A09093C746436
:106BC0003E266E6273703B7E4469676974616C50E7
:106BD0004F52542831342C54525545297E0A090904
:106BE0003C696E707574207E4469676974616C538A
:106BF0007744697361626C6564283134297E206E44
:106C0000616D653D22503134222076616C75653DA1
:106C1000227E4469676974616C504F525428313444
:106C20002C46414C5345297E2220747970653D22C3
:106C30007375626D6974223E3C2F74643E0A0909C3
:106C40003C2F74723E0A09093C74723E0A09093CE1
:106C500074643E266E6273703B7E506F72744E6138
:106C60006D65283233297E266E6273703B5B7E44ED
:106C700069676974616C54524953283135297E5DC6
:106C8000266E6273703B3C2F74643E0A09093C74A3
:106C9000643E266E6273703B7E4469676974616C02
:106CA000504F52542831352C54525545297E0A09EB
:106CB000093C696E707574207E4469676974616C03
:106CC000537744697361626C6564283135297E208D
:106CD0006E616D653D22503135222076616C75659F
:106CE0003D227E4469676974616C504F525428316B
:106CF000352C46414C5345297E2220747970653DE0
:106D0000227375626D6974223E3C2F74643E0A09D9
:106D1000093C2F74723E0A09093C74723E0A090943
:106D20003C74643E203C2F74643E0A09093C746440
:106D30003E3C696E7075742076616C75653D2252BB
:106D4000656C6F616422206E616D653D2252454C19
:106D50004F4144302220747970653D227375626D15
:106D60006974223E3C2F74643E0A09093C2F7472F8
:106D70003E0A09093C2F74626F64793E0A09093C96
:106D80002F7461626C653E0A0A09093C2F666F72B6
:106D90006D3E0A09093C2F64643E0A09093C2F64D0
:106DA0006C3E0A0A09093C666F726D206D65746855
:106DB0006F643D22706F73742220616374696F6E1B
:106DC0003D226C63642E636769223E0A0909093C0F
:106DD00068333E4C43443C2F68333E0A0909093C62
:106DE000646C3E0A090909093C64643E0A09090900
:106DF00009093C7461626C6520626F726465723D62
:106E00002231223E0A0909090909093C74626F64AA
:106E1000793E0A090909090909093C74723E0A09FF
:106E2000090909090909093C74643E266E627370F8
:106E30003B4C696E652031266E6273703B3C2F744B
:106E4000643E0A09090909090909093C74643E3CC0
:106E5000696E707574206E616D653D226C31222003
:106E600076616C75653D227E4C43446C696E652885
:106E700030297E22206D61786C656E6774683D22D2
:106E800031362220747970653D2274657874223E13
:106E90003C2F74643E0A090909090909093C2F7449
:106EA000723E0A090909090909093C74723E0A0976
:106EB000090909090909093C74643E266E62737068
:106EC0003B4C696E652032266E6273703B3C2F74BA
:106ED000643E0A09090909090909093C74643E3C30
:106EE000696E707574206E616D653D226C32222072
:106EF00076616C75653D227E4C43446C696E6528F5
:106F000031297E22206D61786C656E6774683D2240
:106F100031362220747970653D2274657874223E82
:106F20003C2F74643E0A090909090909093C2F74B8
:106F3000723E0A090909090909093C74723E0A09E5
:106F4000090909090909093C74643E203C2F74644D
:106F50003E0A09090909090909093C74643E3C69AA
:106F60006E707574206E616D653D224C63537622A0
:106F70002076616C75653D2253656E6422207479BC
:106F800070653D227375626D6974223E3C696E7056
:106F900075742076616C75653D2244656661756C1B
:106FA0007422206F6E636C69636B3D22496E697455
:106FB000436F6D6669726D28746869732922207445
:106FC0007970653D22627574746F6E223E3C2F7439
:106FD000643E0A090909090909093C2F74723E0A2D
:106FE0000909090909093C2F74626F64793E0A098D
:106FF000090909093C2F7461626C653E0A09090997
:10700000093C2F64643E0A0909093C2F646C3E0A5E
:1070100009093C2F666F726D3E0A0A09093C666FCA
:10702000726D206D6574686F643D226765742220FF
:10703000616374696F6E3D22636F6E6669672E636C
:107040006769223E0A0909093C68333E436F6E6650
:10705000696775726174696F6E3C2F68333E0A0907
:1070600009093C646C3E0A090909093C64643E3C18
:10707000696E7075742076616C75653D22476F741A
:107080006F20436F6E66696775726174696F6E20F9
:107090005061676522206E616D653D22676F5F6399
:1070A0006F6E662220747970653D227375626D691A
:1070B00074223E3C2F64643E0A0909093C2F646C2B
:1070C0003E0A09093C2F666F726D3E0A0A09093CA7
:1070D00068723E0A0909436F70797269676874289B
:1070E000432920323031302D323031312062792045
:1070F0003C6120687265663D22687474703A2F2F77
:107100007777772E74726973746174652E6E652E4D
:107110006A70223E547269537461746520436F2E05
:107120002C4C74642E3C2F613E3C62723E0A093C3A
:107130002F626F64793E0A3C2F68746D6C3E0AA121
:1071400002000055000000E903000031000000FDCE
:1071500003000056000000400400005700000077C4
:10716000040000320000008B04000058000000CE34
:10717000040000590000000505000033000000195C
:107180000500005A0000005C0500005B0000009351
:1071900005000034000000A70500005C000000EAC4
:1071A0000500005D000000210600003900000035E8
:1071B000060000660000005E060000670000007D1B
:1071C00006000068000000A506000069000000EC51
:1071D0000600003A000000000700006A00000029D5
:1071E0000700006B000000480700006C0000007002
:1071F0000700006D000000B70700003B000000CC56
:107200000700006E000000F50700006F000000148A
:10721000080000700000003C0800007100000083BE
:107220000800003C0000009808000072000000C147
:1072300008000073000000E008000074000000086F
:10724000090000750000004F0900003D00000064C7
:10725000090000760000008D09000077000000ACF6
:1072600009000078000000D4090000790000001B2C
:107270000A00003E000000300A00007A00000059B9
:107280000A00007B000000780A00007C000000A0DB
:107290000A00007D000000E70A00003F000000FC3B
:1072A0000A00007E000000250B00007F0000004463
:1072B0000B0000800000006C0B000081000000B398
:1072C0000B000040000000C80B000082000000F12D
:1072D0000B000083000000100C0000840000003848
:1072E0000C000085000000FB0D0000350000000FC1
:1072F0000E00005E000000520E00005F00000089DA
:107300000E0000360000009D0E000060000000E04E
:107310000E000061000000170F0000370000002B76
:107320000F0000620000006E0F000063000000A567
:107330000F000038000000B90F000064000000FCDE
:107340000F000065000000331000004100000048FD
:1073500010000086000000711000008700000090FF
:1073600010000088000000B810000089000000FF35
:1073700010000042000000141100008A0000003DCF
:107380001100008B0000005C1100008C00000084E4
:107390001100008D000000CB11000043000000E050
:1073A0001100008E0000000A1200008F0000002A69
:1073B0001200009000000054120000910000009C98
:1073C00012000044000000B112000092000000DB37
:1073D00012000093000000FB120000940000002542
:1073E000130000950000006D1300004500000082AE
:1073F00013000096000000AC13000097000000CCC2
:1074000013000098000000F6130000990000003EF1
:1074100014000046000000531400009A0000007D94
:107420001400009B0000009D1400009C000000C799
:107430001400009D0000000F15000047000000240C
:107440001500009E0000004E1500009F0000006E19
:10745000150000A000000098150000A1000000E049
:1074600015000048000000F5150000A20000001FF4
:10747000160000A30000003F160000A400000069F1
:10748000160000A5000000EE170000A60000007E18
:10749000180000A70000002530330D0A25303125E3
:0774A00030352530390D0ADB
:0174A70000E4
:0874A80015EC51F0FE0EDB5063
:1074B0000701A25D22E0FE0EA25D0CE01C0EE66E4E
:1074C000E66AC10EE66E030EE66EA2514EEC57F070
:1074D00082EC53F0FE0EDBCFA2F7DB50FE080DE08E
:1074E0001C0EE66EE66AFE0EDB504EEC57F0C10E47
:1074F000E66E030EE66E82EC53F01AEF51F00701D0
:10750000A251A35D01E11200FE0EA35D19E0270E5A
:10751000E66EE66A010EE66E9A0EE66E030E2DEC3E
:1075200054F01B0E3EEC51F0EF502DEC54F0CAEC31
:1075300052F0270E86EC55F0C4EC54F0C1EC56F036
:10754000A2C7A3F7270EE66EE66ADCC3E6FFC1C357
:1075500014F0C2C315F086EC55F0C4EC54F0010EE3
:10756000E66E9A0EE66E030EE66EC1EF56F015EC6F
:1075700051F00B0EE126670EF36E090EF3CFDBFF21
:10758000150EF36E0A0EF3CFDBFF0301985199112C
:107590000FE162EC9DF006C098F307C099F3FF0E6F
:1075A00003019817070E9917000E9827040E9923C8
:1075B0003C0EE66EE66AE66AC40EE66E020EE66E03
:1075C000D2ECD8F0146E050EE15E1450010EDB6AA9
:1075D000DF6AFFEC51F001E392D0B1EC53F01EEC06
:1075E00051F07AEC51F0F62A000EF722F82208004A
:1075F000080EF5CFDBFF1EEC51F07AEC51F0020ED5
:10760000F626000EF722F8220900020EF5CFDBFF66
:107610000A00030EF5CFDBFF1EEC51F0F5EC57F03E
:10762000040EF626000EF722F8220900040EF5CF0C
:10763000DBFF0A00050EF5CFDBFF080EDB502BE168
:10764000090EDBCF08F00A0E6BEC53F022EC57F07A
:10765000270E1626000E1722ECEC55F0040E4AEC0D
:1076600057F0050EDB50172051EC51F0D950090F9F
:1076700036EC56F0090EDBCF14F00A0E14EC54F081
:10768000D8807D0E14541F0E1554000E1654000E93
:10769000175402E2EFD7FFD7080EDBCFDCF3060E5C
:1076A000DBCFC1F3070EDBCFC2F3270E0301C127E7
:1076B000000EC223020EDB50C125C36F030EDB5048
:1076C000C221C46F010EC327000EC423040EDB5079
:1076D000C325C56F050EDB50C421C66F0D0ED76FD5
:1076E000D8970DDF1EEC51F004C017F0F5EC57F001
:1076F0000800F5CFC0F325EC49F0DF2A6AD70B0E5E
:10770000E15C02E2E16AE552E16E1AEF51F015EC3C
:1077100051F0E652DF6AFFEC51F001E392D0B1EC98
:1077200053F00D0E0301D75D01E089D0E8DEF70EBE
:10773000DB500301C05D01E082D0180EBD6F020E68
:10774000BE6FFA0EDB5010E1F80EDBCFAAF3F90E94
:10775000DBCFABF3D887040ED76FF80EDBCFDAF3AD
:10776000F90EDBCFDBF369D0000E985D040E99595A
:1077700006E3880ED8809855130E995503E2986B4E
:10778000040E996F98C3AAF399C3ABF3982B000E1C
:107790009923F80EDBCFA8F3F90EDBCFA9F346EC63
:1077A00056F00301D889FA0EDB50040A2AE0070AD2
:1077B00012E0020A02E0030A40E1D9EC53F0FA0EAB
:1077C000DB50020802E0000E01D0010EBC95E8B0CB
:1077D000BC85D76B32D0FB0EDBCF18F0FC0EDBCFB5
:1077E00019F0FD0EDB501824166EFE0EDB5019202A
:1077F00005EC53F0D9EC53F08AEC55F0020ED76F3C
:107800001CD0B1EC51F0020E3EEC51F0EECF18F06E
:10781000EFCF19F0B1EC51F01850EE24166E19505C
:10782000EE2005EC53F074EC57F00301050ED76F12
:10783000010EE66E020E46EC51F0DF5003D0DF2A57
:107840006AD7FE0EE5521AEF51F0D7EC56F003015D
:10785000D9A903D0D999010E01D0000E1AEF51F029
:10786000D7EC56F0070E0301D75D02E0000E01D001
:10787000010E1AEF51F0D7EC56F0F1EC55F0030180
:10788000D751080A32E0010A30E0050A2EE0020A68
:1078900029E0050A1CE00D0A0FE0010A0DE0070AC5
:1078A00028E0020A26E0010A24E0060A22E0040A8F
:1078B0001CE17AECC8F01DD07AEC57F006E0A65136
:1078C000C719FAE1A751C819F7E1080E0CD07AECF4
:1078D00057F006E0A651C719FAE1A751C819F7E118
:1078E0000C0E01D00D0ED76F06D0E66A140E46ECD2
:1078F00051F025EC49F01AEF51F0D7EC56F00301A6
:10790000D89775EC56F0B7DFE5521AEF51F0D7EC87
:1079100056F0F5DD14EC56F0B7EC53F0DD0EE66EE4
:10792000030EE66E89EC53F0A8C3E7F3A9C3E8F3AE
:10793000DD0E146E030EF2EC56F01AEF51F0D7EC98
:1079400056F0DDDD0301A651C71902E1A751C819A0
:1079500002E0C8EC56F01AEF51F015EC51F0E65287
:10796000FBEC50F0D7C3DFFF070EDF5C06E00B0E29
:10797000DF5C03E0F36AF46A1FD00301C951C75DFD
:10798000CA51C85910E3BFEC51F01606000E175A41
:10799000C951C75D186EC851CA55196EF7EC56F03B
:1079A000F2EC56F009D0C751C95D146ECA51C855E2
:1079B0007BEC58F019EC54F0E5521AEF51F015EC4D
:1079C00051F0020EE12680EC58F0BBEC56F002E1DB
:1079D000000E36D084EC58F004E1ED5002E188EC62
:1079E00051F00301D951010B09E1BCEC53F0BFEC9C
:1079F00051F008EC54F002E389EC58F0010EE66E09
:107A0000E66AE66E91EC55F0B5EC52F034EC51F0CC
:107A10000301C72B000EC823C351C75DC451C85909
:107A200002E3C9EC54F084EC58F005E1ED5003E1B9
:107A300088EC51F004D0D8BB02D069EC51F0010EB3
:107A4000146E020EE15C02E2E16AE552E16E14504E
:107A50001AEF51F0B3EC58F005E188EC51F0F36AFD
:107A6000F46A39D083EC57F0DBEC56F042EC51F07D
:107A700003E2FA0E1EEC54F00301D951010B05E1AB
:107A8000FBEC57F002E389EC58F023EC53F00DE3E4
:107A900003EC57F057EC57F018EC56F0D950FC0FA8
:107AA000ABEC51F0ED22E1EC58F0B3EC57F057ECB1
:107AB00057F0D2EC58F012EC51F0DBEC56F042ECFF
:107AC00051F003E388EC51F004D0D8BB02D069EC4C
:107AD00051F00AEC53F0060EE15C02E2E16AE55275
:107AE000E16E1AEF51F0B3EC58F005E188EC51F07B
:107AF000F36AF46A3CD00301D951010B05E1FBECB8
:107B000057F002E389EC58F083EC57F0F90EDBCF25
:107B100016F0FA0E42EC51F003E2F90E1EEC54F0AE
:107B200023EC53F010E303EC57F001EC58F018ECA1
:107B300056F0166AD950FB0FABEC51F0EE221650FE
:107B4000EE22E1EC58F0B3EC57F001EC58F0D2EC37
:107B500058F029EC57F042EC51F003E388EC51F077
:107B600004D0D8BB02D069EC51F00AEC53F0060EF9
:107B7000E15C02E2E16AE552E16E1AEF51F015ECC8
:107B800051F0FC0EDBCF16F0FD0EDBCF17F08EECC4
:107B900058F0FC0E57EC51F078ECD9F0E552E55274
:107BA000F3CF18F0F4CF19F0F3CFE6FFF4CFE6FFF0
:107BB000FC0ECBEC58F04EDF1A6E050EE15E1A504B
:107BC0005EEC55F0F324146E1750F420F2EC56F0EE
:107BD0001AEF51F015EC51F0E8EC51F086ECD9F0C9
:107BE000E552E552E55207C01AF008C01BF007C085
:107BF000E6FF08C0E6FFE8EC51F075EC56F073DFE5
:107C00001C6E060EE15E1C50F3CF17F0F4CF18F097
:107C1000196A18EC59F0EE50F324146EEE50F4206B
:107C2000156EEE501920166E14C007F015C008F03E
:107C3000096E1AEF51F0B8EC57F0FBEC50F003016D
:107C40008EEC51F01406000E155A0FEC52F090EC29
:107C500053F01BEC52F002E2E16AE552E16E1AEFDA
:107C600051F015EC51F0C6EC51F016EC52F0F35017
:107C7000F41006E0FBEC50F0F1EC55F0C8EC56F0D7
:107C80001AEF51F0D7EC56F0030154EC55F006E32F
:107C9000CD51CB5D146ECC51CE5513D0CD51C55DB9
:107CA000166EC651CE55176EECEC55F0C351CB5D38
:107CB000186ECC51C455196E16501824146E1750F6
:107CC0001920F2EC56F01AEF51F015EC51F0020EBB
:107CD000E126C6EC51F0BBEC56F002E1000E24D0D8
:107CE000FBEC50F0BDEC57F008E0010EE66EE66AE2
:107CF00080EC54F0E66ECDEC56F00301CD2B000E77
:107D0000CE23CD51C55DCE51C65902E2F6EC55F0F9
:107D100084EC58F004E1ED5002E1D98504D0D8BBE1
:107D200002D04FEC52F0010E146E020EE15C02E242
:107D3000E16AE552E16E14501AEF51F0B8EC57F0D9
:107D4000020EDB6A030EDB6AC6EC51F0BBEC56F0A8
:107D500003E1F36AF46A72D0FBEC50F095EC53F057
:107D6000F2EC54F008E264EC51F0FA0EEECFDBFFD7
:107D7000FB0EEDCFDBFFFA0EDB500301CD2500013A
:107D8000146EFB0EDB500301CE21000187EC54F092
:107D900024E2CD51DDEC54F0CE5551EC51F00FEC16
:107DA00052F0BDEC57F00FE0020EDBCFE6FF030E02
:107DB000DBCFE6FFE5EC58F012EC51F0D950FC0FA8
:107DC000ABEC51F0ED2212EC51F0D950FA0F70ECFF
:107DD00056F0A1EC51F0F6EC55F0BDEC57F004E094
:107DE00030EC57F0E5EC58F08FEC54F008500301FC
:107DF000CD270950CE2312EC51F0D950FA0FABEC3D
:107E000051F0ED22DECF16F0DDCF17F0FA0E3BEC8D
:107E100059F0FB0EDB501758156EFA0EDBCF18F039
:107E2000FB0E8BEC54F002E3D98504D0D8BB02D012
:107E30004FEC52F095EC53F019EC54F0040EE15C69
:107E400002E2E16AE552E16E1AEF51F0B8EC57F048
:107E5000FBEC50F00301C351DDEC54F0C455156E3A
:107E60000FEC52F0C6EC51F01BEC52F002E2E16A6A
:107E7000E552E16E1AEF51F037EC57F0D950FA0F96
:107E80004CEC51F003E1F36AF46A73D093EC58F0D0
:107E900079EC54F0DBEC56F0DBCF17F0EBEC58F05C
:107EA000156E020EDBCF18F0030E8BEC54F00FE2D0
:107EB00022EC57F0F80E3BEC59F0F90EDB50175856
:107EC000156EFA0E14C0DBFFFB0E15C0DBFFF80EBB
:107ED000FBEC55F0F90EDB50CE2114C0DEFFDD6E59
:107EE000BCEC53F0C1EC57F004E251EC56F0AFECAF
:107EF00057F0DE50C55D146EDD50C6591CEC59F0CC
:107F000095EC53F0040EDBCF16F0050E42EC51F069
:107F100007E330EC57F035EC52F0CDEC56F025D0BD
:107F2000BCEC52F035EC52F0CDEC56F0DBEC56F0F8
:107F300068EC56F047EC54F0010EE66E040EDBCF11
:107F40001AF0050EDBCF1BF0FC0EDB501A24186E66
:107F5000FD0EDB501B20196E18C0E6FFE66EECEC40
:107F60004FF01C6E080EE15E1C5095EC53F019ECBE
:107F700054F0060EE15C02E2E16AE552E16E1AEFAE
:107F800051F015EC51F0E652FC0E57EC51F0010E99
:107F900097EC58F075EC56F06FDF146E070EE15E4B
:107FA0001450DF50E5521AEF51F015EC51F0300E3D
:107FB000E126D950FA0F4CEC51F003E1F36AF46A70
:107FC00024D193EC58F0F80EDB50F35C146EF90EEC
:107FD000DB50F458156E0FEC52F0F1EC58F001E262
:107FE0000AD1D950F60F4CEC51F00FE012EC51F0E1
:107FF000F60EDBCF16F0F70E42EC51F006E2F60E6D
:10800000DBCF08F0F70EF7EC54F0F80EFBEC55F070
:10801000F90E54EC52F002E2F6EC58F094EC56F003
:10802000F80EDBCF08F0F90E6BEC53F08FEC54F048
:108030009FEC55F0FC0EDBCF08F0FD0E00EC55F088
:1080400007EC52F001E3DB2A0D0EEFCFDBFF0F0E42
:10805000DB6AF50EDB500AE0610E3CEC57F006E3FC
:108060000D0EDB507A0802E399EC52F0200EF36E0D
:108070000E0E32EC53F006E2040EDB50E76E0E0EED
:10808000E7CFDBFF0E0EE6EC53F006E2020EDB500C
:10809000E76E0E0EE7CFDBFF0E0E07EC58F0100F69
:1080A000FBEC52F034EC51F00E0EDB50DE26000EED
:1080B000DD220E0EBCEC58F002E109EC55F0F50E95
:1080C000DB505BE00C0EDB6A0EEC58F001E38BD06A
:1080D000D950100F156E0C0E60EC57F012E3D9500A
:1080E000100F176EDACF18F00C0E14EC58F009E3ED
:1080F000E00E166E42EC55F014244AEC52F0165085
:10810000EF2642EC55F0FDEC56F00D0EDB50F35C23
:108110001BE1FA0EDB06DBCF14F0FB0E01E2DB06FF
:1081200059EC55F042E007EC52F001E3DB2A12EC87
:1081300055F0610E3CEC57F01DE30D0EDB507A0854
:1081400019E399EC52F016D03CEC53F013E09FEC9D
:1081500056F001E3DB2A0D0EEFCFDBFF610E3CECA6
:1081600057F006E30D0EDB507A0802E399EC52F06B
:108170000F0EDB6A0C0EDB2AA7D70C0EDB6A0EECA7
:1081800058F031E242EC55F00F01FDEC56F00D0EC7
:10819000DB50F35C19E1FA0EDB06DBCF14F0FB0ECB
:1081A00001E2DB0659EC55F008E147EC53F00C0E08
:1081B0004AEC57F01BEC58F028D007EC52F001E3E2
:1081C000DB2A12EC55F00CD03CEC53F009E09FECAC
:1081D00056F001E3DB2A0D0EEFCFDBFF0F0EDB6A5B
:1081E0000C0EDB2ACCD70E0E23EC54F09DEC57F08E
:1081F000F1EC58F003E2F368F46807D00E0E23ECBC
:1082000054F0060F36EC56F031D7300EE15C02E246
:10821000E16AE552E16E1AEF51F015EC51F0310EC2
:10822000E126D950F90F4CEC51F003E1F36AF46AFE
:1082300011D193EC58F0F70EDB50F35C146EF80E8E
:10824000DB50F458156E0FEC52F029EC57F09CEC13
:1082500053F001E2F5D0D950F50F4CEC51F00FE09E
:1082600012EC51F0F50EDBCF16F0F60E42EC51F0A9
:1082700006E2F50EDBCF08F0F60EF7EC54F0F70E41
:10828000FBEC55F0F80E54EC52F002E2F6EC58F02C
:1082900094EC56F0F70EDBCF08F0F80E6BEC53F0D1
:1082A00096EC54F09FEC55F018EC59F00A0EEECF16
:1082B000DBFF0B0EEECFDBFF0C0EEECFDBFF01EC96
:1082C00051F0100EDB6AF40EDB5009E0A0EC57F021
:1082D00006E30E0EDB507A0802E3A4EC52F0200E07
:1082E000F36E0F0E32EC53F003E2040E48EC55F03F
:1082F0000F0EE6EC53F003E2020E48EC55F00F0EC1
:1083000007EC58F0110FFBEC52F034EC51F00F0E6B
:10831000DB50DE26000EDD220F0EBCEC58F002E131
:1083200009EC55F0F40EDB5052E00D0EDB6A0F0E37
:10833000DB503CEC57F001E379D0D950110F156EAA
:108340000D0E60EC57F012E3D950110F176EDACF13
:1083500018F00D0E14EC58F009E3E00E166E4EEC1A
:1083600055F014244AEC52F01650EF264EEC55F01E
:10837000FDEC56F00E0EDB50F35C16E1F90EDB0659
:10838000DBCF14F0FA0E01E2DB0659EC55F039E0D0
:10839000CFEC57F0A0EC57F017E30E0EDB507A0845
:1083A00013E3A4EC52F010D056EC53F00DE079EC4E
:1083B00056F0A0EC57F006E30E0EDB507A0802E30D
:1083C000A4EC52F0100EDB6A0D0EDB2AB0D70D0EB6
:1083D000DB6A0F0EDB503CEC57F028E24EEC55F018
:1083E0000F01FDEC56F00E0EDB50F35C15E1F90EBB
:1083F000DB06DBCF14F0FA0E01E2DB0659EC55F098
:1084000008E147EC53F00D0E4AEC57F01BEC58F026
:1084100021D0CFEC57F007D056EC53F004E079ECC4
:1084200056F0100EDB6A0D0EDB2AD3D70F0E23ECAD
:1084300054F09DEC57F029EC57F09CEC53F003E21C
:10844000F368F46807D00F0E23EC54F0060F36ECF7
:1084500056F045D7310EE15C02E2E16AE552E16E89
:108460001AEF51F015EC51F0F80EDBCFE6FFF90EE4
:10847000F0EC52F0B8EC51F0010EE66EE66A91ECC9
:1084800055F075EC56F091DD146E0A0EE15E145055
:108490001AEF51F015EC51F00A0EE126DF6AFFECFD
:1084A00051F001E3DCD1B1EC53F0030EDB6A010EB5
:1084B000DB6A020EDB6A0301D951020B03E1D951D9
:1084C000040B10E0B2EC88F000090CE0100E00EC98
:1084D00053F00301D951040B01E0010EE76E010EC8
:1084E000E7CFDBFF0301D8AB11D0D1ECE3F0030100
:1084F0000650D35D146E0750D459156EE83402E26D
:10850000D3EC54F003E3100E00EC53F0D8AD09D0D7
:108510004FEC54F002E2D3EC54F003E3100E00EC05
:1085200053F00B0ED75D0BE14FEC54F002E2D3ECAD
:1085300054F005E3110E00EC53F00C0ED76F040E4F
:10854000D75D46E1CEEC54F0AFEC52F041E220ECC6
:1085500059F03EE05DEC56F0CAEC52F0DA511418D6
:1085600031E1DB5115182EE17FEC3AF014EC56F0B6
:1085700095EC50F01BEC55F0B7EC53F082EC53F057
:10858000A5EC57F0EECFA8F3EDCFA9F395EC50F0A2
:108590000C0E3EEC51F0EECFA2F3EECFA3F3EECFF4
:1085A000A4F3EFCFA5F30301A22BA323A423A523B8
:1085B0005DEC52F0120E00EC53F0060ED76FB0ECEB
:1085C00050F006D0040EDB2A050EBEE3DB2ABCD732
:1085D000030EDB5009E0010EDB5002E0000E01D07B
:1085E000010EE66E66EC55F00301D8B931D0070EE6
:1085F000D75D01E032D16AEC52F001E02ED10301E7
:10860000D851070B06081AE1D851080B01E0010EFA
:10861000E76E030EE7CFDBFFDFCFE6FF3BEC3CF07E
:10862000E552DFCFE6FF3BEC3CF0E552030EDB50BA
:1086300001E013D103010E0ED76F0FD17FEC3AF09A
:10864000020EE66E100E46EC51F06EEC51F005D1C4
:108650006AEC52F001E001D17FEC3AF00301D7510E
:108660000C0A01E1BCD0060A01E1B4D0030A01E121
:10867000C0D0010A01E1A9D00F0A01E19DD00C0A86
:1086800001E19AD00D0A01E18ED0030A01E189D0FF
:10869000060A5DE0010A4CE0030A23E0010A01E05A
:1086A000B0D075ECC8F0000901E1ABD00301010EB8
:1086B000D76FBCA50BD0E66EB0C3E6FFB1C3E6FF33
:1086C000B2C3E6FFA5ECC8F0E55207D0E66EB0C332
:1086D000E6FFB1C3E6FF87ECC8F0E552E552E5528C
:1086E00090D0D950060FFBEC52F0C8ECC8F0E55220
:1086F000E552000901E185D07AECC8F0000914E0E8
:10870000060EDBCFB0F3070EDBCFB1F3080EDBCFE5
:10871000B2F3090EDBCFB3F30301020ED76F5DECAA
:1087200052F08AEC55F06DD06EEC51F0D76B69D0F9
:10873000D1ECE3F006C0D3F307C0D4F3B7EC53F0A9
:108740004CECCDF0E552E5520301030E28D0B40EF7
:10875000E66E030EE66EB7EC53F09DECCDF0A6ECA2
:1087600051F0000915E1D1ECE3F00301D351065CAF
:10877000146ED4510758156E14509A5D15509B59BC
:1087800040E2060EBF5D02E2A6EC55F0020E07D0F5
:10879000020E00EC53F0010EDB6A0301050ED76FE9
:1087A00030D0020E20D0020EBF5D02E2120E1BD0AE
:1087B000D8B71FD0020E06D0050EBF5D0EE3080E1F
:1087C000D76F110EF36E030E1AD0050EBF5D11E2C6
:1087D000110E09D0050EBF5D0CE2100E04D0050E7F
:1087E000BF5D07E2110E00EC53F0DE52010EDD6EAC
:1087F00008D0140E00EC53F0010EF36E020EF3CF0E
:10880000DBFF030EDB5024E0010EDB501DE0030113
:10881000A6EC55F041EC54F0156E166A176A15AEC9
:1088200002D0166817683CEC52F040EC57F008E2B2
:10883000C6EC57F015AE02D0166817683CEC52F043
:1088400000EC56F0E66A02D0010EE66E66EC55F0DA
:10885000020EDB5002E025EC49F0DF2A20D6CEECF8
:1088600054F0AFEC52F028E220EC59F025E095EC02
:1088700050F0120E3EEC51F028EC54F08EEC58F013
:10888000D1ECE3F05EEC55F0065C146E175007581F
:10889000156E250ED8801454020E155407E2B0EC64
:1088A00050F0040EDB06050E01E2DB06040EDB2AA7
:1088B000050ED7E3DB2AD5D70A0EE15C02E2E16AB6
:1088C000E552E16E1AEF51F015EC51F0250EE1265C
:1088D000A9EC50F0E1EC54F0170EEECFDBFFB1EC59
:1088E00051F0180EEECFDBFF190EEECFDBFF1A0EA4
:1088F000EECFDBFF1B0EEECFDBFF1C0EDB6A060E9E
:10890000F36E1D0EF3CFDBFF96EC54F01E0E08C085
:10891000DBFF1F0E09C0DBFF1E0EDBCFE6FF1F0EC5
:10892000DBCFE6FFC1EC53F01E0EF3CFDBFF1F0ED3
:10893000ADEC55F0140F0DEC57F0200E14C0DBFF1A
:10894000210E15C0DBFFF90EF0EC52F043EC8BF07A
:10895000E552E552220EF3CFDBFF230EF4CFDBFF0F
:10896000200EDBCF14F0210EDBCF15F0220EDB50F2
:1089700014184BE1230EDB50151847E1000E9DEC57
:1089800054F0140E97EC58F0E0EC8CF0A6EC51F09B
:10899000F6EC52F0E7EC48F0E552E552D9500C0FF6
:1089A0003AEC51F074EC53F0146E156A140E86EC28
:1089B00055F0240E14C0DBFFDB50166E176A96ECE0
:1089C00054F01650085C146E17500958156E140EAA
:1089D00086EC55F0F90E14C0DBFFFA0E15C0DBFF74
:1089E000FD0EDBCFE6FF75EC56F0F6EC52F0AEDA9A
:1089F000A6EC51F0000909E0F90EF0EC52F0F6ECAB
:108A000052F0D9EC49F0A6EC51F0B9EC88F0010E27
:108A1000146E250EE15C02E2E16AE552E16E14504B
:108A20001AEF51F015EC51F02A0EE1267FEC3AF0E6
:108A3000FE0EDBA004D00301D987FE0EDB900301FC
:108A4000D89BD89DD89FD993D995D991B2EC88F06D
:108A50000009FCE0FE0EDB50060B05E0260EDB6A8B
:108A6000270EDB6AD7D00301A651C71910E1A75121
:108A7000C8190DE1260EDB6A270EDB6AD9A7CAD01A
:108A8000AC51AD1101E1C6D0FE0EDB80C3D0C751A1
:108A9000A65DC851A75934E2A651C75D146EC851EE
:108AA000A755CFEC52F003E341EC54F004D0BFECF7
:108AB00051F039EC54F088EC56F002E2EEEC53F051
:108AC00021EC58F002E26EEC55F0D9A712D0CCECB4
:108AD00051F0280EDB50141803E1290EDB50151855
:108AE00008E024EC55F002E1BE51171802E0FE0E3A
:108AF000DB80A4EC54F0E0EC56F0D7EC57F08AD0D1
:108B0000A651C35D146EC451A75576EC55F0240EE2
:108B1000DB50C7250001166E250EDB500301C8216E
:108B20000001176E0301C151165C146EC251175833
:108B3000CFEC52F003E341EC54F004D0BFEC51F021
:108B400039EC54F088EC56F002E2EEEC53F021ECF4
:108B500058F002E26EEC55F0D9A712D0CCEC51F0EF
:108B6000280EDB50141803E1290EDB50151808E01D
:108B700024EC55F002E1BE51171802E0FE0EDB8036
:108B8000240EDBCF14F0250EDBCF15F0260EDBCF45
:108B900016F0270E42EC51F004E2A3EC53F0B4ECD3
:108BA00055F0ABEC54F0E0EC56F028EC58F0240E05
:108BB0003BEC59F0250EDB50175876EC55F0D950A8
:108BC000240F41EC56F01DE0ABEC54F0DCC3E6FFA3
:108BD000C1C3E6FFC2C3E6FFE66A0301A651C35D57
:108BE000146EC451A755156E166A176AAC0E14267A
:108BF0000F0E1522000E16221722C4EC54F02FEC93
:108C000058F0D7EC57F0C351A65DC451A75902E301
:108C100036EC58F0D950260F41EC56F004E1FE0E28
:108C2000DB50030B16E0D950260F41EC56F002E062
:108C3000FE0EDB86FD0EDBA008D00301BF6B1B0E12
:108C40009A6FB70E9B6F9C6B9D6B13EC53F0D8899A
:108C500031D0FD0EDBA21FD0D80EE96E030EEA6EF6
:108C6000EF50070BE82AF36EE850070BF36EF46E33
:108C7000F80EEF14F310EF6EF45003019E07000E90
:108C80009F5BA05BA15B010EF36E260EF3CFDBFFB3
:108C9000270EDB6A0FD00301D8A90CD0DBB008D0B7
:108CA000BF5106E0BF07D8909D339C339B339A3366
:108CB00013EC53F0020EAAC3DBFF030EABC3DBFFC2
:108CC000040EA8C3DBFF050EA9C3DBFF060E9EC37F
:108CD000DBFF070E9FC3DBFF080EA0C3DBFF090EFF
:108CE000A1C3DBFF0A0EA2C3DBFF0B0EA3C3DBFF96
:108CF0000C0EA4C3DBFF0D0EA5C3DBFF0F0EDB9C28
:108D0000DB9E0E0EDB90DB92DB94DB96FE0E48ECD6
:108D100055F0140EDB6A150EDB6ACCEC51F0000145
:108D20005AEC54F0FE0EDBA215D0DBB808D00A0EC8
:108D3000DB6A0B0EDB6A0C0EDB6A0D0EDB6ABCA372
:108D400003D0DAEC58F006D09E2B000E9F23A02310
:108D5000A123BC83FE0EDBA00BD0BCA103D0DAECB8
:108D600058F006D09E2B000E9F23A023A123BC8188
:108D700054EC55F003E37DEC52F002D0EBEC54F0F0
:108D8000100E14C0DBFF110E15C0DBFFE9EC88F0FC
:108D900016EC52F0400E86EC55F005EC56F0BCECAB
:108DA00053F00001800E151402E0DE6ADD6AAAECC1
:108DB00053F0F2EC54F008E264EC51F0100EEECFF8
:108DC000DBFF110EEDCFDBFFD950020FFBEC52F0B1
:108DD000FED9E552E552D950260F3AEC51F0140E67
:108DE000EE26000EED220E0EDB88DB9ADB8CDB9E7E
:108DF000FE0EDBA22FD0D950260F3AEC51F0040E14
:108E0000EE26000EED22020EF36E160EF3CFDBFF00
:108E1000040EF36E170EF3CFDBFF020EF36E180E87
:108E2000F3CFDBFF140E0AEC56F0010E146ED9508E
:108E30000E0F3AEC51F03DEC58F014240F0BF36E8A
:108E4000F46EF346F346F346F3460F0EEF14F310B9
:108E5000EF6EF4501A0E61C0DBFF1B0E62C0DBFF29
:108E60001C0E63C0DBFF1D0E64C0DBFF1E0EB0C313
:108E7000DBFF1F0EB1C3DBFF200EB2C3DBFF210EF1
:108E8000B3C3DBFF220EDB6A060EF36E230EF3CFB5
:108E9000DBFFA3EC53F0B4EC55F0ABEC54F0C1ECB9
:108EA00053F0240EF3CFDBFF250EADEC55F01A0F77
:108EB0000DEC57F0120E14C0DBFF130E15C0DBFFD4
:108EC000840E7EEC55F0A4EC54F0060EE66EB7EC82
:108ED00053F088ECDAF0146E050EE15E1450140EB7
:108EE000E66EE66AD950020FFBEC52F0CBEC57F07D
:108EF000FE0EDBA209D0040EE66EE66AD950160F0C
:108F0000FBEC52F0CBEC57F0980EE66E0F0EE66ECF
:108F100012EC8BF0E552E552A4EC54F043EC8BF0EC
:108F2000E552E55224EC59F0A80E7EEC55F0020E05
:108F300097EC58F0CBEC57F083EC8AF02A0EE15C0A
:108F400002E2E16AE552E16E1AEF51F037EC57F0B8
:108F50001CEC56F0EE50ED1001E1A5D0DE52FE0EF5
:108F6000DD6EB1EC51F0020E3EEC51F0EECF1AF096
:108F7000EFCF1BF0B1EC51F01A50EE24186E1B50DD
:108F8000EE20196EA9EC50F01850EE24166E195010
:108F9000EE20176E1CEC56F01650EE18146E17509B
:108FA000EE18156E0FEC52F0DF6AFFEC51F047E25D
:108FB000B1EC53F00D0E0301D75D3FE0040ED75D19
:108FC0000CE1CFEC58F01450DA1937E11550DB19E9
:108FD00034E1010EDFCFDBFF30D0DAC314F0DBC3A6
:108FE00015F0020EDB50141828E1030EDB501518A3
:108FF00024E17FEC3AF0CFEC58F00301AA511418A9
:109000001CE1AB51151819E1A9EC50F028EC54F013
:10901000A851161812E1A95117180FE1B1EC51F03F
:10902000EE50B0190AE1EE50B11907E1EE50B21955
:1090300004E1EE50B31901E128E0DF2AB6D7010EB2
:10904000DB50FE0824E0010EDBCFE6FF54EC3AF0E3
:10905000E5527FEC3AF0010EDB50FE0818E0020EFC
:10906000DBCFDAF3030EDBCFDBF374EC57F0A9ECC4
:1090700050F0EECFA8F3EDCFA9F31CEC56F0EECFF5
:10908000AAF3EDCFABF30FEC56F0010E96D0A9EC9E
:1090900050F00D0E3EEC51F0EF50020B04E00201D7
:1090A000FC51FD1102E0000E88D0CEEC54F0AFEC84
:1090B00052F036E220EC59F033E05DEC56F0CAECA9
:1090C00052F01CEC56F028EC54F01650141822E123
:1090D000175015181FE1A5EC57F0CAEC52F0A9EC97
:1090E00050F028EC54F01650141814E117501518CD
:1090F00011E1B1EC51F086EC57F0EE50000114187C
:1091000008E1EE50151805E1EE50161802E1EE5098
:10911000171844E0040EDB2A050EC9E3DB2AC7D783
:10912000DF6AFFEC51F048E2B1EC53F00301D8A73D
:1091300041D07FEC3AF0CFEC58F014500301AA195B
:1091400039E11550AB1936E114EC56F0B8EC51F09A
:1091500095EC50F01BEC55F082EC53F0A9EC50F07C
:10916000CAEC52F0A5EC57F014C0EEFF15C0EDFFAD
:10917000A9EC50F0040E3EEC51F086EC57F00C0ECA
:109180003EEC51F014C0EEFFC4EC58F0CFEC58F0B8
:109190005DEC56F014C0EEFF15C0EDFFD1ECE3F02E
:1091A00007C015F095EC50F0120E9BEC58F015C06E
:1091B000EDFF03D0DF2AB5D7000E146E060EE15C7A
:1091C00002E2E16AE552E16E14501AEF51F015EC3B
:1091D00051F0A9EC50F0A5EC58F0A9EC50F0D8EC07
:1091E00054F01CEC56F0A5EC58F01CEC56F029ECB1
:1091F00059F0040E21EC56F0040E9BEC58F0C4EC30
:1092000058F0A9EC50F0080E21EC56F0080E9BEC3B
:1092100058F0C4EC58F0D2EC56F0A5EC58F0D2EC73
:1092200056F029EC59F0100E3FEC59F0100E3EECC0
:1092300051F029EC59F0120E3FEC59F0120E3EECB1
:1092400051F0D8EC54F01AEF51F07FEC3AF0AAC389
:10925000DAF3ABC3DBF3C9EC54F0C1C3C9F3C2C347
:10926000CAF3C3C3CBF3C4C3CCF3F6EC55F003018C
:10927000D851080B02E0040E01D00D0ED76FD89123
:10928000D893D895D899D89BD89DD89FD991D99360
:10929000D995D997D989BC91BC93BC97BC990FEC4F
:1092A00056F0B7ECE0F0F3CF9EF3F4CF9FF3B7ECBA
:1092B000E0F0F3CFA0F3F4CFA1F30301BA69BB69E7
:1092C000010EAC6FAD6B1200B8EC57F00C0E9DECBC
:1092D00054F0D3EC8CF0DF6EF00EDF14E840E84081
:1092E0003F0B146E156A140E86EC55F01450DF6EA9
:1092F000DF5053E0070EE66E8DEC57F0DF50DF06CF
:1093000000094BE00CEC54F048E0010EDB04F6E001
:10931000010EDB50020831E1030EDF5C3EE3020E7A
:10932000DB6A030EDB6A0CEC54F004080CE1D3ECAE
:109330008CF0E76E030EE7CFDBFFD3EC8CF0E76E2B
:10934000020EE7CFDBFF12EC51F0180E145C020E98
:10935000155823E3D950020F3AEC51F0B40ED880DF
:10936000EE54050EED5404E2B40EF36E050E18D063
:1093700012EC51F019EC54F014D0020EDF5C0DE346
:109380000CEC54F0DF5C09E3010EDBCFE6FF8DEC63
:1093900057F0010EDB50DF5EB1D7180EF36E020EF0
:1093A000F46E040EE15C02E2E16AE552E16E1AEF4E
:1093B00051F015EC51F01A0EE126A9EC50F00D0E0B
:1093C0003EEC51F00E0EEFCFDBFFA9EC50F0080E93
:1093D0003EEC51F00F0EEECFDBFF100EEECFDBFFB9
:1093E000110EEECFDBFF120EEECFDBFFA9EC50F03B
:1093F000040E3EEC51F0130EEECFDBFFE1EC54F027
:109400000301D891D893D895D8B902D06EEC51F019
:10941000D751050A25E0010A10E0B2EC54F0170E0E
:1094200008C0DBFF180E09C0DBFF0E0EDBA04ED01C
:10943000170EDB2A180E4AE348D00E0EDBB406EFF7
:109440004FF0DBA805D0F2EC51F0E66A040EA9D289
:10945000DBA206EF4FF0DEEC52F0BBEC55F02BD068
:109460000E0EDBB40DEF4FF0DBA810D044EC58F03B
:1094700001E01CD1EE509F1901E018D1EE50A01967
:1094800001E014D1EE50A11901E010D10E0EDBA2C3
:109490000DEF4FF0DEEC52F0FAEC58F0BBEC55F06B
:1094A0000E0EDBA808D0C8EC56F00301070ED76FEC
:1094B000D8990DEF4FF0010EE66E120E46EC51F00A
:1094C0000301060ED76F0DEF4FF0DB2A0E0EDBA265
:1094D00005D0170EDB2A180E01E3DB2A54EC55F0F9
:1094E00003E37DEC52F002D0EBEC54F00C0E14C010
:1094F000DBFF0D0E15C0DBFFD950130F3AEC51F016
:10950000A251EE5C146EA351EE58156EA451EE58A4
:10951000166EA551EE58176E4BEC58F0080E16C09B
:10952000DBFF090E17C0DBFF060EDBCF08F0070ECE
:1095300000EC55F0190EDB6AD950170F41EC56F0CC
:109540006EE0D9500C0F41EC56F001E183D000ECF5
:1095500059F002E628EC55F005E3ABEC58F079EC55
:1095600053F040E3170EDBCF14F0180E14EC54F058
:109570003DEC56F031EC55F01734000E171809E6A3
:10958000D880000E1454000E1554000E1654000E10
:1095900017542BE20C0EDBCF1CF00D0EDBCF1DF0B1
:1095A000170EDB501C5C186E180EDB501D58196E20
:1095B0001A6A1B6A19AE02D01A681B683DEC56F095
:1095C000030EEBCFF3FF1B50F318E8AE02D0F334D9
:1095D00008D0EE50185CEE501958EE501A58EE5064
:1095E0001B5803E3010E0AEC56F0ABEC58F0030EE7
:1095F000EB501718E8AE02D0173402D079EC53F0D4
:1096000029E2170EDBCF1AF0180E65EC54F0E8349F
:1096100021E218500008000E19541CE218D052EC38
:1096200058F0080EDBCF16F0090EDBCF17F0145000
:109630001510161017100BE000EC59F002E628EC9C
:1096400055F008E3ABEC58F079EC53F003E2010E6F
:109650000AEC56F0190EDB5004E10E0EDBB4DDD33C
:10966000D8D30E0EDB50060B01E0D0D30E0EDBA8D4
:10967000D4D3D7510C0A01E1ADD10B0A39E00F0A5E
:1096800037E0010A35E0020A33E0010A31E00C0A52
:1096900001E0B3D144EC58F008E1EE509F1905E128
:1096A000EE50A01902E1EE50A11920E0130E9EC366
:1096B000DBFF140E9FC3DBFF150EA0C3DBFF160EEE
:1096C000A1C3DBFFF2EC51F0010EE66E040E46EC96
:1096D00051F0130EDBCF9EF3140EDBCF9FF3150E6C
:1096E000DBCFA0F3160EDBCFA1F397D3070ED76F16
:1096F000A651C75D146EC851A755156E5DEC51F0AB
:10970000040EB9EC54F007E003018EEC51F0D9508F
:10971000040F36EC56F02DEC59F014EC54F09E0E7C
:10972000E96E030EEA6E31EC55F029EC52F0ADEC27
:1097300056F01850EE5C146E1950EE58156E1A5013
:10974000EE58166E1B50EE58176E0001800E17145F
:1097500002E0E66A60D30301C951A65D186EA75105
:10976000CA55196E1A6A1B6A19AE02D01A681B68AC
:1097700018509E5D146E19509F59156E1A50A059BD
:10978000166E1B50A159176E29EC52F040EC57F0A1
:109790000CE2C6EC57F064EC51F01450EE5E15503C
:1097A000EE5A1650EE5A1750EE5AADEC56F0EE50F7
:1097B000185C146EEE501958156EEE501A58166E4D
:1097C000EE501B58176E29EC52F0DECF07F0DECFBB
:1097D00008F0DECF09F0DDCF0AF0DD52DD520A34A9
:1097E000000E0A1809E6D880000E0754000E08542F
:1097F000000E0954000E0A5461E2C6EC57F064EC06
:1098000051F0EE50145CEE501558EE501658EE50D4
:10981000175854E3BC97BC99D991040EC9C3DBFF18
:10982000050ECAC3DBFF64EC51F0EE50C927EE50C1
:10983000CA2318EC56F01450A65D1550A7590BE337
:1098400040EC57F028E2A651C95D146ECA51A755E5
:10985000156E00011CD0BFEC51F0A6511624146EF9
:10986000A7511720156E5DEC51F018EC56F0C95158
:10987000145CCA5115580FE2040EDB50C95D00019B
:10988000146E050EDB500301CA590001156E5AEC27
:1098900054F000EC56F0C351C95DC451CA5906E3F7
:1098A0008EEC51F01450C95F1550CA5BC351A65DD0
:1098B000C451A75928E336EC58F025D0A651C91950
:1098C00002E1A751CA191FE0BCA71CD0BCA919D03E
:1098D00041EC54F0156E166A176A15AE02D0166880
:1098E00017683CEC52F040EC57F008E2C6EC57F039
:1098F00015AE02D0166817683CEC52F000EC56F03A
:10990000D985BC89BC87C751C91917E1C851CA1983
:1099100014E1D9B702D0D89910D056EC56F00DE129
:109920009F51EE180AE1A051EE1807E1A151EE187F
:1099300004E103E1D899D997BC91AC51AD1106E18E
:10994000D2EC56F0EE50ED1001E0D983FAEC58F06D
:10995000080ED75D1CE156EC56F04FE19F51EE1812
:109960004CE1A051EE1849E1A151EE1846E145E164
:1099700046EC56F0870E0301CF27930ED023030E3B
:10998000D123000ED223D889090ED76F36D0090E05
:10999000D75D0AE10E0EDBB030D0F2EC51F0E66A92
:1099A000140E46EC51F032D20A0ED75D26E156EC89
:1099B00056F001E032D29F51EE1801E02ED2A051B4
:1099C000EE1801E02AD2A151EE1801E026D201E002
:1099D00024D21CD256EC56F001E01FD29F51EE1853
:1099E00001E01BD2A051EE1801E017D2A151EE18F0
:1099F00001E013D201E011D209D20E0EDBBA0DD272
:109A00000B0ED75D01E109D20A0ED75D01E105D247
:109A10000C0ED75D01E101D2D950FB0F4CEC51F097
:109A200001E176D1C3EC52F0153402E2D3EC54F0EC
:109A300001E2A7D0DFEC57F0166E176A0A0EDB5072
:109A4000F35C146E0B0EDB50175845EC57F005EC29
:109A5000DBF0E552E552C3EC52F0D950FB0FABEC12
:109A600051F0ED22FB0EDBCF14F0FC0EDBCF15F036
:109A70000C0EDBCF16F00D0E42EC51F00CE20C0E8A
:109A8000DBCF08F00D0EDBCF09F0FB0E08C0DBFFCB
:109A9000FC0E09C0DBFFFB0EDBCF14F0FC0ECBECA1
:109AA00053F0FB0EDB50CB250001146EFC0EDB5097
:109AB0000301CC21000187EC54F019E2CB51DDEC1D
:109AC00054F0CC551CEC59F0BCEC52F062EC56F062
:109AD00059EC58F095EC51F006EC59F0156E030175
:109AE000C3511424CB6FC4511520CC6F0BD032EC72
:109AF00059F059EC58F0B2EC54F008500301CB2760
:109B00000950CC23BA1D01E1BB1D01E101D1B2EC2A
:109B100054F00850BA5F0950BB5BAE51BA25146EC1
:109B2000AF51BB21156EC9DB040EDBCF14F0B9ECCD
:109B300054F002E0030122D00301BB3504E2BA5124
:109B40000008000EBB5501E2E3D02DEC59F0CBEC40
:109B500053F0040EDBCF08F0050EDBCF09F0085000
:109B6000CB270950CC23CB51C55DCC51C65906E259
:109B700051EC56F01450CB5F1550CC5BBA69BB6901
:109B8000C7D0C3EC52F0153401E3C2D0D3EC54F08B
:109B900001E3BED00A0EDBCF16F00B0EDBCF17F0C1
:109BA0000CEC59F0156E0C0EDBCF18F00D0E8BEC93
:109BB00054F00EE20C0EDBCF16F00D0EDBCF17F0DB
:109BC0003AEC55F0FB0E14C0DBFFFC0E15C0DBFFBA
:109BD000DFEC57F09DEC54F0FBEC53F00CEC59F03B
:109BE00087EC54F030E2CB51C55D166EC651CC55B2
:109BF000176EECEC55F03AEC55F05FDB040EB9EC67
:109C000054F00BE1BCEC52F062EC56F00A0EDB5063
:109C100003018DEC52F089DB1CD032EC59F0FBECE7
:109C200053F00301C351C55D186EC651C455196E7A
:109C3000010E1826000E1922F7EC56F045EC57F0ED
:109C40005FEC58F006D032EC59F00A0EDB508DEC88
:109C500052F00301BA1D07E1BB1D05E1C9EC55F047
:109C6000C2EC55F055D0C3EC52F0BA51145CBB5164
:109C7000155829E298DB13E3FB0EDBCF1CF0FC0E3A
:109C8000DBCF1DF00A0EDB501C241A6E0B0EDB50CE
:109C90001D201B6EBA511A5CBB511B5803E2C2EC6B
:109CA00055F00ED0D0EC55F00A0EDB500001145CDC
:109CB0000301AE6F0B0EDB50000115580301AF6FAF
:109CC000C9EC55F025D06FDB23E2C3EC52F0BA515A
:109CD000AE25166EBB51AF21176E1450165C155091
:109CE000175816E3FB0EDBCF1AF0FC0E65EC54F0B0
:109CF000BA51185C166EBB511958176EAE51165CEE
:109D0000146EAF511758156E1450AE271550AF236F
:109D1000D950170F41EC56F017E0070ED75D02E05F
:109D2000F1EC55F0D8AF05D0C8EC56F07FEC3AF026
:109D30000BD0D88FD8BD08D0D88DD7EC55F0120EE7
:109D40000301D527000ED6230E0EDBA066D0A2C3DA
:109D500014F0A3C315F0A4C316F0A5C317F0142A7A
:109D6000000E152216221722170EDBCF18F0180E40
:109D7000DBCF19F01A6A1B6AD950130F7BDAEE5049
:109D80001826EE501922EE501A22EE501B221450C3
:109D9000181843E11550191840E116501A183DE102
:109DA00017501B183AE139E10301A22B000EA3233F
:109DB000A423A523D751090A26E0010A14E00F0ABB
:109DC00008E0010A26E10C0ED76F010EE66E110EB7
:109DD00023D00B0ED76FD7EC55F0240E0301D527F7
:109DE000000ED62316D056EC56F00AE19F51EE181D
:109DF00007E1A051EE1804E1A151EE1801E103E0E2
:109E00000A0ED76F06D0E66A100E40DA25EC49F04C
:109E100004D0010EE66E100E39DA1A0EE15C02E291
:109E2000E16AE552E16E06D237EC57F0E4D9BDECB9
:109E300057F007E1010EF36EFC0EF3CFDBFFFD0ED2
:109E4000DB6A0301C151DDEC54F0C2557BEC58F0E4
:109E500005EC56F061EC53F0DECF18F0DDCF19F0D1
:109E6000A0EC58F06CE37FEC3AF0F90EDB50030BFA
:109E700003E1F90EDB80DB828FEC54F0040E08C0A6
:109E8000DBFF050E09C0DBFF61EC53F0AFEC57F0D0
:109E9000F90EDBA20ED0DBA006D0BCEC53F0D890BC
:109EA0001532143202D0BCEC53F0D950040F36EC0A
:109EB00056F0040EDB500301C1250001146E050E9F
:109EC000DB500301C2210001ECD905EC56F0020E73
:109ED000CBC3DBFF030ECCC3DBFF0301BA1D01E1E3
:109EE000BB1D0FE0D0EC55F0D950020F36EC56F008
:109EF00099D9C1EC57F005E251EC56F0D9509DECE0
:109F000057F090D91450CD5D1550CE590BE2BCECF2
:109F100053F01450CD5D1550CE591BE2F90EDBB451
:109F20000ED00FD066EC58F00CE2BCEC53F014509D
:109F3000C35D1550C4590DE2F90EDBA402D0000E2A
:109F400042D0DECFCDF3DDCFCEF3DECFCBF3DDCF0E
:109F5000CCF366EC58F025E2F90EDB50040B21E05F
:109F6000020EDBCF08F0030EDBCF09F0C351085C13
:109F7000146EC451095847EC54F0DCC3E6FFB3EC4F
:109F800057F0C1EC56F0030154EC55F00AE2DE50F4
:109F9000C35D146EDD50C459156E1450CB5F15505F
:109FA000CC5BDECFC3F3DDCFC4F30FEC56F0C1C3FF
:109FB000C9F3C2C3CAF3C9EC54F0070ED75D02E17E
:109FC000C8EC56F0010E146E060EE15C02E2E16A86
:109FD000E552E16E14502ED128D9F90EDB501EE067
:109FE000010A45E1FC0EDB5008E0010A40E1EDEC1E
:109FF00056F0CBEC58F08DDB3AD0D950FD0FC0ECC9
:10A0000054F002E1FF0EED1802E070EC54F0EDECBC
:10A0100056F0DBCFE6FF2FEC8DF019D0FC0EDB50B5
:10A0200018E0010A24E1D950FA0FC0EC54F002E123
:10A03000FF0EED1806E030EC57F012EC8BF0E55215
:10A04000E55236EC59F0CBEC58F0E0EC8CF07ED9D0
:10A050000ED0EDEC56F0CBEC58F0FEEC8BF0146E1D
:10A06000060EE15E1450CDEC8CF00009FCE0E2D06D
:10A07000DCD8120EE126FC0EDB500DE0010A4EE1A9
:10A0800036EC59F0DBCFE6FFE6EC57F0CBEC58F0BE
:10A09000DEEC55F043D0D950FD0FC0EC54F002E196
:10A0A000FF0EED1802E070EC54F0100EF36EDB6E54
:10A0B000110EDB6AD950F70FEFD830E04BDBF70E0B
:10A0C000DBCF16F0F80EDED80CE2F70EDBCF08F08F
:10A0D000F80EDBCF09F0100E08C0DBFF110E09C02F
:10A0E000DBFFE5EC55F0E6EC57F0DBCFE6FF7EDA80
:10A0F000DEEC55F0E5EC55F079DACBEC57F02ADBE5
:10A10000166AD950F90F27D9EE221650EE2222DB1B
:10A11000D950F70F70EC56F014D9CCD7120EE15C81
:10A1200002E2E16AE552E16E85D0040EDBCFE9FF81
:10A13000050EDBCFEAFF140EEA02F3CFEAFFE902D5
:10A14000F3CFE9FFF450EA26C40EE926020EEA2214
:10A150001200FD0EDBCFE9FFFE0EDBCFEAFF12009F
:10A1600018EC56F0020ED8801456000E1556140E38
:10A170001502F3CF15F01402F3CF14F0F4501526A6
:10A18000F3CFE6FF15C0E6FF010EE66EE76E6DEC5D
:10A1900058F0E7501626000E1722140E1702F3CFC0
:10A1A00017F01602F3CF16F0F4501726C40E162639
:10A1B000020E17228EEC58F0010EE66E040EDBCF75
:10A1C00018F0050EDBCF19F0140E1902F3CF19F0B9
:10A1D0001802F3CF18F0F4501926C40E1826020EF8
:10A1E000192218C0E6FF19C0E6FF5FEC58F0020123
:10A1F000FC6BFD6B120075EC56F054EC3AF0E55236
:10A20000120018EC59F0EFCFF6FFEE2AEFCFF7FF70
:10A21000000EEE22EFCFF8FFEE2208000E0EF5CF73
:10A22000DBFF1200020E12EF59F0D9CFE6FFE1CFAB
:10A23000D9FF1200E552E7CFD9FF12000A0E146EC3
:10A24000CD0E156E010E166EDFCF17F0186A196A63
:10A25000060E0C6E0D6A0E6A17C007F018C008F0E3
:10A2600019C009F020EFE1F0B7DE146E080EE15ED0
:10A2700014501200E96EDACFEAFF1200E926000E50
:10A28000EA221200DBCF17F0AAEF57F0E66E12ECCD
:10A2900045F0E552E552120070EC56F0EE50ED102C
:10A2A0001200156E010E1426000E15221200DBCFCF
:10A2B000E6FFFD0EDBCFE6FF1200040E14C0DBFF4D
:10A2C000050E15C0DBFF1200D9CFE9FFDACFEAFF98
:10A2D00012006AEC57F0070E18EF57F046EC56F0F4
:10A2E0000E0E0301CF27270ED023070ED123000E19
:10A2F000D223120014500424F36E15500520F46E7E
:10A3000016500620F86EF4CFF7FFF3CFF6FF1200D9
:10A3100075EC56F09FEC3CF0E5521200C151C35D64
:10A32000146EC451C255156E120006EC59F045EC7E
:10A3300057F062EC56F0C3C3E6FFC4C3E6FF2FEF4D
:10A3400058F01450EE5E1550ED5A1200E552E552E9
:10A35000E552E552120070EC56F01450EE261550FE
:10A360001200FB0EDBCFE9FFFC0EDBCFEAFF120091
:10A37000FB0EDBCFE6FFFC0EDBCFE6FF1200C15188
:10A38000C35D166EC451C255176E120075EC56F0BF
:10A3900042EC3EF0E5521200260EDBCF14F0270E01
:10A3A000DBCF15F01200FB0EDBCF16F0FC0EDBCF7F
:10A3B00017F00A0E4AEC57F00B0EDB501720156E03
:10A3C000BA51AE25186EBB51AF21196EA0EF58F0EF
:10A3D000FB0EDBCFE6FFFC0EDBCFE6FFFD0EDBCF97
:10A3E000E6FF12000F0EDBCF9EF3100EDBCF9FF3C4
:10A3F000110EDBCFA0F3120EDBCFA1F31200DF5062
:10A40000146E156A070E145C000E15581200FC0E2F
:10A41000DBCFE9FFDB2AFD0EDBCFEAFF1200020EE5
:10A4200014C0DBFF030E15C0DBFF1200F3CF14F0E6
:10A43000F4CF15F0120024EC59F022EC57F0DE5066
:10A44000165C146EDD501758F2EC56F0040EE15C09
:10A45000120014C0DFFF010E15C0DBFF020E16C094
:10A46000DBFF030E17C0DBFF1200DCC3E6FFB3EC1B
:10A4700057F0010EE66E120014509E5F15509F5B60
:10A480001650A05B1750A15B1200DBCFF4FFF35016
:10A49000F45C1200E96E000EDA20EA6E12006AEC3B
:10A4A00057F0240E18EF57F0DB50CE21156E4BEC11
:10A4B00058F052EC58F0C1EF57F0B251B025166E7B
:10A4C000B351B121176E1650A825146E1750A9214B
:10A4D00095EF57F0C7ECE3F00301CF51065C146E23
:10A4E000D0510758156ED1510858166ED2510958DF
:10A4F000176E0001800E17141200C351C55D166E51
:10A50000C651C455176ECD51CB5D186ECC51CE558A
:10A51000196EF7EC56F0156E1200CB250001146E83
:10A520000B0EDB500301CC21000145EC57F0C1EFCD
:10A5300056F0E00E146E0D0EDBCFE7FF1450E72649
:10A540000D0EE7CFDBFF1200E00E146E0E0EDBCF18
:10A55000E7FF1450E7260E0EE7CFDBFF120068DBA3
:10A56000030E145C000E15581200DCC3E6FFC7C3CF
:10A57000E6FFC8C3E6FF1200040EDBCFE6FF050EC0
:10A58000DBCFE6FF12000A0EDBCF14F00B0EDBCFA1
:10A5900015F01200EECF14F0EFCF15F01200156E8B
:10A5A000260E14C0DBFF270E15C0DBFF280EACC340
:10A5B000DBFF290EADC3DBFF40EF57F0130EDBCFFF
:10A5C000A2F3140EDBCFA3F3150EDBCFA4F3160E0C
:10A5D000DBCFA5F3A22B000EA323A423A5231200F7
:10A5E000DBCFE6FFFA0EDBCFE6FF1200D9CFE6FFA6
:10A5F000DACFE6FF1200E66E000EDA20E66E1200F9
:10A60000F36E030EF3CFDBFF1200176EEBEC58F086
:10A6100095EF57F06DEC58F0DE501624146EDD50B7
:10A620001720F2EF56F0C7ECE3F0065003019A252D
:10A63000CF6F07509B21D06F08509C21D16F0950DC
:10A640009D21D26F1200DE50C7250001146EDD502F
:10A650000301C8210001156E0301C351145CC451EC
:10A6600015581200F3CFDBFFDBCF14F0040EDBCF65
:10A6700015F0050EEEEF57F074EC58F0FA0E08C026
:10A68000DBFFFB0E09C0DBFF0F0EDB501200060ED6
:10A69000DBCF18F0070EDBCF19F0080EDB50185C8B
:10A6A000166E090EDB501958176E120074EC58F034
:10A6B000F90E08C0DBFFFA0E09C0DBFF100EDB50FD
:10A6C000120079DBDBCF17F0FC0EE4DBFD0EDB5074
:10A6D0001720156E1200DBCF09F0060E08C0DBFF55
:10A6E000070E09C0DBFF12003DEC58F0040DF350DB
:10A6F00012001450EE5C1550EE581650EE581750DC
:10A70000EE58120084ECD8F0166E060EE15E16507C
:10A71000120084ECD8F0146E060EE15E14501200A4
:10A72000E4DAADEC3CF0E5521200FA0EDBCF14F0A7
:10A73000FB0EDBCF15F01200DBCF17F01650145CC8
:10A74000175015581200260EDBCF08F0270EDBCF6E
:10A7500009F01200100EDBCF14F0110EDBCF15F054
:10A760001200DFCFE6FF54EC3AF0E5521200B00ED3
:10A77000E66E030EE66E1200DECF14F0DDCF15F0AC
:10A78000120088ECA1F0E552E5521200EECFE6FF90
:10A79000EFCFE6FF1200DBCF15F0000114500301EC
:10A7A000A227000115500301A323000EA423A52313
:10A7B0001200FB0EDBCFB0F3FC0EDBCFB1F3FD0ECE
:10A7C000DBCFB2F3FE0EDBCFB3F31200DBCF14F01E
:10A7D000020EDBCF15F0030EEEEF57F0280EDBCFA5
:10A7E00008F0290EDBCF09F0260E08C0DBFF270E8C
:10A7F00009C0DBFF12000A0EDB500301CB2500016C
:10A80000166E0B0EDB500301CC210001176E1200F7
:10A81000D890173216329ED3D3EC8CF0E76E010E2F
:10A82000E7CFDBFFDB501200DBCF15F0166A176AAB
:10A83000120014C0F3FF15C0F4FF1200DBCFDEFFDF
:10A84000DBCFDDFF1200DB50146E156AD950120009
:10A85000EECF16F0EFCF17F01200E66EA3511C0DED
:10A86000F3CFE9FFF4CFEAFF000EE926020EEA2259
:10A870001200A651C95D186ECA51A755196EF7EF9F
:10A8800056F0C951A65D146EA751CA551200FDDAE3
:10A89000DCC3E6FFC3C3E6FFC4C3E6FF1200D1EC8E
:10A8A000E3F003010650D55D146E0750D659156EBE
:10A8B000E8341200145003019E27000115500301D3
:10A8C0009F23000EA023A1231200DBCF1BF00A0E52
:10A8D000DB501A24186E0B0EDB501B20196E120071
:10A8E000FD0EDBCFE6FF01DA02EC8BF0E552E5521C
:10A8F0001200020EF3CFDBFF030EF4CFDBFF1200DA
:10A90000DCC3E6FFCDC3E6FFCEC3E6FF1200156E43
:10A910000301C1EF57F0DBCF19F0A0EF58F0FA0EAA
:10A92000DBCF08F0FB0EDBCF09F01200F90EDBCF16
:10A9300008F0FA0EDBCF09F01200E66EE66A05ECCD
:10A94000DBF0E552E5521200260EDBCFE6FF270EC4
:10A95000DBCFE6FF1200240EDBCFE6FF250EDBCFB8
:10A96000E6FF1200FB0EDBCF08F0FC0EDBCF09F098
:10A970001200050EDBCF15F00001800E1514120039
:10A98000AFD9FF0EEE18120014C0E6FF15C0E6FFA7
:10A990001200C1C3C7F3C2C3C8F31200040EDB6ABE
:10A9A000050EDB6A120014500008000E1554120048
:10A9B000F3CFEEFF15C0EDFF1200C55D146EC6515A
:10A9C0001200140EEECFDBFF150EEECFDBFF160EDE
:10A9D000EECFDBFF1200CB51CD5D146ECE51CC55C6
:10A9E0007BEF58F0DECF16F0DDCF17F0B3D2DBCF20
:10A9F00009F0020E08C0DBFF030E09C0DBFF1200E6
:10AA0000DBCF09F00A0E08C0DBFF0B0E09C0DBFF2D
:10AA10001200C3C3DEFFC4C3DDFF040EDB68050EF6
:10AA2000DB6812000D0EEFCFDBFF010EF36E0F0E91
:10AA3000F3CFDBFF1200E9CF14F0EACF15F0E9CF36
:10AA4000E6FFEACFE6FF120003DBBD511618120045
:10AA5000000EEE5C000EEE58000EEE58000EEE58A2
:10AA60001200EE501426EE501522EE501622EE5033
:10AA7000172212000A0E3BEC59F00B0EDB50175850
:10AA8000156E1200D950100F146E0C0EDB50120010
:10AA9000DB50E76E0F0EE7CFDBFF1200D950110F2E
:10AAA000146E0D0EDB501200CD51CB5DCE51CC5942
:10AAB0001200DBCF15F0145015101200E552E7CF4D
:10AAC00017F0E552E7CF16F016501200030EDBCF59
:10AAD000E6FF12EC45F0E552E5521200260EBDC32A
:10AAE000DBFF270EBEC3DBFFD9851200156E240ED7
:10AAF00014C0DBFF250E15C0DBFF1200E66E0F0E43
:10AB0000E66E02EC8BF0E552E5521200145E000E88
:10AB1000155A1200BF6B2D0E9A6F9B6B9C6B9D6B31
:10AB20001200D950FD0FE66EFF0EDA20E66E12001D
:10AB300038EC50F0146E080EE15E14501200080E4E
:10AB400008C0DBFF090E09C0DBFF1200BF2BD89045
:10AB50009A379B379C379D371200F4CFDBFF0C0EE2
:10AB6000E66EE66AD9501200240E08C0DBFF250EFF
:10AB700009C0DBFF120064EC49F0F3CFBDF3F4CF62
:10AB8000BEF31200FB0EDBCFAEF3FC0EDBCFAFF358
:10AB900012000A0EDBCFBAF30B0EDBCFBBF31200B1
:10ABA000BA51AE25146EBB51AF21156E1200D1EC17
:10ABB000E3F006C0D5F307C0D6F31200AFECD8F02F
:10ABC000146E070EE15E14501200100EDBCFE6FF8C
:10ABD000110EDBCFE6FF1200010E1626000E172223
:10ABE0001200CBC3CDF3CCC3CEF31200C3C3CDF35D
:10ABF000C4C3CEF31200DB500301CD25146E120046
:10AC0000C9C3A6F3CAC3A7F3120014C0DEFF15C060
:10AC1000DDFF1200F36E190EF3CFDBFF1200C1C38C
:10AC2000A6F3C2C3A7F312000A0EE66EE66A12008C
:10AC300014DBDBCF15F01200A9EC50F0020E3EEF52
:10AC400051F03EEC51F0EECFE6FFEECFE6FF9EDD99
:10AC5000ABECA1F0A6EC51F006C014F007C015F063
:10AC600008C016F009C017F0A9EF50F03AEC51F007
:10AC70001450EE261550ED221200D950060F3AEF6F
:10AC800051F03AEC51F0EE50ED101200C7ECE3F049
:10AC900006C0CFF307C0D0F308C0D1F309C0D2F388
:10ACA0001200C3518ADEC45551EF51F0D9500F0F35
:10ACB0003AEC51F09E51EE18120095EC50F0100E47
:10ACC0003EEF51F0E66AE668E668DCC3E6FF120094
:10ACD000DBCF17F0040ECFDA050EDB501758120049
:10ACE000E96EFF0EDA20EA6E1200FE0EDBCFE6FF01
:10ACF0001200D9500A0F3AEC51F0FB0EEECFDBFFF9
:10AD0000FC0EEECFDBFFFD0EEECFDBFF01EF51F0CF
:10AD1000156ED950280FB8DACCEC51F0280EDBCFE5
:10AD200016F0290E42EF51F0060E88DDDB50C55DAE
:10AD3000146E070EDB50C65900011CEF59F00A0EC5
:10AD4000DBCF08F00B0EDBCF09F0FC0E08C0DBFFF9
:10AD5000FD0E09C0DBFF07EF52F00F0EDBCF18F03E
:10AD6000100EDBCF19F0110EDBCF1AF0120EDBCF75
:10AD70001BF064EF51F068DA64EC51F0EE50ED1026
:10AD80001200ECEC4FF0166E080EE15E1650120049
:10AD9000010EE66E100E46EF51F0FC0E57EC51F02E
:10ADA00034EF51F0A9EC50F00E0E3EEF51F015ECDF
:10ADB00051F0FBEF50F0FA0EDBCF16F0FB0E120055
:10ADC000DCC3E6FFA6C3E6FFA7C3E6FFE66AAC0E58
:10ADD000E66E0F0EE66E34EF51F048DAF0EC52F00A
:10ADE000FB0E1200156E14C0F3FFF46E1200185023
:10ADF000165C146E19501758120014244AEC52F0C5
:10AE0000EF50F36E1200C751C35D146EC451C855A4
:10AE1000156E5DEC51F0BCEF52F0FBEC52F0D2EC51
:10AE2000A1F0A6EC51F016EC52F0141E151E120003
:10AE30001426000E15221622172214C0D3F315C0B3
:10AE4000D4F31200020EDBCF16F0030EDBCF17F0A7
:10AE5000120012EC51F0F90EDBCF16F0FA0E1200D0
:10AE6000FA0EDBCFE6FFFB0EDBCFE6FF120015ECA0
:10AE700051F0060EE1261200F36E0D0E45EF52F072
:10AE8000C951A65DCA51A7591200156E14C0E6FF3C
:10AE9000E66E1200DB501624146E12001C0D16EC28
:10AEA00052F0000E1426020E1522C4EF54F0010ECB
:10AEB000E66EFC0E57EC51F0B5EC52F034EF51F069
:10AEC000DB500F0115244AEC52F0EFCF14F0610E65
:10AED000145C1200D88BD1ECE3F006C014F007C06C
:10AEE00015F0166A176A12009FDEB8EC51F03FDCCD
:10AEF00089EF53F0010EE66E110E46EC51F003019E
:10AF0000AC51AD111200020E99DC8CD1EECF14F0D1
:10AF1000EECF15F09DDC95EF50F0E66A000EE66E80
:10AF2000E66AE0EC8CF0A6EF51F0156E1450AA1909
:10AF3000DA6F1550AB19DB6F1200020F44EF59F0B6
:10AF4000610EF36E0E0E45EF52F095EC50F00A0EC6
:10AF50003EEF51F01450165C15501758120064EC77
:10AF600051F0A1EF51F0DECFE6FFDDCFE6FF12009A
:10AF700015EC51F0040EE1261200D950FC0F4CEFF5
:10AF800051F01450C55D1550C65912008EEC51F0A9
:10AF9000166A176A12002FEC8DF0A6EF51F001EC43
:10AFA00051F0010EF36E100EF3CFDBFF1200A3EC95
:10AFB00053F008500301A6270950A7231200A9EC5B
:10AFC00050F00C0E3EEC51F074EF53F0F90EDBCF65
:10AFD000E6FFFA0EDBCFE6FFFB0E1200DBCF16F02A
:10AFE0001450155C000E1658120005C018F006C06B
:10AFF00019F07AEF51F012EC51F0BFEC51F008EF7C
:10B0000054F0E8EC51F0B5EC52F098EF55F0DBCF8E
:10B01000E6FFE66A35EC52F0D95012000E0EDB5016
:10B02000F36E0C0E45EF52F0DB5017244AEC52F051
:10B03000EF507A081200000E172051EC51F019EF72
:10B0400054F0CCEC51F01450BD5D1550BE591200B7
:10B05000260EDBCF16F0270EDBCF17F01200ECEC3C
:10B060004FF0186E080EE15E185012008EEC51F091
:10B070001450A65F1550A75B1200EF50F00BE8428A
:10B08000E842E842E8421200D9500F0F3AEC51F082
:10B09000EE509E191200060E14C0DBFF070E15C0FD
:10B0A000DBFF1200060EDBCF14F0070EDBCF15F02E
:10B0B0001200CBC3E6FFCCC3E6FF34EF51F0ECEC5B
:10B0C0004FF01A6E080EE15E1A50120012EC51F0A9
:10B0D000CD51145CCE5115581200040EDBCF16F082
:10B0E000050EDBCF17F01200080EDBCF08F0090EBB
:10B0F000DBCF09F01200156E1406000E155A12006F
:10B10000FBEC50F090EF53F064EC51F0010EEE18B0
:10B11000120088EC51F00301D981120016C0E6FF3D
:10B1200017C0E6FF1200FBEC50F0C6EF51F0E66EE0
:10B13000E66AF6EF52F03EEC51F006C0EEFF120068
:10B140001450185C155019581200C6EC53F0C1EC9D
:10B1500053F016EF52F00C0EDBCF14F00D0E14EC82
:10B1600054F03DEF56F083DE19DCCADF79EC54F081
:10B17000D950020F41EF56F023EC54F0040F84D85D
:10B18000D950040F41EF56F015C0EEFF16C0EEFF88
:10B1900017C0EEFF120057EC51F075EF56F04CDD82
:10B1A000CAEF52F064EC51F0EE500301C727EE50A5
:10B1B000C823120062DDEE06000EEE5AEE5AEE5A79
:10B1C000120036DDCCDEC9EF54F080EC54F0010EF5
:10B1D000E66ECDEF56F0F80E5DDEF90EDB5017206F
:10B1E000120012EC51F0E7DD9CEF53F05ADD45DD23
:10B1F000A1EF51F0D7DDEECFACF3EDCFADF3120000
:10B200003CDDD890030EEB50000A1200FB0EDBCFA2
:10B2100016F0FC0E68EF56F0FB0E3CDEFC0EDB5029
:10B2200017201200DBCF14F0030EDBCF15F0120055
:10B23000D950FB0F70EF56F051EC51F05DEF51F02B
:10B240003CDDEE50ED101200F3CFDEFFF4CFDDFF5A
:10B250001200D8EC54F0A9EF50F0040EDBCF14F03C
:10B26000050E1200B8EC51F062EF56F0F70EDBCF8E
:10B27000E6FFF80E1200DB50165C146E12003EEC76
:10B2800051F063DFA9EF50F03AEC51F0A1EF51F02B
:10B29000DFEC6AF0FB0EDBCF07F0FC0EDBCF08F033
:10B2A000FD0EDBCF09F0FE0EDBCF0AF0A70E07186C
:10B2B00005E1085003E1095001E10A5002E122EFE3
:10B2C00062F0A60E071805E1085003E1095001E1FC
:10B2D0000A5002E120EF62F0A50E071805E10850C0
:10B2E00003E1095001E10A5002E115EF62F0A40EFA
:10B2F000071805E1085003E1095001E10A5002E195
:10B300000FEF62F0A30E071805E1085003E10950A2
:10B3100001E10A5002E10DEF62F0A20E071805E10B
:10B32000085003E1095001E10A5002E107EF62F021
:10B33000A10E071805E1085003E1095001E10A5088
:10B3400002E102EF62F0A00E071805E1085003E1E8
:10B35000095001E10A5002E100EF62F09F0E071868
:10B3600005E1085003E1095001E10A5002E1FEEF56
:10B3700061F09E0E071805E1085003E1095001E154
:10B380000A5002E1FCEF61F09D0E071805E108503C
:10B3900003E1095001E10A5002E1F7EF61F09C0E70
:10B3A000071805E1085003E1095001E10A5002E1E4
:10B3B000F5EF61F09B0E071805E1085003E1095015
:10B3C00001E10A5002E1F3EF61F09A0E071805E17E
:10B3D000085003E1095001E10A5002E1F1EF61F088
:10B3E000990E071805E1085003E1095001E10A50E0
:10B3F00002E1ECEF61F0980E071805E1085003E157
:10B40000095001E10A5002E1EAEF61F0970E0718D6
:10B4100005E1085003E1095001E10A5002E1E8EFBB
:10B4200061F0960E071805E1085003E1095001E1AB
:10B430000A5002E1E6EF61F0950E071805E10850A9
:10B4400003E1095001E10A5002E1E1EF61F0940EDD
:10B45000071805E1085003E1095001E10A5002E133
:10B46000DFEF61F0930E071805E1085003E1095082
:10B4700001E10A5002E1DDEF61F0920E071805E1EB
:10B48000085003E1095001E10A5002E1DBEF61F0ED
:10B49000910E071805E1085003E1095001E10A5037
:10B4A00002E1D6EF61F0900E071805E1085003E1C4
:10B4B000095001E10A5002E1D4EF61F08F0E071844
:10B4C00005E1085003E1095001E10A5002E1D2EF21
:10B4D00061F08E0E071805E1085003E1095001E103
:10B4E0000A5002E1D0EF61F08D0E071805E1085017
:10B4F00003E1095001E10A5002E1CBEF61F08C0E4B
:10B50000071805E1085003E1095001E10A5002E182
:10B51000C9EF61F08B0E071805E1085003E10950EF
:10B5200001E10A5002E1C7EF61F08A0E071805E158
:10B53000085003E1095001E10A5002E1C5EF61F052
:10B54000890E071805E1085003E1095001E10A508E
:10B5500002E1C0EF61F0880E071805E1085003E131
:10B56000095001E10A5002E1BEEF61F0870E0718B1
:10B5700005E1085003E1095001E10A5002E1BCEF86
:10B5800061F0860E071805E1085003E1095001E15A
:10B590000A5002E1BAEF61F0850E071805E1085084
:10B5A00003E1095001E10A5002E1B5EF61F0840EB8
:10B5B000071805E1085003E1095001E10A5002E1D2
:10B5C000B3EF61F0830E071805E1085003E109505D
:10B5D00001E10A5002E1B1EF61F0820E071805E1C6
:10B5E000085003E1095001E10A5002E1AFEF61F0B8
:10B5F000810E071805E1085003E1095001E10A50E6
:10B6000002E1AAEF61F0800E071805E1085003E19E
:10B61000095001E10A5002E1A8EF61F07F0E07181E
:10B6200005E1085003E1095001E10A5002E1A6EFEB
:10B6300061F07E0E071805E1085003E1095001E1B1
:10B640000A5002E1A4EF61F07D0E071805E10850F1
:10B6500003E1095001E10A5002E19FEF61F07C0E25
:10B66000071805E1085003E1095001E10A5002E121
:10B670009DEF61F07B0E071805E1085003E10950CA
:10B6800001E10A5002E19BEF61F07A0E071805E133
:10B69000085003E1095001E10A5002E199EF61F01D
:10B6A000790E071805E1085003E1095001E10A503D
:10B6B00002E194EF61F0780E071805E1085003E10C
:10B6C000095001E10A5002E192EF61F0770E07188C
:10B6D00005E1085003E1095001E10A5002E190EF51
:10B6E00061F0760E071805E1085003E1095001E109
:10B6F0000A5002E18EEF61F0750E071805E108505F
:10B7000003E1095001E10A5002E189EF61F0740E92
:10B71000071805E1085003E1095001E10A5002E170
:10B7200087EF61F0730E071805E1085003E1095037
:10B7300001E10A5002E185EF61F0720E071805E1A0
:10B74000085003E1095001E10A5002E183EF61F082
:10B75000710E071805E1085003E1095001E10A5094
:10B7600002E17EEF61F0700E071805E1085003E179
:10B77000095001E10A5002E17CEF61F06F0E0718F9
:10B7800005E1085003E1095001E10A5002E17AEFB6
:10B7900061F06E0E071805E1085003E1095001E160
:10B7A0000A5002E178EF61F06D0E071805E10850CC
:10B7B00003E1095001E10A5002E175EF61F06C0EFE
:10B7C000071805E1085003E1095001E10A5002E1C0
:10B7D00073EF61F06B0E071805E1085003E10950A3
:10B7E00001E10A5002E16FEF61F06A0E071805E10E
:10B7F000085003E1095001E10A5002E16DEF61F0E8
:10B80000690E071805E1085003E1095001E10A50EB
:10B8100002E16BEF61F0680E071805E1085003E1E3
:10B82000095001E10A5002E169EF61F0670E071863
:10B8300005E1085003E1095001E10A5002E166EF19
:10B8400061F0660E071805E1085003E1095001E1B7
:10B850000A5002E164EF61F0650E071805E1085037
:10B8600003E1095001E10A5002E15EEF61F0640E6C
:10B87000071805E1085003E1095001E10A5002E10F
:10B8800058EF61F0630E071805E1085003E1095015
:10B8900001E10A5002E156EF61F0620E071805E17E
:10B8A000085003E1095001E10A5002E154EF61F050
:10B8B000610E071805E1085003E1095001E10A5043
:10B8C00002E152EF61F0600E071805E1085003E154
:10B8D000095001E10A5002E150EF61F05F0E0718D4
:10B8E00005E1085003E1095001E10A5002E14EEF81
:10B8F00061F05E0E071805E1085003E1095001E10F
:10B900000A5002E14CEF61F05D0E071805E10850A6
:10B9100003E1095001E10A5002E14AEF61F05C0ED7
:10B92000071805E1085003E1095001E10A5002E15E
:10B9300048EF61F05B0E071805E1085003E109507C
:10B9400001E10A5002E146EF61F05A0E071805E1E5
:10B95000085003E1095001E10A5002E144EF61F0AF
:10B96000590E071805E1085003E1095001E10A509A
:10B9700002E142EF61F0580E071805E1085003E1BB
:10B98000095001E10A5002E140EF61F0570E07183B
:10B9900005E1085003E1095001E10A5002E13EEFE0
:10B9A00061F0560E071805E1085003E1095001E166
:10B9B0000A5002E13CEF61F0550E071805E108500E
:10B9C00003E1095001E10A5002E139EF61F0540E40
:10B9D000071805E1085003E1095001E10A5002E1AE
:10B9E00036EF61F0530E071805E1085003E10950E6
:10B9F00001E10A5002E133EF61F0520E071805E150
:10BA0000085003E1095001E10A5002E130EF61F012
:10BA1000510E071805E1085003E1095001E10A50F1
:10BA200002E12AEF61F0500E071805E1085003E12A
:10BA3000095001E10A5002E128EF61F04F0E0718AA
:10BA400005E1085003E1095001E10A5002E126EF47
:10BA500061F04E0E071805E1085003E1095001E1BD
:10BA60000A5001E1F0D34D0E071805E1085003E13B
:10BA7000095001E10A5001E1E3D34C0E071805E13A
:10BA8000085003E1095001E10A5001E1D2D34B0E05
:10BA9000071805E1085003E1095001E10A5001E1EE
:10BAA000C4D34A0E071805E1085003E1095001E12B
:10BAB0000A5001E1B8D3490E071805E1085003E127
:10BAC000095001E10A5001E1ABD3480E071805E126
:10BAD000085003E1095001E10A5001E19BD3470EF0
:10BAE000071805E1085003E1095001E10A5001E19E
:10BAF0008FD3460E071805E1085003E1095001E114
:10BB00000A5001E183D3450E071805E1085003E10F
:10BB1000095001E10A5001E177D3440E071805E10D
:10BB2000085003E1095001E10A5001E16BD3430ED3
:10BB3000071805E1085003E1095001E10A5001E14D
:10BB40005FD3420E071805E1085003E1095001E1F7
:10BB50000A5001E153D3410E071805E1085003E1F3
:10BB6000095001E10A5001E147D3400E071805E1F1
:10BB7000085003E1095001E10A5001E13BD33F0EB7
:10BB8000071805E1085003E1095001E10A5001E1FD
:10BB90002FD33E0E071805E1085003E1095001E1DB
:10BBA0000A5001E123D33D0E071805E1085003E1D7
:10BBB000095001E10A5001E117D33C0E071805E1D5
:10BBC000085003E1095001E10A5001E10BD33B0E9B
:10BBD000071805E1085003E1095001E10A5001E1AD
:10BBE000FFD23A0E071805E1085003E1095001E1C0
:10BBF0000A5001E1F3D2390E071805E1085003E1BC
:10BC0000095001E10A5001E1E7D2380E071805E1B9
:10BC1000085003E1095001E10A5001E1DBD2370E7F
:10BC2000071805E1085003E1095001E10A5001E15C
:10BC3000CFD2360E071805E1085003E1095001E1A3
:10BC40000A5001E1C3D2350E071805E1085003E19F
:10BC5000095001E10A5001E1B7D2340E071805E19D
:10BC6000085003E1095001E10A5001E1ABD2330E63
:10BC7000071805E1085003E1095001E10A5001E10C
:10BC80009FD2320E071805E1085003E1095001E187
:10BC90000A5001E193D2310E071805E1085003E183
:10BCA000095001E10A5001E187D2300E071805E181
:10BCB000085003E1095001E10A5001E17AD22F0E48
:10BCC000071805E1085003E1095001E10A5001E1BC
:10BCD00067D22E0E071805E1085003E1095001E173
:10BCE0000A5001E15BD22D0E071805E1085003E16F
:10BCF000095001E10A5001E14CD22C0E071805E170
:10BD0000085003E1095001E10A5001E140D22B0E35
:10BD1000071805E1085003E1095001E10A5001E16B
:10BD200031D22A0E071805E1085003E1095001E15C
:10BD30000A5001E125D2290E071805E1085003E158
:10BD4000095001E10A5001E116D2280E071805E159
:10BD5000085003E1095001E10A5001E10AD2270E1F
:10BD6000071805E1085003E1095001E10A5001E11B
:10BD7000FBD1260E071805E1085003E1095001E147
:10BD80000A5001E1EFD1250E071805E1085003E143
:10BD9000095001E10A5001E1E0D1240E071805E144
:10BDA000085003E1095001E10A5001E1D4D1230E0A
:10BDB000071805E1085003E1095001E10A5001E1CB
:10BDC000C5D1220E071805E1085003E1095001E131
:10BDD0000A5001E1B9D1210E071805E1085003E12D
:10BDE000095001E10A5001E1AAD1200E071805E12E
:10BDF000085003E1095001E10A5001E19ED11F0EF4
:10BE0000071805E1085003E1095001E10A5001E17A
:10BE10008FD11E0E071805E1085003E1095001E11A
:10BE20000A5001E183D11D0E071805E1085003E116
:10BE3000095001E10A5001E174D11C0E071805E117
:10BE4000085003E1095001E10A5001E168D11B0EDD
:10BE5000071805E1085003E1095001E10A5001E12A
:10BE600059D11A0E071805E1085003E1095001E104
:10BE70000A5001E14DD1190E071805E1085003E100
:10BE8000095001E10A5001E13ED1180E071805E101
:10BE9000085003E1095001E10A5001E132D1170EC7
:10BEA000071805E1085003E1095001E10A5001E1DA
:10BEB00023D1160E071805E1085003E1095001E1EE
:10BEC0000A5001E117D1150E071805E1085003E1EA
:10BED000095001E10A5001E108D1140E071805E1EB
:10BEE000085003E1095001E10A5001E1FCD0130EB2
:10BEF000071805E1085003E1095001E10A5001E18A
:10BF0000EFD0120E071805E1085003E1095001E1D6
:10BF10000A5001E1E1D0110E071805E1085003E1D4
:10BF2000095001E10A5001E1D5D0100E071805E1D2
:10BF3000085003E1095001E10A5001E1C8D00F0E99
:10BF4000071805E1085003E1095001E10A5001E139
:10BF5000B8D00E0E071805E1085003E1095001E1C1
:10BF60000A5001E1A8D00D0E071805E1085003E1C1
:10BF7000095001E10A5001E19CD00C0E071805E1BF
:10BF8000085003E1095001E10A5001E190D00B0E85
:10BF9000071805E1085003E1095001E10A5001E1E9
:10BFA00084D00A0E071805E1085003E1095001E1A9
:10BFB0000A5001E178D0090E071805E1085003E1A5
:10BFC000095001E10A506DE0080E071805E108501C
:10BFD00003E1095001E10A5062E0070E071805E18C
:10BFE000085003E1095001E10A5057E0060E071816
:10BFF00005E1085003E1095001E10A504BE0050E4C
:10C00000071805E1085003E1095001E10A503FE03B
:10C01000040E071805E1085003E1095001E10A5038
:10C0200033E0030E071805E1085003E1095001E170
:10C030000A5027E0020E071805E1085003E10950F5
:10C0400001E10A501BE0010E071805E1085003E169
:10C05000095001E10A500FE0075001E0FBD1085000
:10C0600001E0F8D1095001E0F5D10A5001E0F2D128
:10C07000B3EC73F0FFD175EC73F0FCD1DCEC70F035
:10C08000F9D195EC73F0F6D18BEC73F0F3D19FEC12
:10C0900073F0F0D1A9EC73F0EDD1000E0DD0010ECC
:10C0A0000BD0000E0FD0020E07D0010E0BD0030EE6
:10C0B00003D0020E07D0040EE66EE66ADFEC73F0E2
:10C0C000C6D1030EE66EE66A3CEC73F0C0D192EC8A
:10C0D0006CF06AD0000E01D0010EE66EE66A64D004
:10C0E00096EC6BF061D0010E01D0000EE66EE66AB0
:10C0F000020E5AD0010E01D0000EE66EE66A030E63
:10C1000053D0010E01D0000EE66EE66A040E4CD04C
:10C11000010E01D0000EE66EE66A050E45D0010E56
:10C1200001D0000EE66EE66A060E3ED0010E01D08A
:10C13000000EE66EE66A070E37D0010E01D0000E43
:10C14000E66EE66A080E30D0010E01D0000EE66EF3
:10C15000E66A090E29D0010E01D0000EE66EE66AED
:10C160000A0E22D0010E01D0000EE66EE66A0B0E1A
:10C170001BD0010E01D0000EE66EE66A0C0E14D044
:10C18000010E01D0000EE66EE66A0D0E0DD0010E16
:10C1900001D0000EE66EE66A0E0E06D0010E01D04A
:10C1A000000EE66EE66A0F0EE66EE66A08EC71F0C7
:10C1B00044D1EAEC6FF05ED1000E2DD0010E2BD0F1
:10C1C000020E29D0030E27D0040E25D0050E23D051
:10C1D000060E21D0070E1FD0080E1DD0090E1BD051
:10C1E0000A0E19D00B0E17D00C0E15D00D0E13D051
:10C1F0000E0E11D00F0E0FD0100E0DD0110E0BD051
:10C20000120E09D0130E07D0140E05D0150E03D050
:10C21000160E01D0170EE66EE66A5AEC71F017D1D1
:10C2200092EC6CF008D0000E01D0010EE66EE66ACA
:10C2300002D096EC6BF0E66EE66AE3EC70F0FDD0AF
:10C240001FEC71F017D1F5EC6FF014D1020E03D092
:10C25000000E01D0010EE66EE66A3DEC71F0F7D0FB
:10C2600026EC71F007D14FEC71F004D147EC71F07E
:10C2700001D182EC70F0FED0000E1BD0000E1FD05A
:10C28000010E17D0010E1BD0020E13D0020E17D0D4
:10C29000030E0FD0030E13D0040E0BD0040E0FD0DC
:10C2A000050E07D0050E0BD0060E03D0060E07D0E4
:10C2B000070EE66EE66A1FEC72F0C9D0070EE66E56
:10C2C000E66AA3EC70F0C3D0000EA2D092EC6CF042
:10C2D000B0D0000EA5D0000E03D0010E99D0010EF3
:10C2E000E66EE66AA6D0010E9BD096EC6BF0A1D06C
:10C2F000020E8ED0010E03D0020E92D0000EE66E1A
:10C30000E66A020E96D0030E83D0010E03D0030E10
:10C3100087D0000EE66EE66A030E8BD0040E78D04E
:10C32000010E03D0040E7CD0000EE66EE66A040E09
:10C3300080D0050E6DD0010E03D0050E71D0000E19
:10C34000E66EE66A050E75D0060E62D0010E03D0C9
:10C35000060E66D0000EE66EE66A060E6AD0070E7E
:10C3600057D0010E03D0070E5BD0000EE66EE66AD2
:10C37000070E5FD0080E4CD0010E03D0080E50D02F
:10C38000000EE66EE66A080E54D0090E41D0010E8A
:10C3900003D0090E45D0000EE66EE66A090E49D0BC
:10C3A0000A0E36D0010E03D00A0E3AD0000EE66E09
:10C3B000E66A0A0E3ED00B0E2BD0010E03D00B0EF8
:10C3C0002FD0000EE66EE66A0B0E33D00C0E20D096
:10C3D000010E03D00C0E24D0000EE66EE66A0C0EA1
:10C3E00028D00D0E15D0010E03D00D0E19D0000E61
:10C3F000E66EE66A0D0E1DD00E0E0AD0010E03D0B9
:10C400000E0E0ED0000EE66EE66A0E0E12D00F0E65
:10C41000E66EE66A0BEC72F01AD0010E07D00F0E32
:10C42000E66EE66A71EC72F012D0000EE66EE66A15
:10C430000F0EE66EE66A81EC72F0E552E55207D027
:10C44000000E01D0010EE66EE66AE0EC72F0E552F5
:10C45000E55210D0040EE66EE66A7A0EE66E3A0EEB
:10C46000E66E010EC0EC6DF073EC3DF0146E060E3E
:10C47000E15E1450E4EF6AF07E0EC0EC6DF0DFEC8C
:10C480003CF0E552E5521200DFEC6AF0020EE126C4
:10C49000060114691569816B010E815D1FE22CECA8
:10C4A0006BF0080EE66E8AC0E6FF8BC0E6FFE66A18
:10C4B000E66AE66AE66AE66A87EC3BF0146E080E06
:10C4C000E15E1450E66EA0EC6DF0EE52E552E750DE
:10C4D000EF6EAAEC6AF00601812BDED7020EE15C5A
:10C4E00002E2E16AE552E16EE4EF6AF0DFEC6AF045
:10C4F000E652DF6A010EDF5C33E249EC6DF0FE08C4
:10C500002DE049EC6DF0E66E25EC3CF0E5520009BB
:10C5100014E0DFCFE6FF27D8E55206012CEC6BF0E4
:10C52000FF0E145D02E07AEC6BF0FF0E155D02E089
:10C5300082EC6BF0040ECAEC6CF00AEC6BF0EF507E
:10C5400008E149EC6DF0E66E42EC3EF01BEC6BF05E
:10C5500005E0DFCFE6FF07D8E5522ED8DF2ACAD79D
:10C56000E552E4EF6AF0DFEC6AF0020EE126FE0E1F
:10C57000DB500601815D18E0AAEC6AF0FE0EDB508C
:10C580006BEC6DF012EC8BF0A3EC6DF0E0EC8CF04A
:10C59000DBEC6CF0E552EFEC6CF012EC8BF0E5525A
:10C5A000E552FE0EDBCF81F6020EE15C02E2E16AAB
:10C5B000E552E16EE4EF6AF0DFEC6AF0190EE12675
:10C5C00070EC6BF0A0EC6DF0EF500B0A01E1B5D30D
:10C5D000010A01E18DD3030A01E176D3010A01E1E9
:10C5E00070D30F0A01E1C9D2010A01E1AAD2030AFC
:10C5F00001E152D2010A01E147D2070A01E129D241
:10C60000010A01E194D1030A27E0010A01E0A3D362
:10C6100055EC6AF042EC3EF0E552D1EC6CF005ECE2
:10C620006BF0EE50ED1001E196D306011A0E106F7B
:10C63000060E116FABEC6CF0010EEF6E1769166B06
:10C6400092EC6AF00C690D690E690F6997EC6CF059
:10C650007E6B050ECAEC6CF0DAEC6AF00A0EC0ECE8
:10C660006DF0AAEC6BF00001F31C11E1151C0FE159
:10C67000B6EC6CF04DEC6DF002E111EC6DF0C7EC36
:10C680006AF002E642EC6BF001E365D31DD292EC56
:10C690006AF0E66AE66EE66AE66EE66A31EC6DF02E
:10C6A00005EC6BF0050E99EC6BF003E2050EDE6E07
:10C6B000DD6A14EC6BF035EC6BF0B6EC6CF0DCEC96
:10C6C0006BF0030EE66EE66AA30EE66E360EE66EBD
:10C6D000010EE66E35EC6BF03CEC6CF003E106010C
:10C6E000186B15D0040EE66EE66A9E0EE66E360EE8
:10C6F000E66E010EE66E35EC6BF03CEC6CF004E19E
:10C700000601010E186F03D00601070E1ED2DAECE7
:10C710006AF031EC6DF020EC6CF03F0EC0EC6DF087
:10C72000F7EC6CF020EC6BF051EC6DF05AEC6CF027
:10C730001850165C1950175803E2C5EC6CF002D083
:10C74000E8EC6AF09CEC6CF005EC6BF0580E99ECA0
:10C750006BF001E2D1D0C7EC6DF020EC6BF0FEEC99
:10C760006CF056EC6DF02AEC6DF035EC6BF05BEC98
:10C770006DF020EC6BF056EC6BF002E0B2EC6BF07D
:10C78000FF0E0601145D23E156EC6BF008E0F2ECBD
:10C790006AF001E3DB2A56EC6DF02F0EEF6E61ECD0
:10C7A0006CF036EC6DF0D6EC6CF05FECD9F0166EF8
:10C7B000050EE15E165061EC6CF0F8EC6BF09EEC4F
:10C7C0006BF00750EE261550ED22B2EC6BF036EC14
:10C7D0006DF01406000E155A070E14C0DBFF080E8C
:10C7E00015C0DBFF070EDBCF14F0080EDBCF15F012
:10C7F0001A0E141802E1060E15180FE0070EDBCF13
:10C80000E9FF080EDBCFEAFFEF502E0806E0070E27
:10C81000DB06080EE7E2DB06E5D7070EDB2A080E8B
:10C8200001E3DB2A0601196B0B0EE76E1919E8AE5E
:10C8300002D0E73402D0E750195D1BE2B70E146E48
:10C84000CB0E156E010E166E19C617F0186A196A0E
:10C8500017AE02D0186819685AEC6AF068EC6CF0F0
:10C8600028ECA1F0A1EC6CF0000903E00601192B03
:10C87000DBD71B0EE66E060EE66ECEEC6DF0E552D3
:10C88000E5520601176FFF0E145D15E06FEC6CF0BA
:10C89000020B11E014C6E6FF18ECA8F0E552C0EC5C
:10C8A0006CF01DEC6DF0D6EC6CF040ECA5F0E552B0
:10C8B000E5520601156FDAEC6AF0200EC0EC6DF05F
:10C8C000B8EC6AF005EC6BF0EE50ED1028E00601D4
:10C8D000010E166F60EC6DF055EC6AF065EC3EF001
:10C8E000DBEC6CF0DF06010E01E2DB06C5EC6CF060
:10C8F000620E52EC6CF003E30601050E26D1C7EC84
:10C900006DF0F35006011027F450112310C6E9FF13
:10C9100011C6EAFF102B000E1123260EEF6E78ECE5
:10C920006DF08FEC6DF0A0EC6DF0020EEF6E78EC18
:10C930006DF005EC6BF0FF0EEE1812E1FF0EED1836
:10C940000FE1B6EC6CF04DEC6DF002E111EC6DF026
:10C95000C7EC6AF002E642EC6BF001E3FCD1B4D024
:10C9600092EC6AF005EC6BF0010EEE1809E1ED5067
:10C9700007E1020EA8EC6DF0A0EC6DF0030EE8D01C
:10C9800020EC6CF03A0EE66E55EC6AF0AAEC6BF017
:10C99000020E1426000E1522020E14C0DBFF030E39
:10C9A00015C0DBFF060EDB6A9EEC6BF0100E99ECF7
:10C9B0006BF04CE38AEC6BF0090F27EC6BF08CEC1E
:10C9C0006DF0D950090F146E020EDBCF16F0030E76
:10C9D000DBCF17F01606000E175A14501624E96E16
:10C9E000DA501720EA6EEF6AADEC6DF0050EDB6AE7
:10C9F000DB50146E156A030E52EC6CF022E21D0E31
:10CA0000146ECC0E156E010E166E050EDBCF17F0F0
:10CA1000186A196A5AEC6AF0D950090F27EC6BF0C2
:10CA200028ECD9F0A1EC6CF0000908E1050EDBCF91
:10CA3000E6FF47DAE55270EC6BF003D0050EDB2A17
:10CA4000D7D7060EDB5002E078EC6DF08FEC6DF07E
:10CA50006ED7800E175D02E2030E77D010C6E9FF95
:10CA600011C6EAFF2AEC6DF0F3CF10F6F4CF11F601
:10CA7000A0EC6DF0040EEF6E165102E176EC6BF057
:10CA8000060EDB6A166B67D1F5EC6DF0020801E16A
:10CA900062D1060176EC6BF055EC6AF000EC6CF0BC
:10CAA000F35006010C1915E115500D1912E116503D
:10CAB0000E190FE117500F190CE10BE1C7EC6AF0EA
:10CAC00002E642EC6BF005E23CEC6DF02FEC6BF013
:10CAD0003FD0180532E15CEC6FF0E76E040EE7CF53
:10CAE000DBFFDB5002080BE1B6EC6CF024EC6CF0E1
:10CAF000010E0C5F000E0D5B0E6B0F6B2CD1040E44
:10CB0000DB041BE1B6EC6CF024EC6CF00E6B0F6BED
:10CB100092EC6AF0A4EC6BF00C5DEE500D59EE5007
:10CB20000E59EE500F5906E255EC6AF04DEC6DF0DF
:10CB300001E011D10601060E08D0A0EC6DF0060E42
:10CB4000EF6EFF0E145D06E1040E186FEFEC6AF055
:10CB5000EF6EB4D097EC6CF0FF0E155D05E1046943
:10CB600005690669076905D0040EE66E060E5EECDF
:10CB70006BF00601EFEC6AF0EF6E020ECAEC6CF09F
:10CB8000FF0E146ECB0E156E010E166E18C617F042
:10CB9000186A196A17AE02D0186819685AEC6AF058
:10CBA00068EC6DF0080E0601185D1AE135EC6BF0CB
:10CBB00055EC6AF0BFEC3DF0DBEC6CF0800EE66EFD
:10CBC000360EE66E010EE66E68EC6DF035EC6BF03D
:10CBD000B6EC6CF0BFEC3DF0DBEC6CF0CBEC6DF048
:10CBE0000601185105E0180503E02FEC6BF0A3D007
:10CBF0000B0E195D1CE0710EE66E360EE66E010E30
:10CC0000E66E9DEC6DF0DB0E146ECB0E156E010E14
:10CC1000166E19C617F0186A196A17AE02D018688E
:10CC200019685AEC6AF068EC6DF0CBEC6DF06FECC3
:10CC30006CF0010B08E0580EE66E360EE66E010E43
:10CC4000E66E68EC6DF0480EE66E360EE66E010E8E
:10CC5000E66E68EC6DF0060118050CE0E868041952
:10CC600008E1E868051905E1E868061902E1E868E5
:10CC7000071907E03F0EE66E360EE66E010EE66E11
:10CC80000FD0360EE66E360EE66E010EE66E9DECA9
:10CC90006DF0340EE66E360EE66E010EE66E06019F
:10CCA0009DEC6DF0CBEC6DF00601165104E0ABECA1
:10CCB0006CF0080E02D00CEC6DF0EF6E060EDB6A25
:10CCC0004AD00CEC6DF0EF6E060EDB6A50D800090E
:10CCD00007E07AEC6BF02FEC6BF0EF6E70EC6BF022
:10CCE000B5EC6DF01BEC6BF036E170EC6BF033D013
:10CCF00070EC6BF0DADBADEC3CF0E552C0EC6CF0C4
:10CD0000100EF35C000EF45826E308C6E6FF09C6D1
:10CD1000E6FF0AC6E6FF0BC6E6FF48EC59F0BDEC9D
:10CD20006DF006010C510D110E110F1114E1060EDC
:10CD3000DB6A32EC6BF0EF6E0ED0FF0E145D02E09A
:10CD40007AEC6BF0FF0E155D02E082EC6BF03CECD0
:10CD50006DF02CEC6BF0060EDB5001E131D4190EB6
:10CD6000E15C02E2E16AE552E16EE4EF6AF0DFECD9
:10CD70006AF0450EE126B5EC6DF0E55220EC6BF063
:10CD80005AEC6CF01A6A1B6AA4EC6BF00601045DA5
:10CD90001C6EEE5005591D6EEE5006591E6EEE507B
:10CDA00007591F6E1C50185C1D5019581E501A58F8
:10CDB0001F501B5805E2E8EC6AF0166A176A0DD09E
:10CDC000A4EC6BF0045D146EEE500559156EEE5038
:10CDD0000659166EEE500759176E9CEC6CF0C5ECB8
:10CDE0006CF00001145006010027000115500601E7
:10CDF0000123000E0223032319EC6DF01CE22DEC3D
:10CE00006CF003E2C5EC6CF003D0400E146E156AB2
:10CE1000D6EC6CF0D950050F27EC6BF014C6E6FF8A
:10CE2000DFEC6CF002E1010E43D08AEC6BF0050FF1
:10CE3000B1EC6DF0E1D7A4EC6BF00601041937E119
:10CE4000EE50051934E1EE50061931E1EE500719A4
:10CE50002EE12DE1ABEC6CF00A0EEF6E0C6B0D6B5E
:10CE60000E6B0F6BC3EC6DF044EC6CF060EC6DF08E
:10CE700044EC6CF0000906E076EC6CF0040EDB503C
:10CE80007E08F4E176EC6CF0080EE66E060E5EECC1
:10CE90006BF0040EE66E060E5EEC6BF0000907E127
:10CEA0000601046905690669076982EC6BF0000EEA
:10CEB000146E450EE15C02E2E16AE552E16E145047
:10CEC00083D37DDBFE0EDB0402E107D805D0FE0E26
:10CED000DB50020801E183D877D371DB2C0EE12609
:10CEE000060117BF75D0060EA8EC6DF084EC6DF04E
:10CEF000030EDE26000EDD22FC0EDE16DD6A51EC8E
:10CF00006DF0240E165C000E175803E2C5EC6CF0B1
:10CF100003D0240E146E156A9CEC6CF0D950020FED
:10CF2000146EDACF15F07DEC6CF019EC6DF01DE2AB
:10CF3000040ECBDB8CEC6DF0030EC7DB040EC5DBFF
:10CF4000ACEC9FF0146E080EE15E14505EDB040E34
:10CF5000EE5E000EED5AD9502A0FE96EDACFEAFFE5
:10CF6000030EEE26000EED22E0D784EC6CF0EF6AA3
:10CF7000DE6ADD6AD950020F146E7DEC6CF0C5ECF0
:10CF80006CF0280E52EC6CF00FE284EC6CF0EF5079
:10CF90003A080AE0DF2A010E01E3DB2A2A0EDB2A27
:10CFA0002B0EEDE3DB2AEBD72A0EDBCFE9FFDB2AE2
:10CFB0002B0EDBCFEAFF01E3DB2AEF6A42EC6DF0D8
:10CFC00064EC6DF0D8EC6DF0BDEC6DF00601176F00
:10CFD0002C0EE15C02E2E16AE552E16EF5D2EFDA95
:10CFE0000C0EE12684EC6DF0C5EC6CF00A0E52ECF0
:10CFF0006CF006E30601020E186F97EC6CF022D07D
:10D00000EFEC6CF064EC6DF08CEC6DF0D1EC6CF04E
:10D01000D950020F146EDACF15F0DE501424E96EE9
:10D02000DD501520EA6EEF6A64EC6DF005ECE0F07F
:10D03000E552E55206C000F607C001F608C002F648
:10D0400009C003F60C0EE15C02E2E16AE552E16E12
:10D05000BBD2B5DA090EE126B9EC6CF05BEC6DF0F1
:10D06000040EF3CFDBFF050EF4CFDBFFFD0EDBCFAD
:10D0700008F0FE0EDBCF09F0020E08C0DBFF030E46
:10D0800009C0DBFF08C0DEFF09C0DDFFD950040F77
:10D09000E96EDACFEAFFEE50ED105DE094DB01E3DC
:10D0A000DB2A060EEFCFDBFF040EDB06050E01E2E6
:10D0B000DB06060EDB503D0804E0060EDB502608BA
:10D0C00005E190DA01E3DB2AEF6AE0D7060EDB50D8
:10D0D0002B0805E187DA01E3DB2A200E33D0060EA8
:10D0E000DB50250831E1040EDBCF14F0050EDBCF59
:10D0F00015F0020ED7DB05E2040EDB6A050EDB6AD3
:10D10000C5D761DB01E3DB2A080EEFCFDBFF5BDB7A
:10D1100001E3DB2A070EEFCFDBFF040EDB06050E73
:10D1200001E2DB06040EDB06050E01E2DB06D0DBC6
:10D13000DDECA0F0E552E552E66E54DA01E3DB2ABD
:10D14000E552E750EF6EA2D74DDA01E3DB2A060E77
:10D15000DBCFEFFF9BD746DA01E3DB2AEF6AFEEC79
:10D160006CF0EF6A35DA14C0F3FF15C0F4FF090E56
:10D17000E15C02E2E16AE552E16E26D220DA7ADA77
:10D1800018E0F7DB05EC6DF008ECD9F0BDEC6DF0C4
:10D1900000090CE1FADA05EC6DF078ECD9F037DB38
:10D1A000F324146E1750F4203ADB05D0ACD9ABD978
:10D1B000E6D7F36AF46A08D202DA5CDA22E06CDAC3
:10D1C00017DB09C016F0142A000E15221622EEDB1A
:10D1D00063DACFDB65ECD8F0176E070EE15E17500F
:10D1E00000090CE1D2DA58DA86ECD9F0E5520FDB0F
:10D1F0000724146E1750082012DB05D084D983D978
:10D20000DCD7F36AF46AE0D1DAD9E65211DA3D0EDE
:10D21000E66E88DAD950FD0F5CDA03E02BDA01E024
:10D22000BFDADF50E552D0D1CAD9E65201DA260E74
:10D23000E66E78DA020EDF5C13E198DBE1DA0601D4
:10D240000051F3180DE1015115180AE102511618A9
:10D2500007E10351171804E103E1EAD9E66A62DA4B
:10D26000D950FD0F36DA03E005DA01E099DADF5034
:10D27000E552AAD1A4D9030EE126FE0EDB5007E049
:10D2800099D9FE0EDBCFE6FF71DBB1DB04D06EDB9C
:10D2900042EC3EF0E552DE5284DBDD52D950010F04
:10D2A000E96EDACFEAFFFF0EEE1805E1FF0EED188A
:10D2B00002E1020E80D0EEDAF5DA07E2D950FC0F77
:10D2C00008DA03E07DEC6DF052D0D950FC0F01DAA2
:10D2D00003E17DEC6DF054D01EDBFA0EDBCF16F0CF
:10D2E000FB0EDBCF17F0020E165E000E175A14501D
:10D2F000165C155017583EE2FA0EDBCF18F0FB0E05
:10D30000DBCF19F0020E185E000E195A18C0E6FFA6
:10D3100019C0E6FF95EC6DF09EEC3EF012DB30DBC1
:10D320002AD9FA0EDBCF1AF0FB0EDBCF1BF0020E70
:10D330001A5E000E1B5A010EDBCF08F0020EDBCF87
:10D3400009F01A50085C186E1B500958196E18C065
:10D35000E6FFE66E49DB9EEC3EF01C6E050EE15EDC
:10D360001C5009D997DA145E000E155A5FDA010EC7
:10D37000DF6E07D02FDAD9DB34DAFDD8CCDA56DA13
:10D38000DF6AFE0EDB5016E02FDB65EC3EF013DBB0
:10D39000146E156A166A176A14AE03D015681668FB
:10D3A000176814500601005F1550015B1650025BB0
:10D3B0001750035BDF50146E030EE15C02E2E16A7A
:10D3C000E552E16E145000D1FAD8450EE12606016F
:10D3D0000C510D110E110F1117E1FC0EDBCFE6FF02
:10D3E000FD0EDBCFE6FFFE0EDBCFE6FFB2ECA4F0D6
:10D3F000E55239DA53E05ADA18ECA8F0E552F3CFE7
:10D400000CF6F4CF0DF61FD00CC6E6FF0DC6E6FFF6
:10D4100040ECA5F028DA42E0020EE66E0EC614F0EB
:10D420000FC615F0166A176A0EC6E6FF0FC6E6FFAE
:10D4300016C0E6FF17C0E6FF39DA49ECA6F0186E11
:10D44000060EE15E185091DBE552ABDAF2DA1AE231
:10D4500004DA02E29ADA03D0400E146E156AA6DAF4
:10D460002FDB24DAACDA0AE121DA7EECA5F0E55212
:10D4700006010C6B0D6B0E6B0F6B10D04BD9040FAC
:10D4800070DBE4D713DAFFECA7F0E55206C00EF626
:10D4900007C00FF60BDA7EECA5F0E552450EE15C15
:10D4A00002E2E16AE552E16E8FD055DAEE52EF50BA
:10D4B000E66E1200030E0C6E0D6A0E6A17C007F0BE
:10D4C00018C008F019C009F020ECE1F004C017F012
:10D4D00005C018F006C019F014500424F36E15505E
:10D4E0000520F46E16500620F86EF4CFF7FFF3CF48
:10D4F000F6FF0900F5CFE6FF0900F5CFE6FF0800CB
:10D50000F5CFE6FF120035DAD6DA3ADA96DAD950F4
:10D51000FD0FE96EFF0EDA20EA6E1450EE2615506C
:10D52000ED221200C7ECE3F006C008F607C009F6CA
:10D5300008C00AF609C00BF6BF0E060108272F0E19
:10D540000923200E0A23000E0B231200EAEC3DF003
:10D55000BDEF6DF08151BFDA02EC8BF0F4DA2FEC05
:10D560008DF00BDB3CDA02EC8BF0E552E552120059
:10D570003EDAD1EF6CF0166A176AF3500601005FCD
:10D58000F450015B1650025B1750035B1200C7ECAE
:10D59000E3F006010851065C146E09510758156E38
:10D5A0000A510858166E0B510958176EE834000ED0
:10D5B00017181200E66AE7DAE66EE66A1200D9CFBB
:10D5C000E6FFE1CFD9FF1200E552E7CFD9FF120005
:10D5D000020EDBCF14F0030EDBCF15F01200BBD927
:10D5E000070E1200020EDBCFE9FFDB2A030EDBCFB2
:10D5F000EAFF12009EEC3EF0B8EF6DF0B40EE66E5E
:10D60000CB0EE66E010EE66E1200D9CFE9FFDACF3F
:10D61000EAFF1200EA6ADF34FE0BEA36E96E7F0E9B
:10D62000E926060EEA221200B0D907DAD6EF6CF02E
:10D63000ECD9B9EF6CF0E552A3D9F350F410120015
:10D64000020EF3CFDBFF030EF4CFDBFF1200E66E1A
:10D65000000EDA20E66E12007ED9EF6A12007BD946
:10D660000B0E120078D9090E12001A0EE66E060E85
:10D67000E66E1200FD0EDBCFE9FFFE0EDBCFEAFF08
:10D68000EF501200D880000E1454000E1554000EF6
:10D690001654000E17541200FA0EDBCFE6FFFB0EF5
:10D6A000DBCFE6FFFC0EDBCFE6FF1200A7D9E906D1
:10D6B000000EEA5AFBD9EF502F081200E66E15C68D
:10D6C000E6FF2FECA6F0DBEF6CF0E66EE66A42EFC9
:10D6D0006DF0E96EFF0EDA20EA6EEE50ED101200EA
:10D6E000010EF36E060EF3CFDBFF120034D9050EE8
:10D6F000EF6E120014C6E6FF7EECA5F0E5520601BF
:10D700001469120015C6E6FF7EECA5F0E55206018D
:10D7100015691200020EDBCFE6FF030EDBCFE6FF3A
:10D72000D9501200A7DD24DADF6E12002CDA010EC8
:10D730001200D880EE54000EED541200D950020FA2
:10D74000E96EDACFEAFF1200000EE96E060EEA6E0D
:10D75000EE50120032EC42F0166E070EE15E1650EB
:10D76000C0EF6CF01B0EE66E060EE66E16ECA4F033
:10D77000E552E5520601146F12000DEC41F0146EF3
:10D780000B0EE15E1450D1EF6CF0FD0EDBCF16F006
:10D79000FE0EDBCF17F016C0E6FF17C0E6FF120043
:10D7A000E8D857DCE552E552120014EC4FF0146E45
:10D7B000060EE15E145012009EEC3EF0166E050E51
:10D7C000E15E16501200DFCFE9FFDF2A010EDBCF4A
:10D7D000EAFF1200010EDBCFE6FF020EDBCFE6FF11
:10D7E00012009EEC3EF0186E050EE15E185012001D
:10D7F00086ECD9F0E0D807C014F008C015F012008C
:10D8000042EC3EF0E552BCD8166A176A1200D3D833
:10D81000E7CF17F0E552E7CF16F016501200156E5D
:10D820000CD914C0F3FF15C0F4FF1200FC0EDB503E
:10D830001424E96EFD0EDB501520EA6EEF6A12002B
:10D84000E66ACDD8C3EF6DF042EC3EF0E552F3CF7F
:10D850000CF6F4CF0DF60601120023D9400E165C2B
:10D86000000E17581200E552E552E76E440EE7CF5E
:10D87000DBFFDB50FF08120065ECD8F0146E070EDA
:10D88000E15E14500009120014C6E6FF8CECA5F00E
:10D89000DBEF6CF0FA0EDBCF14F0FB0EDBCF15F0F4
:10D8A000020E1200145C000E15581200440EDBCF5D
:10D8B000E6FF1200020EDBCF18F0030EDBCF19F0EB
:10D8C0001200930EE66E360EE66E010EE66E120044
:10D8D000070EDBCFE6FF080EDBCFE6FF120014C613
:10D8E000E6FF3EECA7F0E552F35012000601002BD4
:10D8F000000E01230223032312002A0E14C0DBFFB3
:10D900002B0EDACFDBFF12002A0EDBCFE9FF2B0E46
:10D91000DBCFEAFF1200010EDBCF14F0020EDBCFEB
:10D9200015F01200010EE66EE66A000E1200006BA2
:10D93000016B026B036B120014C0DEFF15C0DDFF2C
:10D9400012001A6E050EE15E1A5012001450EE5EBF
:10D950001550ED5A12008151E96EEA6AD890E93605
:10D96000EA367F0EE926060EEA221200060155EF7E
:10D970006AF0FD0EDBCFE6FFFE0EDBCFE6FF120006
:10D98000F3CF14F0F4CF15F01200DECF14F0DDCF9A
:10D9900015F01200E66ECADEE66EE66A86DDD5EFA9
:10D9A0006BF0F3CFDEFFF4CFDDFF120014C0E6FF13
:10D9B00015C0E6FF1200E552E552E5521200D6EC22
:10D9C000A5F0186E050EE15E18503ADEB7DEEE5097
:10D9D000ED1012002AEC3DF0CBD8ADEF6DF0DECFAC
:10D9E000E6FFDDCFE6FF1200CED855EF6AF032EC4D
:10D9F00042F0146E070EE15E14501200020EDBCFEF
:10DA0000E9FF030EDBCFEAFF1200FB0EDBCFE6FFE0
:10DA1000FC0EDBCFE6FF1200F1DD8FD8060132EFFE
:10DA20006BF00601050E186FDADDEF6E060EDB6A8D
:10DA30001200EBDD000E99EF6BF0010E1426000EC4
:10DA4000152212007F0EE66EE66A000EE66E060EE6
:10DA5000E66E1200EF6A09DE29EC68F0E552E55245
:10DA60001200200EE66E21DDB8EF6AF0B1DD1A0E6D
:10DA70001426060E1522120018DD3BEC3CF0E55290
:10DA8000060112002A0EDBCFE6FF2B0EDBCFE6FFEE
:10DA90001200C0DDEE52EF50120026EC3FF01BEFFB
:10DAA0006BF0DECF16F0DDCF17F012001A0EE9266C
:10DAB000060EEA22120078ECD9F0E552E552120087
:10DAC000D950040F27EF6BF0D950020F27EF6BF0FE
:10DAD0004DDFA6EF6AF07F0D53DF166A176A7D0EE1
:10DAE00014261F0E1522000E16221722D6EF6CF0F8
:10DAF00061DD0A0E45D8B8EF6AF06CDE44D836DF37
:10DB000070DE3EDFBBEF6AF055DD020EE66EE66AC0
:10DB100075DD2CDFBDEF6BF029DFFAEF6AF084DDF5
:10DB2000E66EE66A23DFDCEF6BF0FC0EDBCFE6FF90
:10DB3000FD0EDBCFE6FFB6EF6CF0B7DCA6EF6AF0C8
:10DB40000601ABEF6CF0E552E5522BDF22EF6DF0F2
:10DB5000E66EE66A49DFFAEF6AF03ADD56DDA6EFD7
:10DB60006CF075DD03DFEAEF6CF000DFADEF3CF049
:10DB7000146E050EE15E14501200E552DBEF6CF0FE
:10DB8000E66EB6EF6CF0000EE66EE66A120027DF76
:0CDB90006CDD8CEF6DF032DD68EF6DF0A5
:04DB9C00D9CFE6FFF8
:10DBA000000181A902D0000E01D0800E91EF7BF020
:10DBB0009AEC7BF09B0EE66E330EE66E010EE66E7F
:10DBC000A6EC7CF0E5EC7CF00DE189EC7DF0FB0E41
:10DBD000DBCFE6FFFC0EDBCFE6FFAEEC7DF002E133
:10DBE000800E01D0000E91EF7BF09AEC7BF0160EC8
:10DBF000E126140EE66EE66A56EC7DF06CEC7CF0E5
:10DC0000000905E0D950020F146EDACF15F00A0EA4
:10DC1000E66EE66A7C0EE66E330EE66E010EE66E8A
:10DC200056EC7DF09EEC7CF001E022D1790EE66EA0
:10DC3000330EE66E010E29EC7BF00AE09FEC7BF0E0
:10DC400002E0000E01D0010EE8B08D80E8A08D90BA
:10DC5000760EE66E330EE66E010E29EC7BF00AE0DE
:10DC60009FEC7BF002E0000E01D0010EE8B08D8247
:10DC7000E8A08D92730EE66E330EE66E010E29EC6F
:10DC80007BF00AE09FEC7BF002E0000E01D0010E79
:10DC9000E8B08D84E8A08D94700EE66E330EE66ECB
:10DCA000010E29EC7BF00AE09FEC7BF002E0000E15
:10DCB00001D0010EE8B08D86E8A08D966D0EE66E5F
:10DCC000330EE66E010E29EC7BF00AE09FEC7BF050
:10DCD00002E0000E01D0010EE8B08D88E8A08D981A
:10DCE0006A0EE66E330EE66E010E29EC7BF00AE05A
:10DCF0009FEC7BF002E0000E01D0010EE8B08D8AAF
:10DD0000E8A08D9A670EE66E330EE66E010E29ECE2
:10DD10007BF00AE09FEC7BF002E0000E01D0010EE8
:10DD2000E8B08D8CE8A08D9C640EE66E330EE66E36
:10DD3000010E29EC7BF00AE09FEC7BF002E0000E84
:10DD400001D0010EE8B08D8EE8A08D9E610EE66ECA
:10DD5000330EE66E010E29EC7BF00AE09FEC7BF0BF
:10DD600002E0000E01D0010EE8B09180E8A0919091
:10DD70005E0EE66E330EE66E010E29EC7BF00AE0D5
:10DD80009FEC7BF002E0000E01D0010EE8B0918222
:10DD9000E8A091925A0EE66E330EE66E010E29EC63
:10DDA0007BF00AE09FEC7BF002E0000E01D0010E58
:10DDB000E8B09184E8A09194560EE66E330EE66EBC
:10DDC000010E29EC7BF00AE09FEC7BF002E0000EF4
:10DDD00001D0010EE8B09186E8A09196520EE66E51
:10DDE000330EE66E010E29EC7BF00AE09FEC7BF02F
:10DDF00002E0000E01D0010EE8B09188E8A09198F1
:10DE00004E0EE66E330EE66E010E29EC7BF00AE054
:10DE10009FEC7BF002E0000E01D0010EE8B0918A89
:10DE2000E8A0919A4A0EE66E330EE66E010E29ECDA
:10DE30007BF00AE09FEC7BF002E0000E01D0010EC7
:10DE4000E8B0918CE8A0919C460EE66E330EE66E2B
:10DE5000010E29EC7BF021E09FEC7BF002E0000E4C
:10DE600001D0010EE8B0918EE8B017D0919E15D088
:10DE70000A0EE66EE66AADEC7CF056EC7DF09EECA8
:10DE80007CF00FE1270EE66E330EE66E010E29ECF4
:10DE90007BF003E058EC7BF002D0EEEC7BF0080E58
:10DEA000186F000E146E160EE15C02E2E16AE55294
:10DEB000E16E145091EF7BF09AEC7BF0140EE126AA
:10DEC000D8EC7DF06CEC7CF0ADEC7CF095EC7BF06C
:10DED000E5EC7CF003E18EEC74F043D0120EE66EBC
:10DEE000330EE66E010EA7EC7DF003E1F5EC77F062
:10DEF00038D0060EE66E330EE66E010EA7EC7DF00E
:10DF000003E1CAEC76F02DD0FA0EE66E320EE66E24
:10DF1000010EA7EC7DF003E13EEC77F022D0F10E8C
:10DF2000E66E320EE66E010EA7EC7DF003E1A2EC88
:10DF300078F017D0E90EE66E320EE66E010EA7EC11
:10DF40007DF003E1C0EC79F00CD0E10EE66E320E0C
:10DF5000E66E010EA7EC7DF003E1CCEC7AF001D087
:10DF6000000E146E140EE15C02E2E16AE552E16E0D
:10DF7000145091EF7BF00601010E0C6F91EC7DF0D7
:10DF80006BEC7DF0166A0AEC7CF016C0E6FFB4EC90
:10DF90007CF086ECD9F053EC7BF0E7CF16F0E5523D
:10DFA000E7CF15F0E552E7CF14F00750145C0850A6
:10DFB00015580950165801E21200A6EC7BF0B4EC9B
:10DFC0007CF0E0EF7CF0C60EE66E320EE66E010EDF
:10DFD000E8EF7DF06EEC7DF00F0EF4EC7CF002E2E9
:10DFE000E16AE552E16E91EF7BF06EEC7DF0200E80
:10DFF000F4EC7CF002E2E16AE552E16E91EF7BF035
:10E0000025EC7DF0146A90EC7CF00DE3FE0EDB5005
:10E01000070809E363EC7CF003E09AEC7CF0FDE197
:10E02000F350961415D0080E146E90EC7CF012E3A9
:10E03000FE0EDB500F080EE3FE0EDB50F80F146EE1
:10E04000010E145204E0E846FE0B1406FCE19A149B
:10E05000DF6E01D0DF68DF50E55291EF7BF025ECF9
:10E060007DF0146A90EC7CF01EE3FE0EDB50070896
:10E070001AE3FD0EDB500AE063EC7CF003E09AEC5F
:10E080007CF0FDE1F350000188130AD063EC7CF0D2
:10E0900003E09AEC7CF0FDE1F350F31C00018817DB
:10E0A00088C096FF2CD0080E146E90EC7CF027E30D
:10E0B000FE0EDB500F0823E3080E146EFE0EDBCFBE
:10E0C000E7FF1450E75EFE0EE7CFDBFFFD0EDB50EF
:10E0D0000AE063EC7CF003E09AEC7CF0FDE1F350A5
:10E0E000000189130AD063EC7CF003E09AEC7CF029
:10E0F000FDE1F350F31C0001891789C09AFFE55236
:10E1000091EF7BF09AEC7BF0060EE126280EE66E8E
:10E11000E66A010EE66EE66ABD0EE66E320EE66E49
:10E12000010E5EEC7DF0F3ECE4F0146E090EE15E9E
:10E130001450EBEC7DF0060EE15C02E2E16AE55280
:10E14000E16E91EF7BF09AEC7BF0070EE1260A0E70
:10E15000E66EFD0EDBCFE6FF1AECC1F0E552E552AC
:10E16000F3CFDEFFF4CFDDFF6BEC7DF0040E95EC1A
:10E170007DF004E20601010E0C6F14D0DECFE6FF45
:10E18000DDCFE6FFB90EE66E320EE66E010EE66EEC
:10E1900056EC7DF0D7EC7BF056EC7DF0E2EC7DF0B8
:10E1A00006010C6B91EC7DF0070EE15C02E2E16A86
:10E1B000E552E16E91EF7BF0000181AD02D099EC68
:10E1C0007DF0A6EF7BF025EC7DF0DF6AFEEC7BF0C6
:10E1D000EE50ED100BE1000194BD04D0AAEC7BF0F1
:10E1E00011E00ED0AAEC7BF00DE10AD0000194BF43
:10E1F00004D0AAEC7BF006E003D0AAEC7BF002E1AD
:10E20000010EDF6EDF5002E099EC7DF08EEF7DF0C5
:10E2100025EC7DF0F8EC7BF010E340EC7CF00DE2B7
:10E2200032EC7CF0DF5004E0AAEC7BF006E003D097
:10E23000AAEC7BF002E199EC7DF08EEF7DF000011D
:10E2400081A902D099EC7DF0A6EF7BF00501D451B5
:10E2500012E0020A08E0030A0EE1A20EE66E320E98
:10E26000E66E010E05D0940EE66E320EE66E010EDD
:10E27000E66EE0EC7CF0A6EF7BF09AEC7BF04BECEA
:10E280007CF0E0EC7CF0A6EC7BF091EF7BF0820E72
:10E29000E66E060EE66EE2EC7DF0A6EF7BF06EEC2D
:10E2A0007DF0380EF4EC7CF002E2E16AE552E16EBA
:10E2B00091EF7BF09AEC7BF01A0EE126F8EC7BF004
:10E2C00001E29FD040EC7CF001E39BD044EC7DF078
:10E2D000050ED89014361536E806FBE1C2EC7CF04A
:10E2E000120E14C0DBFF130E15C0DBFF0501D35166
:10E2F00060E0140EDB6A150EDB6ABBEC7CF0180ED6
:10E30000145C000E155850E2160EDB6A170EDB6A1D
:10E31000160EDBCF14F0170EDBCF15F00A0E145CCF
:10E32000000E155808E2C7ECE3F0160EDB2A170EB4
:10E33000EFE3DB2AEDD77CEC7DF0B2EC7BF07CECFC
:10E340007DF095EC7BF052EC7CF0010EE66E4BEC30
:10E350007DF0BBEC7CF0050ED89014361536E8063F
:10E36000FBE1C2EC7CF0C5EC7DF00A0EF36E180EFA
:10E37000F3CFDBFF190EDB6A180EDBCF14F0DB06E0
:10E38000190EDBCF15F001E2DB061450151006E084
:10E390000C0EE66E9AECE6F0E552EED7140EDB2A90
:10E3A000150EABE3DB2AA9D70501D36B0BEC7DF08F
:10E3B00026D0120ED8EC7DF0DBCF14F0130EDBCF9D
:10E3C00015F0CFEC7BF05FECDCF0186E080EE15E30
:10E3D0001850E66A4BEC7DF0000903E00E0EDB6A94
:10E3E0000ED00BEC7DF0010EE66E4BEC7DF0120EC4
:10E3F000DBCF14F0130EDBCF15F0C5EC7DF09FECF6
:10E400007DF0A6EC7BF01A0EE15C02E2E16AE552D7
:10E41000E16E91EF7BF0BFEC7DF00FE0DF5006E0A6
:10E420008C0E146E320E156E010E05D0880E146E11
:10E43000320E156E010EC9EC7DF08EEF7DF025ECED
:10E440007DF059EC7CF0070E081801E1095032E02C
:10E45000060E081801E109502BE0050E081801E12D
:10E46000095023E0040E081801E109501CE0030ED6
:10E47000081801E1095015E0020E081801E10950E1
:10E480000DE0010E081801E1095006E0085026E1F0
:10E49000095024E1010E03D0020E01D0080E92149F
:10E4A0000BD0040E03D0200E01D0400E971404D0E0
:10E4B000100E01D0200E9914DF6EDF5006E08C0E96
:10E4C000146E320E156E010E05D0880E146E320ECB
:10E4D000156E010EC9EC7DF0A6EC7BF0E55291EFD4
:10E4E0007BF0BFEC7DF00AE0DF5008E07F0EE66EC7
:10E4F000320EE66E010EE66EE0EC7CF0E55291EF36
:10E500007BF025EC7DF0F8EC7BF011E3FEEC7BF08A
:10E51000070EC7EC7CF00BE3010EF36EFD0EDB5033
:10E5200003E09AEC7CF0FDE1F35084141DD044EC40
:10E530007DF0080E145C000E15583FE3FEEC7BF0F6
:10E540000F0EC7EC7CF039E3FEEC7BF0080EEE5EBC
:10E55000000EED5A010EF36EFD0EDB5003E09AEC57
:10E560007CF0FDE1F3508814DF6EAAEC7BF00FE045
:10E57000DF5006E07D0E146E320E156E010E05D0D2
:10E580007B0E146E320E156E010E166E0ED0DF501D
:10E5900006E07B0E146E320E156E010E05D07D0E58
:10E5A000146E320E156E010E166E2FEC7DF016C035
:10E5B000E6FFE0EC7CF0A6EC7BF0E55291EF7BF01F
:10E5C0009AEC7BF0110EE126FEEC7BF0EE50ED10A4
:10E5D00006E168EC7CF0CD0EE66E060E05D068EC28
:10E5E0007CF0DD0EE66E060E5EEC7DF084ECD8F07D
:10E5F000146E060EE15E1450100EDB6AEBEC7DF03B
:10E60000110EE15C02E2E16AE552E16E91EF7BF00E
:10E610006EEC7DF0040EDB6AF36EDBCFF4FFE850A6
:10E62000F45C22E2040EDB5003E02E0E3DEC7DF0A4
:10E6300095EC7BF0D950FB0F146EFF0EDA20156EAF
:10E64000040EDB500F011424E96E000E1520EA6E53
:10E65000EF50E66EE66A62ECA0F053EC7BF09FECC4
:10E660007DF0040EDB2AD8D7050EE15C02E2E16AF8
:10E67000E552E16E91EF7BF025EC7DF0DF6A59EC1D
:10E680007CF0030E081801E109501AE0020E081888
:10E6900001E1095011E0010E081801E1095008E0FC
:10E6A000085013E1095011E1000181A10ED00BD0F7
:10E6B000000181A30AD007D0000181A506D003D0B4
:10E6C000000181A702D0010EDF6EDF5003E099EC5C
:10E6D0007DF002D0A6EC7BF0E55291EF7BF00001DB
:10E6E00081AD02D099EC7DF01200000181AD09D01E
:10E6F00061C0E6FF62C0E6FF63C0E6FF64C0E6FFFC
:10E7000008D075C0E6FF76C0E6FF77C0E6FF78C0A8
:10E71000E6FF1EEF7DF07DC0E6FF7EC0E6FF7FC016
:10E72000E6FF80C0E6FF1EEF7DF079C0E6FF7AC00D
:10E73000E6FF7BC0E6FF7CC0E6FF1EEF7DF06DC00C
:10E74000E6FF6EC0E6FF6FC0E6FF70C0E6FF1EEF9B
:10E750007DF071C0E6FF72C0E6FF73C0E6FF74C0D3
:10E76000E6FF1EEF7DF025EC7DF06BEC7DF0120EE8
:10E7700095EC7DF004E20601010E0C6F1BD0DF6A00
:10E78000060EDF5C15E2DF5003E03A0E3DEC7DF053
:10E7900071EC7CF002ECA1F0E5523DEC7DF071EC07
:10E7A0007CF016ECA1F0E5523DEC7DF0DF2AE8D7D5
:10E7B00006010C6B91EC7DF0E55291EF7BF09AEC49
:10E7C0007BF0080EE12659EC7CF0040E081801E1FC
:10E7D00009502BE0030E081801E1095020E0020E59
:10E7E000081801E1095015E0010E081801E109506F
:10E7F0000AE008503FE109503DE116EC7CF08A0E3A
:10E80000EE6E000E17D016EC7CF08C0EEE6E000E45
:10E8100011D016EC7CF08E0EEE6E000E0BD016ECC6
:10E820007CF0900EEE6E000E05D016EC7CF0920E91
:10E83000EE6E000EED6E6BEC7DF0050E95EC7DF04E
:10E8400004E20601010E0C6F17D0060EDBCFE9FFC4
:10E85000070EDBCFEAFFEECFE6FFEFCFE6FF780E45
:10E86000E66E320EE66E010E5EEC7DF0D7EC7BF0CC
:10E870009FEC7DF006010C6B91EC7DF0080EE15CE5
:10E8800002E2E16AE552E16E91EF7BF0FF001200D7
:10E89000B1EC7DF0E2EF7DF09AEC7BF0040EE12626
:10E8A000A6EC7CF005ECE0F0E552E55206C0DEFF98
:10E8B00007C0DEFF08C0DEFF09C0DDFFDD52DD520C
:10E8C0001CEC7CF009E6D880000E0754000E0854BA
:10E8D000000E0954000E0A5419E21CEC7CF009E603
:10E8E000D880FF0E0754FF0E0854000E0954000E86
:10E8F0000A540CE3FB0EDBCFE9FFFC0EDBCFEAFF93
:10E90000000EDFCFEEFF010EDBCFEDFF040EE15C6A
:10E9100002E2E16AE552E16E91EF7BF09AEC7BF066
:10E920003E0EE126010EF36E390EF3CFDBFFAAECAB
:10E930007DF001E223D222EC7DF002E2010E20D232
:10E94000360ED8EC7DF0E66AE66AE66AE66A5FECC7
:10E95000DCF0146E080EE15E145072EC7DF061C0C4
:10E96000EEFF62C0EEFF63C0EEFF64C0EEFF65C065
:10E97000EEFF66C0EEFF67C0EEFF68C0EEFF69C045
:10E98000EEFF6AC0EEFF6BC0EEFF6CC0EEFF6DC025
:10E99000EEFF6EC0EEFF6FC0EEFF70C0EEFF71C005
:10E9A000EEFF72C0EEFF73C0EEFF74C0EEFF75C0E5
:10E9B000EEFF76C0EEFF77C0EEFF78C0EEFF79C0C5
:10E9C000EEFF7AC0EEFF7BC0EEFF7CC0EEFF7DC0A5
:10E9D000EEFF7EC0EEFF7FC0EEFF80C0EEFF81C085
:10E9E000EEFF82C0EEFF83C0EEFF84C0EEFF85C065
:10E9F000EEFF86C0EEFF87C0EEFF88C0EEFF89C045
:10EA0000EEFF8AC0EEFF8BC0EEFF8CC0EEFF8DC024
:10EA1000EEFF8EC0EEFF8FC0EEFF90C0EEFF91C004
:10EA2000EEFF92C0EEFF93C0EEFF94C0EEFF95C0E4
:10EA3000EEFF96C0EEFF200EDB9CDB90DB92DB94BA
:10EA4000DB96E8EC7BF001E1E3D0D9EC7CF001E06F
:10EA500095D1EFEC7CF001E091D1750EE66E320EAF
:10EA6000E66E010E35EC7BF006E1D950140FEAECAE
:10EA70007CF0E7E183D1720EE66E320EE66E010E97
:10EA800035EC7BF006E1D9501C0FEAEC7CF0D9E1C3
:10EA900075D16E0EE66E320EE66E010E35EC7BF031
:10EAA00006E1D950180FEAEC7CF0CBE167D1690E92
:10EAB000E66E320EE66E010E35EC7BF006E1D950C3
:10EAC0000C0FEAEC7CF0BDE159D1640EE66E320E1B
:10EAD000E66E010E35EC7BF006E1D950100FEAEC42
:10EAE0007CF0AFE14BD1610EE66E320EE66E010EA8
:10EAF00035EC7BF003E1D950290F2BD05E0EE66E8A
:10EB0000320EE66E010E35EC7BF003E1D9502B0F8F
:10EB100020D05B0EE66E320EE66E010E35EC7BF019
:10EB200003E1D9502D0F15D0580EE66E320EE66E69
:10EB3000010E35EC7BF003E1D9502F0F0AD0550EB2
:10EB4000E66E320EE66E010E35EC7BF00AE1D9502E
:10EB5000310F8CEC7BF0A2EC7DF09EDE53EC7BF071
:10EB600070D7500EE66E320EE66E010E35EC7BF07D
:10EB700007E1FCEC7CF001E064D7200EDB8C61D770
:10EB8000480EE66E320EE66E010E35EC7BF007E1C4
:10EB9000FCEC7CF001E055D7200EDB8052D7430E11
:10EBA000E66E320EE66E010E35EC7BF007E1FCEC12
:10EBB0007CF001E046D7200EDB8243D73E0EE66EA6
:10EBC000320EE66E010E35EC7BF007E1FCEC7CF0DA
:10EBD00001E037D7200EDB8434D7390EE66E320ED3
:10EBE000E66E010E35EC7BF007E1FCEC7CF001E019
:10EBF00028D7200EDB8625D7340EE66E320EE66E61
:10EC0000010E35EC7BF001E01CD7390EDB6A19D719
:10EC1000D950200FE96EDACFEAFFEF50400B30E118
:10EC200072EC7DF0140EDBCFEEFF150EDBCFEEFFA6
:10EC3000160EDBCFEEFF170EDBCFEEFFD950180F0D
:10EC4000E96EDACFEAFF040EEECFDBFF050EEECF62
:10EC5000DBFF060EEECFDBFF070EEECFDBFFD9505A
:10EC60001C0FE96EDACFEAFF080EEECFDBFF090ECC
:10EC7000EECFDBFF0A0EEECFDBFF0B0EEECFDBFF9E
:10EC8000390EDB5009E0610EE66E000EE66EACEC6C
:10EC900083F0E552E5526ED072EC7DF0EECF61F07C
:10ECA000EECF62F0EECF63F0EECF64F0EECF65F022
:10ECB000EECF66F0EECF67F0EECF68F0EECF69F002
:10ECC000EECF6AF0EECF6BF0EECF6CF0EECF6DF0E2
:10ECD000EECF6EF0EECF6FF0EECF70F0EECF71F0C2
:10ECE000EECF72F0EECF73F0EECF74F0EECF75F0A2
:10ECF000EECF76F0EECF77F0EECF78F0EECF79F082
:10ED0000EECF7AF0EECF7BF0EECF7CF0EECF7DF061
:10ED1000EECF7EF0EECF7FF0EECF80F0EECF81F041
:10ED2000EECF82F0EECF83F0EECF84F0EECF85F021
:10ED3000EECF86F0EECF87F0EECF88F0EECF89F001
:10ED4000EECF8AF0EECF8BF0EECF8CF0EECF8DF0E1
:10ED5000EECF8EF0EECF8FF0EECF90F0EECF91F0C1
:10ED6000EECF92F0EECF93F0EECF94F0EECF95F0A1
:10ED7000EFCF96F038EC85F00501D26B11EC7DF009
:10ED8000146E3E0EE15C02E2E16AE552E16E14505F
:10ED900091EF7BF09AEC7BF0090EE126DE52010E3A
:10EDA000DD6E020EDB6AAAEC7DF05CE322EC7DF006
:10EDB00002E2010E59D0310EE66E320EE66E010E01
:10EDC000E66ED950030F8CEC7BF007EC7DF0E8EC9D
:10EDD0007BF03AE0D9EC7CF045E1EFEC7CF042E1ED
:10EDE000DF6A100EDF5C25E2DFCFE6FFDEEC7BF0B2
:10EDF000D950050F8CEC7BF0D7EC7BF0D950030F8A
:10EE000039EC7DF014E128EC7DF003E1010EE66EB3
:10EE100001D0E66ADFCFE6FF2FEC70F0E552E55255
:10EE20000F0EDF5C02E138EC85F08AEC7CF0DF2A23
:10EE3000D8D7290EE66E320EE66E010E35EC7BF069
:10EE4000C6E1010EDB6AC3D7010EDB5009E0000109
:10EE5000886B896B88C096FF89C09AFF38EC85F073
:10EE60000501D26B11EC7DF0146E090EE15C02E23B
:10EE7000E16AE552E16E145091EF7BF09AEC7BF081
:10EE80001E0EE1268AEC7CF0030EDB6AAAEC7DF014
:10EE900001E2A0D022EC7DF002E2010E9DD0260E10
:10EEA000E66E320EE66E010EE66ED950160F8CEC51
:10EEB0007BF007EC7DF0E8EC7BF001E183D0D9EC4E
:10EEC0007CF001E087D0EFEC7CF001E083D0DF6ADA
:10EED000180EDF5C6AE2DFCFE6FFDEEC7BF0D95094
:10EEE000180F8CEC7BF0D7EC7BF0D950160F39EC77
:10EEF0007DF059E1C3EC7BF0F3CF16F0F4CF17F0BF
:10EF00000F0E95EC7DF003E2DCEC7DF003D00F0EEC
:10EF1000146E156A010E14C0DBFFDBCFE6FFE66A54
:10EF2000A2EC7DF003EC7DF00FEC7CF0D950040FE7
:10EF3000146EDACF15F0010EDB500F011424E96EC8
:10EF4000000EDA20EA6EEF6A010EE66E68EC7CF0E5
:10EF500003EC7DF0E6EC7BF0DF50200D34EC7DF02F
:10EF6000C2EC7CF016EC7DF003EC7DF05AEC7DF009
:10EF70000A0EF36E1C0EF3CFDBFF1D0EDB6A1C0EB8
:10EF8000DBCF14F0DB061D0EDBCF15F001E2DB0654
:10EF90001450151006E00C0EE66E9AECE6F0E55201
:10EFA000EED73AEC7CF0DF2A93D7210EE66E320ED4
:10EFB000E66E010E5ADB01E07ED7020EDB6A3AEC08
:10EFC0007CF079D7020EDB5003E00501010ED36F10
:10EFD0000501D26B11EC7DF0146E1E0EE15C02E2B5
:10EFE000E16AE552E16E14509CD325EC7DF0010EF0
:10EFF000DF6E0501CCEC7CF067E322EC7DF002E2F1
:10F00000010E66D0E5DB50E0D9EC7CF05DE1EFEC81
:10F010007CF05AE11E0EE66E320EE66E010E25DB26
:10F0200016E168EC7CF0200EE66ECD0EE66E060E64
:10F0300077EC7DF003E2DCEC7DF003D0100E146E73
:10F04000156A81EC7CF0CD0EE66E060E1CD01B0E10
:10F05000E66E320EE66E010E08DB1DE168EC7CF018
:10F06000200EE66EDD0EE66E060E77EC7DF003E216
:10F07000DCEC7DF003D0100E146E156A81EC7CF090
:10F08000DD0EE66E060EE66EABECD9F0186E060EDF
:10F09000E15E1850B7D7160EE66E320EE66E010E20
:10F0A000E4DAB0E1DF6AAED7DF500AE0E66A86EC68
:10F0B00082F0E552010EE66E86EC82F0E55202D057
:10F0C00054ECD3F00501D26B89DB080E186F000EEB
:10F0D000E55227D325EC7DF0DF6A82EC7DF0000E4F
:10F0E000C7EC7CF011E2FD0EDBCFE9FFDB2AFE0E60
:10F0F000DBCFEAFF01E3DB2AEF50DF1AFB0EDB0672
:10F10000FC0EEBE2DB06E9D7FA0EDB500BE04FEC2E
:10F110007DF0DFCFEFFFDF1CE66E9CDBE552E750B2
:10F12000EF6E0BD04FEC7DF0EF50DF5C08E1DF1CA1
:10F13000146E90DBEF50145C02E1010E01D0000E62
:10F14000E552EFD2F7DA490EE12694DBAAEC7DF026
:10F1500001E20CD122EC7DF002E2010E08D10001A7
:10F160008199250EDB6A34DB3EE0D9EC7CF001E0CE
:10F17000FDD0EFEC7CF001E0F9D0070EE66E320E28
:10F18000E66E010E72DA0BE1FCEC7CF0ECE10001C2
:10F190008189010EF36E250EF3CFDBFFE4D7030E5A
:10F1A000E66E320EE66E010E60DA05E1200ED6DA6A
:10F1B000D950040F0BD0FF0EE66E310EE66E010E35
:10F1C00054DA07E1200ECADAD950280FDFEC7DF0BF
:10F1D000CAD7FA0EE66E310EE66E010E46DAC3E1CC
:10F1E000030EDB6AC0D7030EDB500EE0E80EE66EBE
:10F1F000310EE66E010EE66E03EC7DF007EC7DF05D
:10F2000000018199250EDB6A46DB03EC7DF0DDDB36
:10F2100014E141DBD950280F7FDA28ECD9F0156EC4
:10F22000050EE15E1550000908E16EDB040FDFEC0E
:10F230007DF06ADB280FDFEC7DF0250EDB5006E069
:10F24000E60E146E310E156E010E05D0E40E146E2E
:10F25000310E156E010E166ED950280F5DDA89EC4D
:10F260007DF0AEEC7DF001E07DD0010EE66E220E69
:10F27000B6EC7DF0ABDAE66A61EC7DF0240EB6EC1C
:10F280007DF05AEC7DF0040EDBCF97F0050EDBCF5E
:10F2900098F0060EDBCF99F0070EDBCF9AF0080E40
:10F2A000DBCF9BF0090EDBCF9CF00A0EDBCF9DF08D
:10F2B0000B0EDBCF9EF00C0EDBCF9FF00D0EDBCFE5
:10F2C000A0F00E0EDBCFA1F00F0EDBCFA2F0100EE0
:10F2D000DBCFA3F0110EDBCFA4F0120EDBCFA5F035
:10F2E000130EDBCFA6F0140EDBCFA7F0150EDBCF8D
:10F2F000A8F0160EDBCFA9F0170EDBCFAAF0180E80
:10F30000DBCFABF0190EDBCFACF01A0EDBCFADF0DC
:10F310001B0EDBCFAEF01C0EDBCFAFF01D0EDBCF34
:10F32000B0F01E0EDBCFB1F01F0EDBCFB2F0200E1F
:10F33000DBCFB3F0210EDBCFB4F0220EDBCFB5F084
:10F34000230EDBCFB6F0240EDBCFB7F0250EDBCFDC
:10F35000B8F0260EDBCFB9F0270EDBCFBAF00501EF
:10F36000010E02D00501020ED46FD26B5ADB146E6F
:10F37000490EE15C02E2E16AE552E16E1450D1D13E
:10F38000D9D9400EE12676DAE5DB01E2FBD05ADB83
:10F3900002E2010EF8D0CCEC7DF0D2ECD8F0146E85
:10F3A000050EE15E145014DA1FE003DB01E0EAD041
:10F3B00016DB01E0E7D0D40EE66E310EE66E010EEC
:10F3C00054D908E1380ECAD91EDBABECD9F0146E63
:10F3D000060EE7D7CF0EE66E310EE66E010E45D96A
:10F3E000E2E1030EDB6ADFD7030EDB500AE0D4DB79
:10F3F00067DABA0EE66E310EE66E010EE66E03DBDC
:10F4000006DB010EE66E3A0EB1DBE0D9800EE66E49
:10F4100058DB3C0EABDB4EDB040EDBCF82F6050E79
:10F42000DBCF83F6060EDBCF84F6070EDBCF85F647
:10F43000080EDBCF86F6090EDBCF87F60A0EDBCF90
:10F4400088F60B0EDBCF89F60C0EDBCF8AF60D0E9D
:10F45000DBCF8BF60E0EDBCF8CF60F0EDBCF8DF6EF
:10F46000100EDBCF8EF6110EDBCF8FF6120EDBCF38
:10F4700090F6130EDBCF91F6140EDBCF92F6150E3D
:10F48000DBCF93F6160EDBCF94F6170EDBCF95F697
:10F49000180EDBCF96F6190EDBCF97F61A0EDBCFE0
:10F4A00098F61B0EDBCF99F61C0EDBCF9AF61D0EDD
:10F4B000DBCF9BF61E0EDBCF9CF61F0EDBCF9DF63F
:10F4C000200EDBCF9EF6210EDBCF9FF6220EDBCF88
:10F4D000A0F6230EDBCFA1F6240EDBCFA2F6250E7D
:10F4E000DBCFA3F6260EDBCFA4F6270EDBCFA5F6E7
:10F4F000280EDBCFA6F6290EDBCFA7F62A0EDBCF30
:10F50000A8F62B0EDBCFA9F62C0EDBCFAAF62D0E1C
:10F51000DBCFABF62E0EDBCFACF62F0EDBCFADF68E
:10F52000300EDBCFAEF6310EDBCFAFF6320EDBCFD7
:10F53000B0F6330EDBCFB1F6340EDBCFB2F6350EBC
:10F54000DBCFB3F6360EDBCFB4F6370EDBCFB5F636
:10F55000380EDBCFB6F6390EDBCFB7F63A0EDBCF7F
:10F56000B8F63B0EDBCFB9F63C0EDBCFBAF63D0E5C
:10F57000DBCFBBF63E0EDBCFBCF63F0EDBCFBDF6DE
:10F580000501D26B4EDA146E400EE15C02E2E16AD4
:10F59000E552E16E1450C5D0CDD8030EE126BAD99C
:10F5A000D9DA3EE34FDA02E2010E3BD011D92CE06A
:10F5B00000DA36E114DA34E1AB0EE66E310EE66EB7
:10F5C000010E53D808E144DA03E10001949DEED71F
:10F5D0000001948DEBD7A70EE66E310EE66E010E9C
:10F5E00044D808E135DA03E10001949FDFD7000138
:10F5F000948FDCD7A20EE66E310EE66E010E35D882
:10F60000D5E1020EDB6AD2D7020EDB5003E0000127
:10F61000949D949F60EC85F038EC85F00501D26BE9
:10F6200000DA146E030EE15C02E2E16AE552E16E7B
:10F63000145077D006018151E96EEA6AD890E93614
:10F64000EA367F0EE926060EEA22EE52EF50E66E0B
:10F65000120017DADCEC68F08DDAF3CFDEFFF4CFBE
:10F66000DDFF40DAEE50ED1012000BDAE5EF7CF032
:10F6700026EC3FF0E552E552E7CF19F0E552E7CF2F
:10F6800018F01850F324146E1950F420156E166AF1
:10F69000176A06010051145C0151155802511658A1
:10F6A000035117581200E552E552E552E552120097
:10F6B0001A0EE66E330EE66E010EE3D9A8D90601E6
:10F6C000266B120042EC3EF0E552CED9166A176A5C
:10F6D00006010051F35C0151F458025116580351D0
:10F6E00017581200DBCFEAFF030EEA02F3CFEAFF5E
:10F6F000E902F3CFE9FFF450EA26890EE926050E68
:10F70000EA22EECFE6FFEECFE6FFEFCFE6FF1200F4
:10F71000E66E18DAE5EF7CF0E66E000EDA20E66EB3
:10F720001200E552E7CFD9FF1200D9CFE6FFDACFBA
:10F73000E6FF1200D9CFE6FFE1CFD9FF1200DECFFE
:10F74000E9FFDDCFEAFFEF504808120006010C6B1D
:10F7500091EF7DF0D7D9EE50ED101200E66EE66A1B
:10F76000A2EF7DF086ECD9F0E552E552E55207C0F4
:10F7700014F008C015F009C016F0142A000E152266
:10F7800016222FEF7DF0DED978ECD9F0E552E55264
:10F790001200BFEC3DF0E552E552E5521200166A48
:10F7A000176A5DD916C0E6FF17C0E6FF1200F3EC3A
:10F7B000E4F0146E070EE15E14501200E66AC30E08
:10F7C000E66E320EE66E010EE66E120083DC81D12B
:10F7D0000601005101110211031112003A0EE66EEA
:10F7E000330EE66E010E4DD912D90601256B1200BB
:10F7F0004BD9000E145C000E15581200D950FD0FA5
:10F80000E96EFF0EDA20EA6E1200ADEC3CF0E55234
:10F8100034EF7DF0F3CFE6FFF4CFE6FF1200ABEC60
:10F82000D9F0146E060EE15E14501200D950060F86
:10F83000E96EDACFEAFF1200DECF07F0DECF08F084
:10F84000DECF09F0DDCF0AF0DD52DD520A34000EC2
:10F850000A181200010EE76E22D9E750E926000EC1
:10F86000EA221200FD0EDBCFE6FF00EC70F0E5525D
:10F87000DF6E1200010EF36E030EF3CFDBFF1200FA
:10F88000FD0EDBCF16F0FE0EDBCF17F0180E165C68
:10F89000000E175812008F0EE66E320EE66E010E45
:10F8A000E66E1200AFECD8F0176E070EE15E17504F
:10F8B0001200FD0EDBCF08F0FE0EDBCF09F01200C8
:10F8C000D2ECD8F006D1010EF36EFE0EDB50120022
:10F8D000100EE66EE66A120014C6E6FFC7ECA7F04B
:10F8E000F8D0DF50EA6A820FE96E000EEA22EF508C
:10F8F000E66E1200F3CF16F0F4CF17F0100E95EF6E
:10F900007DF0ADD8A2EF7DF0200EE66EE66A01D95B
:10F91000D9501200010EF36E020EF3CFDBFF12007E
:10F92000FE0EDB50D88014541200DFEC3CF0E552A0
:10F93000E5521200D890F336E806120065ECD8F0D4
:10F94000146E070EE15E145000091200FD0EDBCFAD
:10F95000E6FFFE0EDBCFE6FF12002F0EE66E330E43
:10F96000E66E010EE66E1200CC0EE66E320EE66E0C
:10F97000010EE66E1200140EDBCF14F0150EDBCF75
:10F9800015F01200000E1426040E15221200D88065
:10F99000EE54000EED541200D26F4CDE42EC3EF0FD
:10F9A000E552F3CF18F0F4CF19F034DF43DE38EF2F
:10F9B0007BF0060EE66EE66AD4D804EC69F005D159
:10F9C00039DEEAEC3DF053EF7BF028ECD9F0D2D8E9
:10F9D00000091200A1DEB6D8E4EC9EF0F6D05C0E71
:10F9E000BDDE14EC69F0F1D0E66EE8DE9EDEDFDE0F
:10F9F000F2D8050EE15C12004D0EE66E320EE66E98
:10FA0000010E88EF7BF0D950040F8CEF7BF05FEC98
:10FA1000D9F0BAEF7DF0C6D8A5DEC4D886DE52EFA5
:10FA20007CF046DE080E186F000E1200B8DE09ECFE
:10FA3000DCF039DE120EE66EE66A120008EC73F0B6
:10FA400053EF7BF0F7DD62EF7BF074DEE6521200DD
:10FA50002E0EE66E320EE66E010E88EF7BF014C0BD
:10FA6000E6FF15C0E6FF1200F3CF14F0F4CF15F057
:10FA7000120052DE76D8AEEF7DF0E66EDBDD95EF5C
:10FA80007CF0E66EB1EF7DF0FD0EDBCF14F0FE0EE4
:10FA9000DBCF15F012001CDF48DEE6EF7BF0FD0E39
:10FAA000DBCFE9FFFE0EDBCFEAFF1200D950020FD9
:10FAB0008CEF7BF024ECDCF053EF7BF0E66E95EFFF
:10FAC0007BF0080EE66EE66AE66A09ECDCF053EFBE
:10FAD0007BF0BAEF7DF0AEDD05EF7CF02BDE050E9E
:10FAE000E1261200D9CFE9FFDACFEAFF1200E66E75
:10FAF000E7DE49DE7AEF7CF0140EDBCFE9FF150E6E
:10FB000072EF7BF0D950FB0FE96EFF0EDA20EA6E40
:10FB10001200970EE66E000EE66E120017DEE5523A
:10FB200000D60D6B0E6B0F6B1200F35C000EF458D9
:10FB30001200B10EE66E320EE66E010E49D0F5DD12
:10FB4000E2EF7DF0200EE66E060EE66E1200B6DFE6
:10FB5000E5EF7CF00501010ECCEF7CF008ECD9F06C
:10FB600034D01A0EE66E060EE66E1200E66EE66AF7
:10FB700003EF7DF0146E050EE15E1450120065DF98
:10FB800071DE1468DF50145C120050DFCEDD5AEFD6
:10FB90007DF0166E64DF1CD03C0EE66EE66AE66A07
:10FBA00003EF7DF0FD0EDBCFE9FFFE0E72EF7BF081
:10FBB000E66EE66A95EF7BF0E6DD34EF7DF0ACDDD6
:10FBC0000FEF7CF037DDC9EF7BF06DDD000912002F
:0CFBD000E66EE0EF7CF0B3DFA6EF7BF008
:04FBDC00D4EC85F0F0
:10FBE00000EE00F0140EE80403E3EECFE4FFFBD7D1
:10FBF00000EE14F0140EE80403E3EECFE4FFFBD7AD
:10FC0000E65213ECE4F0E55200EE27F0140EE8049F
:10FC100003E3E5CFEDFFFBD700EE13F0140EE8048D
:10FC200003E3E5CFEDFFFBD7F2EF85F0D4EC85F0F1
:10FC300000EE00F0140EE80403E3EECFE4FFFBD780
:10FC400000EE14F0140EE80403E3EECFE4FFFBD75C
:10FC5000E6529EAA02D08EEC85F0E55200EE27F027
:10FC6000140EE80403E3E5CFEDFFFBD700EE13F03D
:10FC7000140EE80403E3E5CFEDFFFBD7F2EF85F0C8
:10FC800059EC86F0200EE126DE6ADE6ADE6ADD6A65
:10FC9000DD52DD5296ECE1F057EC83F0A7ECD2F0A8
:10FCA000ACECE3F0FFECA3F01AEC84F090ECC0F0C5
:10FCB00084ECC4F016ECDEF081B815D08B682B0E06
:10FCC000E66E350EE66E010EDCEC87F00EEC86F08B
:10FCD0001A0EE66E350EE66E010E88EC86F0CAEC62
:10FCE00087F007EC92F0E2ECDCF0280EE66EE66AB4
:10FCF000010EE66EE66A090EE66E350EE66E010E40
:10FD0000DCEC87F0146E090EE15E14500101FE5127
:10FD1000E66EE66AF90EE66E340EE66E010E88ECCB
:10FD200086F0F3ECE4F0146E070EE15E145054EC30
:10FD3000D3F0D00EF36E1E0EF3CFDBFF070EF36E83
:10FD40001F0EF3CFDBFF1E0EDBCF14F0DB061F0E02
:10FD5000DBCF15F001E2DB061450151006E00C0EA7
:10FD6000E66E9AECE6F0E552EED7010EE66ECEDBDB
:10FD7000E552C7ECE3F007016D51065C146E6E515D
:10FD80000758156E6F510858166E70510958176E46
:10FD90008D0E145C5B0E1558000E1658000E175889
:10FDA0000BE3C7ECE3F006C06DF707C06EF708C0C1
:10FDB0006FF709C070F78B70CCECB0F00AECDDF097
:10FDC000F9ECDDF040EC83F0710EE96E070EEA6E9F
:10FDD000EE500001611908E1EE50621905E1EE50A4
:10FDE000631902E1EE5064190BE061C071F762C063
:10FDF00072F763C073F764C074F7E66A87DBE55295
:10FE000020ECDEF09AECC0F0010E37EC87F0020E29
:10FE100037EC87F0B2ECD1F006C0DEFF07C0DEFFA2
:10FE200008C0DEFF09C0DDFFDD52DD529CEC86F02C
:10FE300014501510161017109CE0B6EC87F007014F
:10FE40007551EE180AE17651EE1807E17751EE1878
:10FE500004E17851EE1801E18CE0DFCF75F7010E77
:10FE6000DBCF76F7020EDBCF77F7030EDBCF78F729
:10FE700082A40DD06C5101E17CD7E66A47DBE552E4
:10FE8000010EE66E43DBE55207016C6B72D7B6ECF0
:10FE900087F0900EEE267E0EEE22000EEE22EE226F
:10FEA0009CEC86F0CFEC87F013EC86F04BECE6F0A0
:10FEB0007CEC87F03B0E1426F90E15220A0E162252
:10FEC000000E1722140E14C0DBFF150E15C0DBFF49
:10FED000160E16C0DBFF170E17C0DBFFB6EC87F05F
:10FEE0009FEC87F0CFEC87F00E6A4BECE6F0040E47
:10FEF00002C0DBFF050E03C0DBFF060E04C0DBFF04
:10FF0000070E05C0DBFF040EB3EC86F0100E0B6E7F
:10FF10000E0E0C6E0D6A0E6A4BECE6F0180E06C063
:10FF2000DBFF190E23EC87F0100E0B6E0E0E0C6E1D
:10FF30002AEC86F0B3EC86F03C0EBBEC87F04BEC81
:10FF4000E6F01C0E06C0DBFF1D0E23EC87F03C0E16
:10FF50000B6E0C6A2AEC86F0DBCF08F0050EDBCFC7
:10FF600009F01A0E08C0DBFF1B0E09C0DBFF140EE0
:10FF7000DBCF14F0150EDBCF15F0160EDBCF16F02D
:10FF8000170EDBCF17F0310E1426010E1522000ECE
:10FF90001622172289EC87F013EC86F0CEECE0F005
:10FFA0007CEC87F03EEC87F05EEC86F0140EDBCF45
:10FFB00018F0150EDBCF19F0160EDBCF1AF0170E66
:10FFC000DBCF1BF0310E1826010E1922000E1A226B
:10FFD0001B2289EC87F0D7EC86F0CEECE0F07FECCA
:10FFE00086F095EC87F0EDEC86F0640EBBEC87F0C4
:10FFF00013ECE6F07FEC86F0025014260350152235
:020000040001F9
:100000000450162205501722140EDBCF1CF0150EDB
:10001000DBCF1DF0160EDBCF1EF0170EDBCF1FF06F
:10002000310E1C26010E1D22000E1E221F2289ECFD
:1000300087F00E6A1CC006F01DC007F01EC008F055
:100040001FC009F0CEECE0F0E4EC86F095EC87F010
:10005000E4EC86F0D6EC87F006C01CF007C01DF07B
:1000600008C01EF009C01FF0020ED8901C361D36C5
:100070001E361F36E806F9E11C5014261D501522C5
:100080001E5016221F501722140EDBCF20F0150E23
:10009000DBCF21F0160EDBCF22F0170EDBCF23F0E3
:1000A000310E2026010E2122000E2222232289EC6D
:1000B00087F0DAEC86F0CEECE0F047EC86F095ECD9
:1000C00087F047EC86F0D6EC87F047EC86F06D0EB3
:1000D0000B6E010E0C6EAAEC85F006C020F007C076
:1000E00021F008C022F009C023F006501426075062
:1000F00015220850162209501722080E14C0DBFFE3
:10010000090E15C0DBFF0A0E16C0DBFF0B0E17C071
:10011000DBFF080EDBCF20F0090EDBCF21F00A0E4B
:10012000DBCF22F00B0EDBCF23F02006000E215A8E
:10013000225A235A6D0EE7EC87F0DAEC86F013ECC6
:10014000E6F047EC86F0080EDBCF24F0090EDBCF9B
:1001500025F00A0EDBCF26F00B0EDBCF27F0040EC6
:10016000BBEC87F024C006F025C007F026C008F0DD
:1001700027C009F0CEECE0F006C024F007C025F05F
:1001800008C026F009C027F006502026075021227B
:100190000850222209502322A6EC86F0640E42EC7D
:1001A00087F00650205C1C6E075021581D6E0850C9
:1001B00022581E6E095023581F6EA6EC86F03EECA6
:1001C00087F0CEECE0F01C500624186E1D5007207E
:1001D000196E1E5008201A6E1F5009201B6E1F0E2C
:1001E00006EC87F01C0E06EC87F0182A19221A225A
:1001F0001B22D950140F9BEC87F01850EE5C146E44
:100200001950EE58156E1A50EE58166E1B50EE58D7
:10021000176E100E14C0DBFF110E15C0DBFF120E9F
:1002200016C0DBFF130E17C0DBFFD950100F29ECEF
:1002300087F003E6000E2FEC87F017E2D950080F85
:100240009BEC87F0EE06000EEE5AEE5AEE5A6D0E5B
:10025000F36E100EF3CFDBFF010EF36E110EF3CF32
:10026000DBFF120EDB6A130EDB6A030EF36E0C0E5D
:10027000F3CFDBFF0D0EDB6A0E0EDB6A0F0EDB6ABF
:10028000D9500C0F29EC87F003E60F0E2FEC87F006
:100290004CE261EC87F08EEC86F01718E8AE02D0E5
:1002A000173408D01450075C1550085816500958D8
:1002B00017500A5835E30C0EDBCF18F00D0EDBCFCC
:1002C00019F00E0EDBCF1AF00F0EDBCF1BF0020E73
:1002D00006EC87F0320EE7EC87F0D7EC86F013ECF3
:1002E000E6F07FEC86F00A0E0B6E0C6AAAEC85F045
:1002F000EDEC86F07A0E185E000E195A1A5A1B5A47
:100300008EEC86F01B18E8AE02D01B3408D01850D3
:10031000075C195008581A5009581B500A5805E331
:10032000D9500C0FF6EC86F0ABD761EC87F01406D1
:10033000155A165A175AD950100F9BEC87F01450C3
:10034000EE5E1550EE5A1650EE5A1750EE5A0C0E3D
:10035000DBCF07F00D0EDBCF08F00E0EDBCF09F080
:100360000F0EDBCF0AF00A34000E0A1809E6D88017
:100370000C0E0754000E0854000E0954000E0A54C7
:100380000EE2D950080FF6EC86F0D9500C0F9BEC1A
:1003900087F00C0EEE5E000EEE5AEE5AEE5A1A0E72
:1003A000DBCFE6FF1B0EDBCFE6FF1C0EDBCFE6FF4D
:1003B0001D0EDBCFE6FF180EDBCFE6FF190EDBCFFD
:1003C000E6FFCC0EE66E340EE66E010EDCEC87F036
:1003D000146E0B0EE15E1450D950100F3DEC86F0F8
:1003E000D9500C0F3DEC86F0D950080F3DEC86F04B
:1003F000B80EE66E340EE66E010E88EC86F0F3EC75
:10040000E4F0146E110EE15E1450140EDBCF06F012
:10041000150EDBCF07F0160EDBCF08F0170EDBCF83
:1004200009F0070E42EC87F0060E021805E10350B2
:1004300003E1045001E1055059E0050E021805E101
:10044000035003E1045001E105504AE0040E021894
:1004500005E1035003E1045001E105503BE0030EC8
:10046000021805E1035003E1045001E105502CE0BE
:10047000020E021805E1035003E1045001E10550AA
:100480001DE0010E021805E1035003E1045001E1F3
:1004900005500EE002502AE1035028E1045026E105
:1004A000055024E1B30EE66E340EE66E010E23D045
:1004B000AE0EE66E340EE66E010E1DD0A90EE66E8F
:1004C000340EE66E010E17D0A40EE66E340EE66E04
:1004D000010E11D09F0EE66E340EE66E010E0BD0AB
:1004E0009A0EE66E340EE66E010E05D0950EE66E9F
:1004F000340EE66E010EE66EE90EE66E060EE66E50
:10050000CAEC87F00701010E6C6F33D4D2DBFE0E0C
:10051000DB5022E1100EE66EE66A200EBFEC86F09C
:10052000DFEC87F0000181AD03D006012A0E02D076
:100530000601200ECD6F000EE66EE66A61C0E6FF92
:1005400062C0E6FF63C0E6FF64C0E6FF17D8146E22
:10055000060EE15E145011D0100EE66EE66A200E13
:10056000D7DBDFEC87F0840EE66E340EE66E010E0C
:10057000CFDBE3EC87F054ECD3F0ABD39ADB070E80
:10058000E126010EF36E060EF3CFDBFF040EDB6AED
:10059000DB50146E156A040E145C000E155855E2FB
:1005A0001EEC87F0D950FB0F146EFF0EDA20156E8B
:1005B000040EDB500F011424E96E000E1520EA6EC4
:1005C000EF50E66EE66A62ECA0F0C0EC87F068DB04
:1005D00067DB32E1050EDB6ADBCF14F014C0E6FF07
:1005E0001EEC87F078ECD9F0E552E552E552E7CF02
:1005F00014F0F4CF16F0F350145C000EF45413E230
:10060000DACF15F0050EDB500F01D924E96E000E8C
:10061000DA20EA6EEF50E66EB8DBE552E750EF6E97
:10062000050EDB2AD9D745EC87F002E115500DE025
:10063000ACDB2E0EEF6E05D045EC87F002E11550D5
:1006400004E02EDB040EDB2AA3D72ADB12E1200E06
:10065000F36E060EDBCFF4FFF350F45C08E2060EF7
:10066000DB50EA6ACD0FE96E060EEA22EF6A54EC1F
:10067000D3F0070EE15C02E2E16AE552E16E29D3B4
:1006800018DBE652200E0F01E76E0019E8AE02D02B
:10069000E73402D0E750005D03E36550020B02E04F
:1006A0008B8203D08B92ACECD7F0E55212D39490AE
:1006B0009492F36A8B6A010EC26EC088380EC16EC6
:1006C000C16AC00EC26EC098BE0EC16EF19E00011E
:1006D000FD6BFB6BFC6B200EAD6E900EAC6EE66A94
:1006E0004B0EE66EE66AE66A10D8C0EC87F09F8A89
:1006F0009D8AD08EF28EF28CC18CC282C2B2FED79D
:10070000C19C87ECDBF093881200D3DAC5EC87F04C
:1007100047DBFEE187DBD880FF0E1454000E155432
:10072000000E1654000E175409E3C5EC87F038DBB1
:10073000FEE178DB1450B06EAD840DD07EDA030E8E
:100740006BDBE806FDE119DA040E2ADBFEE16ADB69
:100750001450B06EAD94BDD2ACDAD7DBEF8CD5DBE4
:10076000EF8ED3DBEF90D1DBEF92CFDBEF94CDDBDD
:10077000EF96FCD991DB0A0EEE6EF8D9140E79DAF9
:1007800061C0EEFF62C0EEFF63C0EEFF64C0EEFF2B
:10079000EDD9040E6EDAEE68EE68EE68EE6AE6D920
:1007A000180E67DA65C0EEFF66C0EEFF67C0EEFFA9
:1007B00068C0EEFFDBD9080E5CDA6EDBEE6ED6D9D0
:1007C0001C0E57DA69C0EEFF6AC0EEFF6BC0EEFF89
:1007D0006CC0EEFFCBD90C0E4CDAA90EEE6EFE0EFD
:1007E000EE6E010EEE6EEE6EC1D9100E42DAEE6ABA
:1007F000EE6AEE6AEE6ABAD9290E3BDA500EEE6E58
:10080000ED6AB4D92B0E35DA100E8ADB2D0E31DAF3
:10081000110E86DB2F0E2DDA120E82DB310E29DA55
:10082000130E7EDB330E25DAEF9EA0D9330E21DACC
:10083000EF9C4FD23EDA3C0EE12610ECE3F0FEDAFC
:100840001AECE3F0E552E552360EE66EE66AF0DAAF
:10085000B6DB610EE66E000EE66E7EDFE552E55217
:10086000060EE66EE66AEADA820EE66E000EE66EC6
:1008700084ECD8F0146E060EE15E1450360EBDDA2C
:10088000E66AE66A2ADA340EB8DA6BDB02E1F0D8FF
:10089000ADD0060EDBCF61F0070EDBCF62F0080EA5
:1008A000DBCF63F0090EDBCF64F00A0EDBCF65F01F
:1008B0000B0EDBCF66F00C0EDBCF67F00D0EDBCF3F
:1008C00068F00E0EDBCF69F00F0EDBCF6AF0100E72
:1008D000DBCF6BF0110EDBCF6CF0120EDBCF6DF0C7
:1008E000130EDBCF6EF0140EDBCF6FF0150EDBCFE7
:1008F00070F0160EDBCF71F0170EDBCF72F0180E12
:10090000DBCF73F0190EDBCF74F01A0EDBCF75F06E
:100910001B0EDBCF76F01C0EDBCF77F01D0EDBCF8E
:1009200078F01E0EDBCF79F01F0EDBCF7AF0200EB1
:10093000DBCF7BF0210EDBCF7CF0220EDBCF7DF016
:10094000230EDBCF7EF0240EDBCF7FF0250EDBCF36
:1009500080F0260EDBCF81F0270EDBCF82F0280E51
:10096000DBCF83F0290EDBCF84F02A0EDBCF85F0BE
:100970002B0EDBCF86F02C0EDBCF87F02D0EDBCFDE
:1009800088F02E0EDBCF89F02F0EDBCF8AF0300EF1
:10099000DBCF8BF0310EDBCF8CF0320EDBCF8DF066
:1009A000330EDBCF8EF0340EDBCF8FF0350EDBCF86
:1009B00090F0360EDBCF91F0370EDBCF92F0380E91
:1009C000DBCF93F0390EDBCF94F03A0EDBCF95F00E
:1009D0003B0EDBCF96F0000181BD08D075C061F001
:1009E00076C062F077C063F078C064F0240E5BDA02
:1009F000E66A080EE66E71D9220E55DAB2DA0FE118
:100A0000560EE66E340EE66E010EE66E970EE66E3C
:100A1000000EE66ED8DA0001B86B819905D00001AE
:100A2000B8518199E8B081893C0E44DA800EE66EB7
:100A3000080EE66E52D93A0E3DDA93DA0BE11F0E3C
:100A4000E66E340EE66E010EE66E820EE66E060E61
:100A5000E66EB9DA88C096FF89C09AFF8D6A916AFE
:100A60002FD83C0EE15C02E2E16AE552E16E31D141
:100A700001D0FFD7010EE66E340EE66ED9D96AECCE
:100A800078F0CCD8E66AE66AE66AE66A09ECDCF059
:100A900077DA360EE66ECCD924ECDCF0C0EF87F0C6
:100AA00008D9FC0EDBCFE6FFFD0EDBCFE6FFFE0E26
:100AB000DBCFE6FFD2ECE2F0E552E552E55209D198
:100AC000C29200019451400B02E0C28C01D0C29C42
:100AD0009451800B02E0C28E1200C29E12000001EF
:100AE000FD51000801E2010C000CE3D8E6520001C0
:100AF000FD5100080FE2FC51FC2BEA6ABB0FE96EC6
:100B0000000EEA22EFCFDFFF400EFC5D01E3FC6B3D
:100B1000FD0701D0DF6ADF50E552DBD0CAD8E652CC
:100B2000AF50DF6EACA202D0AC98AC88400E000192
:100B3000FD5D0EE2FB51FB2BEA6ABB0FE96E000E76
:100B4000EA22DFCFEFFF400EFB5D01E3FB6BFD2BE5
:100B5000E552BFD00D6A0E6A02C006F003C007F06E
:100B600004C008F005C009F0CEEFE0F0FD0EDBCFC9
:100B7000E9FFFE0EDBCFEAFF12001B0E1926B70EAF
:100B80001A22000E1B22E4D9FB0EDBCF0BF0FC0E69
:100B9000DBCF0CF0FD0EDBCF0DF0FE0EDBCF0EF049
:100BA0004BECE6F07CEF87F0D8CFE4FFE0CFE4FF3A
:100BB000E46EDACFE4FFE2CFDAFFE9CFE4FFEACF79
:100BC000E4FFF6CFE4FFF7CFE4FFF8CFE4FFF5CF83
:100BD000E4FFF3CFE4FFF4CFE4FFFACFE4FFFBCF71
:100BE000E4FF1200E5CFFBFFE5CFFAFFE5CFF4FF0E
:100BF000E5CFF3FFE5CFF5FFE5CFF8FFE5CFF7FF52
:100C0000E5CFF6FFE5CFEAFFE5CFE9FFE5CFDAFF75
:100C1000E550E5CFE0FFE5CFD8FF1000146E050EDC
:100C2000E15E145012000E6A14C006F015C007F001
:100C300016C008F017C009F01200FB0EDBCF18F049
:100C4000FC0EDBCF19F0FD0EDBCF1AF0FE0EDBCF72
:100C50001BF012000D6A0E6A72D94BECE6F005C06B
:100C6000EDFF04C0EDFF03C0EDFF02C0EFFF040E77
:100C70001200E926000EEA2212005DD9EECFE6FF4F
:100C8000EECFE6FFEECFE6FFEFCFE6FF120002C0A9
:100C900020F003C021F004C022F005C023F01200B0
:100CA000D950F90FE96EFF0EDA20EA6EEE50ED1022
:100CB0001200D9CFE6FFE1CFD9FF120013ECE6F026
:100CC00002C014F003C015F004C016F005C017F000
:100CD0001200E552E7CFD9FF1200E66AE66A5FEC40
:100CE000DCF0146E080EE15E1450E66A120004D9BE
:100CF0007A0E145E000E155A165A175A120002C0C8
:100D000018F003C019F004C01AF005C01BF012005F
:100D1000E66EDD0EE66E060EE66E1200100EDBCFFE
:100D200007F0110EDBCF08F0120EDBCF09F0130E27
:100D3000DBCF0AF00A50120019D9EECF14F0EECF33
:100D400015F0EECF16F0EFCF17F01200080EDBCF44
:100D500006F0090EDBCF07F00A0EDBCF08F00B0E12
:100D6000DBCF09F01200DBCF06F0050EDBCF07F07A
:100D7000060EDBCF08F0070EDBCF09F01200E66E9F
:100D8000CD0EE66E060EE66E1200060EDBCFF3FF0A
:100D9000DB2AF350EA6ACD0FE96E060EEA22120052
:100DA000D8901732163215321432E80612000E6A45
:100DB000A8EF87F00E6A20C006F021C007F022C01D
:100DC00008F023C009F0120002C01CF003C01DF09F
:100DD00004C01EF005C01FF0120006C018F007C0C6
:100DE00019F008C01AF009C01BF01200A4D8EE2AAE
:100DF000000EEE22EE22EE221200E66EE66AD950D6
:100E0000060FE66E000EDA20E66E12001826000EBF
:100E100019221A221B221200D890183619361A36B7
:100E20001B3612001406000E155A165A175A1200D5
:100E3000E66A610EE66E000EE66E1200D9CFE6FF9E
:100E4000DACFE6FF120007C0DBFFD950040F9BEF9B
:100E500087F071D8D890030EEB50000A1200EE5CB8
:100E6000000EEE58000EEE58000EEE581200E66E20
:100E7000E66A9DECC4F0E552E5521200900EA7D848
:100E80000E6A120078D8CEEFE0F0040EDB50146E3C
:100E9000156A030E14181200C00EEE6EA80EEE6E48
:100EA000010EEE6E1200E66EE66A970EE66E000E1A
:100EB000E66E1200E66EE66A820EE66E060EE66EDC
:100EC00012000C0EDBCF14F00D0EDBCF15F00E0E62
:100ED000DBCF16F00F0EDBCF17F0142A000E152211
:100EE00016221722320E73D89EDEE8DE0A0E0B6E33
:100EF0000C6A30DE77EF86F006C014F007C015F0FC
:100F000008C016F009C017F0120030DE200E39EFCD
:100F100086F0B10E0B6E3A0E0C6E020E0D6E1200C4
:100F2000EE6E270EED6EB6EF85F0AC0E0B6E8E0EEC
:100F30000C6EAAEF85F0E96EDACFEAFF1200EECF71
:100F400006F0EECF07F0EECF08F0EFCF09F0120079
:100F500018C006F019C007F01AC008F01BC009F04D
:100F600012006AEC78F05ADE00091200D9CFE9FFCE
:100F7000DACFEAFF12000B6E0C6A0D6A0E6A1200DD
:100F8000E552E552E552E552120057DE45DFF5DD48
:100F9000020E1200F3ECE4F041DE54EFD3F0800EC9
:100FA0000B6E510E0C6E010E0D6E1200B50E0B6E17
:100FB000050E0C6EAAEF85F0E2DEF3EFE4F0D2EC62
:100FC000D8F00EEF86F05FECD9F00EEF86F00B6EE6
:080FD000010E0C6E0D6A120007
:080FD80054EC8EF0E6528A840D
:100FE00093949496949A94888A8693969E96200ECB
:100FF000C66EC78CC79E72EC8DF01D0EB0EC8FF0E4
:10100000080EDF14F8E1DF1C010BF5E10101010E10
:10101000FD6FF96BFA6BE66A080E4AEC8EF0E66A31
:10102000090E4AEC8EF0730EE66E0C0E77EC8FF024
:101030000D0E4AEC8EF0730EE66E0A0E77EC8FF012
:101040000B0E4AEC8EF0750EE66E040E77EC8FF008
:10105000050E4AEC8EF0750ECFEC8FF0E66A25ECAB
:101060008DF0E552E66A020EE66E6EEC8EF00D0E25
:10107000E66E69EC8EF0320EE66E020E4AEC8EF0F1
:10108000120EE66E040E4AEC8EF0400EE66E030E73
:101090004AEC8EF03F0EE66E090E4AEC8EF0120E10
:1010A000E66E060E4AEC8EF00C0EE66E070E4AEC6B
:1010B0008EF0EE0EE66E0A0E4AEC8EF0050EE66E2F
:1010C0000B0E4AEC8EF0040E54EC8FF082C0E6FF5B
:1010D000040E4AEC8EF083C0E6FF050E4AEC8EF05B
:1010E00084C0E6FF020E4AEC8EF085C0E6FF030ED8
:1010F0004AEC8EF086C0E6FF69EC8EF087C0E6FF12
:10110000010E4AEC8EF0E66A150E4AEC8EF0120ED5
:101110004FEC8EF0E8CFFEF1E66A010EE66E100E9F
:10112000E66E08EC8EF0E552E552E552720EE66E80
:10113000340EE66E140EE66EDAEC8EF0E66ADAEC49
:101140008EF06EEC8EF0E2EC8EF0E55259EF8EF000
:10115000010EE66ECAEC8DF0E552F350040B01E08F
:10116000010E120011EC8FF0080B080A01E0010ECD
:101170001200C2EC8FF00101FD5123E1010EFD6F61
:10118000F9C114F0FAC115F01406000E155A14C076
:10119000DEFF15C0DDFFC6EC8FF05DEC8EF004E2E3
:1011A000730EDE6E0F0EDD6E400E06EC8FF0DFCF9D
:1011B000E6FF0C0E4AEC8EF024EC8FF00D0E4AEC9C
:1011C0008EF0020EE15C02E2E16AE552E16E59EF57
:1011D0008EF054EC8EF0040EE1269AEC8FF0190E8E
:1011E000B0EC8FF00E0E5BEC8FF00E0E4FEC8EF02D
:1011F00009EC8FF00F0E69EC8FF09AEC8FF0190E5E
:101200004FEC8EF0DF500001145CE9E10C0E5BEC5A
:101210008FF00C0EB0EC8FF00D0EB3EC8FF0C8EC2D
:101220008EF0DECF16F0DDCF17F01450165C15509F
:10123000175821E2730E186E0F0E196E1A6A1B6A88
:10124000020EDBCF20F0030EDBCF21F0DE50205C5E
:101250001C6EDD5021581D6E1E6A1F6A1C50185CE2
:10126000146E1D501958156E1E501A58166E1F50C8
:101270001B58176E1DD0C8EC8EF0DF50141809E112
:10128000DE52DD50151805E1730EF36E0F0EF46E8D
:1012900013D0DECF16F0DDCF17F0020EDB50165C58
:1012A000146E030EDB501758156E1406000E155AF7
:1012B00014C0F3FF15C0F4FF040EE15C02E2E16A22
:1012C000E552E16E59EF8EF0D9CFE6FFE1CFD9FFBD
:1012D000150EE126190EE66E010EE66E1CEC8EF080
:1012E000E552E552190EE66EB4EC8DF0E552146E3F
:1012F000140E14C0DBFF000EE66EE66A1CEC8EF0E6
:10130000E552E552140EDB5002E1000EB7D00101A8
:10131000FD5103E12EDF000EB1D0F9C1FBF1FAC19E
:10132000FCF1FBC1E6FFE66AEDEC8DF0E552E5521B
:10133000FCC1E6FF010EE66EEDEC8DF0E552E552E4
:10134000140EE66EE66AD9CFE6FFDACFE6FF38DBA9
:10135000E552E552E552E552120EDBCFE6FF130EE1
:10136000DBCFE6FF88ECA1F0E552E552120EF3CF99
:10137000DBFF130EF4CFDBFFDECF14F0DDCF15F073
:10138000166A176AD880730E14540F0E1554000E87
:101390001654000E175431E3D9CFE9FFDACFEAFF34
:1013A000EF50010B2AE1D950020FE96EDACFEAFFC4
:1013B000EE52EE52EE52EF50800B1FE1D950020F69
:1013C000E96EDACFEAFFEE52EE52EF50100B15E164
:1013D000D950020FE96EDACFEAFFEE0ED880EE5454
:1013E000050EED540AE3D950020FE96EDACFEAFF99
:1013F000EE52EE52EF50800B01E1FF00DECFF9F12B
:10140000DDCFFAF1060EE66EE66AD9500C0FE66EF5
:10141000000EDA20E66EFD0EDBCFE9FFFE0EDBCF1D
:10142000EAFFE9CF14F0EACF15F014C0E6FF15C0CB
:10143000E6FF84ECD8F0166E060EE15E1650FB0E49
:10144000DBCFE9FFFC0EDBCFEAFFEF68130EDB50CA
:10145000080810E1120EDB5004E0120EDB50060803
:1014600009E1FB0EDBCFE9FFFC0EDBCFEAFF120E3A
:10147000DBCFEFFF0101FD6B010E00D0146E150EE6
:10148000E15C02E2E16AE552E16E1450E552E7CF19
:10149000D9FF120054EC8EF0760ECFEC8FF0D950BD
:1014A000FA0F72EC8EF0830EEE260F0EED22FA0E7E
:1014B000DBCFE6FF060E4AEC8EF0FB0EDBCFE6FF3D
:1014C000070E4AEC8EF0060EE66EE66A0DEC8FF023
:1014D000D6EC8EF017EC8FF0060EE66EE66A820E02
:1014E000E66E000EE66E17EC8FF0080EE66EADDAD3
:1014F000E552FC0EDB5002E1000E01D0060EE66E56
:10150000A4DAE552D6D3D0DB0E0EE12677EC8EF0CE
:10151000050E0101FE5D03E0060EFE5D5CE1DE6A84
:10152000DD6A9EEC8FF010E1D9CFE9FFDACFEAFF58
:10153000EE2A000EED22EECF15F0EDCF16F0E80EFC
:10154000155C030E1658EDE31C0E97EC8FF0E85077
:10155000020B09E1DECF15F0DDCF16F0E80E155CC9
:10156000030E165838E3E6EC8EF0D5EC8FF0060E3D
:1015700096DB040E14C0DBFF070E91DB050E14C0D2
:10158000DBFF040EDB2A050E01E3DB2A32EC8FF0D1
:10159000DB6A100EF36E0D0EDBCFF4FFF350F45C3C
:1015A00018E21C0E97EC8FF0E850020B12E0BDEC35
:1015B0008EF0EE52EE52EE52EF50200B0AE097DB27
:1015C0009EEC8FF0FDE0E6EC8EF032EC8FF0DB2A43
:1015D000E0D75FEC8FF00E0EE15C02E2E16AE552CB
:1015E000E16E67D361DB020E3EEC8FF002E2E9ECC4
:1015F0008EF02CEC8FF0020EE15C02E2E16AE55223
:10160000E16E57D3C2EC8FF0B0EC8FF0030EB3EC69
:101610008FF07EEC8FF0A4EC8FF002E2E16AE552ED
:10162000E16E47D3C2EC8FF04FEC8FF00DEC8FF0F2
:1016300050DBBCDB010EA4EC8FF002E2E16AE55264
:10164000E16E37D331DB040E3EEC8FF001E2C1DBFB
:10165000D5EC8FF02CEC8FF0FB0EDBCFE6FFFC0E11
:10166000DBCFE6FF10D8E552E552F3CFDEFFF4CF33
:10167000DDFF5FEC8FF048DB040EE15C02E2E16A23
:10168000E552E16E16D310DB1E0EE126020EDB6A78
:10169000030EDB6A040EDB6A050EDB6A4FEC8FF08B
:1016A000E3EC8FF075E057EC8FF0140ED880EE5419
:1016B000000EED5404E2140E146E156A06D0FD0EF1
:1016C000DBCF14F0FE0EDBCF15F0060E14C0DBFFEF
:1016D000070E15C0DBFF060EDBCFE6FF070EDBCFE4
:1016E000E6FFD950080F1ADB060EDBCF14F0070E09
:1016F000DBCF15F0DCDB1450EE5E1550ED5A3DDB10
:10170000EF50010B13E0D950080F146EDACF15F02B
:10171000060EDB501424E96E070EDB50DA20EA6E69
:10172000EF6A060EDB2A070E01E3DB2AD950080F09
:10173000146EDACF15F01C0E14C0DBFF1D0EDACFCD
:10174000DBFF1BDBEE50ED10ABE0D9501C0FE96E58
:10175000DACFEAFFEECFF3FFEDCFF4FF020EEE2675
:10176000000EEF22F3CFE9FFF4CFEAFFEECF14F043
:10177000EFCF15F0166A176A35DBEE221650EE220F
:101780001750EE22FADA020EEE5E000EED5AD9D7AD
:1017900063DBFEDA166A176A040EDBCF18F0050E5B
:1017A000DBCF19F01A6A1B6A18501426195015223B
:1017B0001A5016221B5017222CDB030E15C0DBFF1C
:1017C000040E16C0DBFF050E17C0DBFF040EDBCFD7
:1017D00014F0050EDBCF15F005DBED22020EDB1C4D
:1017E000146E030EDB1C156E14C0F3FFF46E1E0E98
:1017F000E15C02E2E16AE552E16E5BD255DA060E87
:10180000E126040EDB6A050EDB6A51DBFF0EEE18E3
:1018100016E1FF0EED1813E1010EF36E040EF3CF87
:10182000DBFF020E84DBE850E66E41DBE552E75059
:10183000EE6EED6A030E33DAFE0E14C0DBFF89DBB9
:10184000FF0EEE1816E1FF0EED1813E1010EF36E18
:10185000050EF3CFDBFF7EDA0001E850E66E79DBA0
:10186000E552E750EE6EED6A010E19DAFC0E14C077
:10187000DBFFADDB010ED880EE54000EED542EE3FD
:10188000050EDB5001E10BDB040EDB5005E1020E1F
:1018900006DABFDA030E1DDBFB0E7DDBFC0E68DB18
:1018A0002DDBE66E9AD9E552E552F90EDBCF14F046
:1018B000DB06FA0EDBCF15F001E2DB061450151043
:1018C00004E071D8E66EC1D8EFD7050EDB5001E118
:1018D000C3DA040EDB505AE117DB57D0040EDB509D
:1018E0000EE0F90EDBCF16F0FA0EDBCF17F03DDA83
:1018F000156E8FDA030E15C0DBFF06DBCBD94FDA8E
:101900001406000E155A63DB1450EE261550ED2216
:101910001F0E0DDB14BAFCD7FB0EDBCFE6FF100E5B
:10192000B9D9FC0EDBCFE6FF110EB4D976DA140E6E
:10193000B1D93CDA150EAED932DABFD903E3F8D902
:1019400001E2EADAF90EDBCFE6FF120EA3D9FA0EB6
:10195000DBCFE6FF130E9ED9100E7ADA200EE66E6C
:101960009CDA050EDB5012E0F90EDB2AFA0E01E3D9
:10197000DB2A15DAA2D903E3DBD901E2CDDAF90ECD
:101980000ADBFA0EDBCFE6FF010E84D9060EE15C1E
:1019900002E2E16AE552E16E8CD143DA200B200AC3
:1019A00001E0010E120080D9E6528A949E963A0E0A
:1019B000C96E9EA6FED7AED9C96A9EA6FED792D2A0
:1019C00073D9030EE1268A949E963A0EC96EDE6A9A
:1019D000DD6AF9DA05E0FD0EDB06FE0E01E2DB064C
:1019E0009EA6FED79E96020EC9CFDBFFCFDAFB0E76
:1019F000DBCF16F0FC0EDBCF17F01650145C17503F
:101A000015581AE2C96ADF2A010E01E3DB2ADBDA84
:101A10000CE0FD0EDB2AFE0E01E3DB2A9EA6FED7BC
:101A20009E960BDAC9CFEFFFE1D79EA6FED79E9612
:101A3000020EC9CFDBFFDAD78A8466D9030EE15CD8
:101A400002E2E16AE552E16E34D187DA9EA6FED762
:101A500061D9FE0EDB50C96E9EA6FED73FD27DDA5D
:101A60009EA6FED757D975DAEE50ED1010E0E5D9F5
:101A7000EF50C96EFD0EDB2AFE0E01E3DB2AFB0EE2
:101A8000DB06FC0E01E2DB069EA6FED7EBD78A84BE
:101A9000E5520FD162DA9EA6FED73CD9D950FA0F93
:101AA00021D9EE50ED101BE0FC0EDBCFF6FFFD0E52
:101AB000DBCFF7FFFE0EDBCFF8FF0800F550C96E55
:101AC000D950FC0F0FD9EE2A000EEE22EE22FA0EAC
:101AD000DB06FB0E01E2DB069EA6FED7DED78A847C
:101AE000E552E7D0E1D8050EE12685D9010EF36E67
:101AF000DB6E020EDB6A010EDBCF14F0DB06020E9A
:101B0000DBCF15F001E2DB061450151006E00C0ED9
:101B1000E66E9AECE6F0E552EED78A949E96C96896
:101B20009EA6FED7F7D88A84010EF36E030EF3CF7C
:101B3000DBFF040EDB6A030EDBCF14F0DB06040EC2
:101B4000DBCF15F001E2DB061450151006E00C0E99
:101B5000E66E9AECE6F0E552EED7050EE15C02E2A5
:101B6000E16AE552E16EA5D0C6D9C96E9EA6FED740
:101B7000D1D8C96A9EA6FED7B5D1BDD9C96E9EA6D9
:101B8000FED7C8D8C96A9EA6FED7C4D8C96A9EA681
:101B9000FED7A8D1F7D998D9010EE66E120E7AD8E1
:101BA0000A0E82D90A0EEFD8000114B0FBD702DA70
:101BB000E66A120E6FD8180EE6D8DF6E190EE3D85B
:101BC000010E14C0DBFF000E76D99ED8020EE15C38
:101BD00002E2E16AE552E16E6CD08DD94009C96E2E
:101BE0009EA6FED79FD99EA6FED778D184D9A009FC
:101BF000C96E9EA6FED796D99EA6FED76FD17BD979
:101C00008009C96E9EA6FED78DD99EA6FED766D145
:101C10004BD85AD9FC0EDBCFE6FF160E3BD8FDD8C9
:101C2000170E38D80A0E40D90A0EADD8000114B0EC
:101C3000FBD7000E40D93DD037D8030E09D9B6D80E
:101C40002CD937D0040E04D91D0E71D914B4FCD789
:101C50001F0E6DD914B6FCD7200E06EF8FF0CBD82F
:101C60001D0E65D914A0FCD7E2EF8EF01DD8150E1D
:101C70001BD99CD8150E0ED8000E1DD91AD014D819
:101C8000E652150E11D9150E6BD9000E14D9DF507E
:101C9000E5520FD0E66EA1DFE552E5521200E66E86
:101CA00063DFE552146E1200D9CFE6FFE1CFD9FF12
:101CB0001200E552E7CFD9FF1200166A176AD880E2
:101CC000730E14540F0E1554000E1654000E1754B4
:101CD0001200E66A82DFE552E5521200ADDFE552FE
:101CE000E5521200E96EFF0EDA20EA6E1200800E55
:101CF000E66ED3D8800EACD80A0EE66E1C0E3DD927
:101D0000080EE66E4DEF8FF041D914C0F3FF15C0F9
:101D1000F4FF12009E96C950DF6E1200E66E000EB0
:101D2000DA20E66E4DDEE552E552E552E55212004C
:101D3000F90EDBCF18F0FA0EDBCF19F01A6A1B6A26
:101D4000D880730E18540F0E1954000E1A54000E3A
:101D50001B541200E66A08DFE552146E1200E652C8
:101D60008A949E96FE0EDB501200FD0EDB50162468
:101D7000146EFE0EDB5017201200D950060FE96ECC
:101D8000DACFEAFF1200E66EF8DEE552146E1200BA
:101D9000020EDBCF14F0030EDBCF15F01200FB0EAA
:101DA000DBCF14F0FC0EDBCF15F01200FE0EDBCF04
:101DB000E6FF12002DDFE552E552E552000EE66E19
:101DC000E66A1200040EE66E4DEF8FF0080E28EF63
:101DD0008FF0D9CFE9FFDACFEAFF740EEE5E0F0E77
:101DE000ED5A1200D950020FE96EDACFEAFF145013
:101DF000EE2615501200200EE66E1E0EBDEF8FF07F
:101E0000E6528A949E967A0EC96E1200E66E1E0EF7
:101E1000D5D0020E14C0DBFF1200FD0EDBCFE6FFB3
:101E200012001F0EE66EA0DEE552E850120017DE2B
:101E3000E552E552E552E5521200FD0EDBCFE9FF17
:101E4000FE0EDBCFEAFF1200010EDBCFE6FF120031
:101E5000E66E1F0EBDEF8FF0DFCFE6FF3ADFF4DF57
:101E60004AEF8EF0040E97D8050E82D8070EE66E64
:101E7000E66AD950060F52DF0D0E1200E126140E4D
:101E80000101176AFB25166EFC5117226EDF14C084
:101E9000DEFFDD6E7BD85DEF8EF01F0E8FD05ADF38
:101EA000DF6E010EB3EF8FF0E66E030E94D0D950C3
:101EB000FD0F72EF8EF0E66EE66A6EEF8EF0020EA8
:101EC0006AD8030EB8EF8FF075D870DF140E4AEFA2
:101ED0008EF0E5DE030E14C0DBFF12001BDF8A84E8
:101EE000E552E7D617DF8A84DF50E552E2D6D2DE2C
:101EF0000F0EE66E1200D8DEAFEF8EF08EDF020E10
:101F0000C9DE54DF030E1200020EDBCFE6FFC2DE95
:101F1000030EDBCFE6FF12005AD8740EEE5E0F0EF2
:101F2000ED5A1200F7DEFD0EDB50C96E1200B7DE6F
:101F300000011200190EE66E010E4DD01C0EAFDE30
:101F40000A0E000114141200A5DEDEDE020EE15CB2
:101F50001200D950FB0F72EF8EF0A6DE00EF8FF06B
:101F60009EDEDF6E12009BDE010E14C0DBFF12004E
:101F7000DBCFE6FF010E4AEF8EF0E66E37DEE5526C
:101F8000E552120091DE020EE1261200DECF14F0BF
:101F9000DDCF15F01200DBCFE6FF69EF8EF0E66EC5
:101FA000020EA5DF030E4AEF8EF0D4DE32DF010E03
:101FB00069EF8FF0140EE66E020E0DD0E66E1FDE96
:101FC000E552E552120073DFEE50ED101200D950C9
:0C1FD000F90F72EF8EF0E66E6EEF8EF0EF
:041FDC00D8EC95F0B8
:101FE000170EE126D950010F146EDACF15F0150E39
:101FF00014C0DBFF160EDACFDBFFDF6A060EDF5CF4
:1020000024E2DF5006E005EC96F001E3DB2A3A0E0D
:10201000EF6E27EC96F002ECA1F0E552E66E05ECCF
:1020200096F001E3DB2AE552E750EF6E27EC96F0DD
:1020300016ECA1F0E552E66E05EC96F001E3DB2A22
:10204000E552E750EF6EDF2AD9D7150EDBCFE9FF57
:10205000160EDBCFEAFFEF6AD950010F33EC96F092
:102060000DEC96F0170EE15C02E2E16AE552E16EDA
:10207000DFEF95F0D8EC95F0060EE126F1EC95F047
:102080008F0EE66E310EE66E010EE66EC7EC95F031
:10209000F3ECE4F0146E070EE15E1450C7EC95F01B
:1020A0000DEC96F0060EE15C02E2E16AE552E16EAB
:1020B000DFEF95F096EC96F014E0030A06E0010AD3
:1020C00010E185ECE2F0DF6E1FD0FE511DE004014F
:1020D000E05102E1000E01D0010EDF6EDF5014E08E
:1020E00011D085ECE2F0DF6EDF500EE00301FE510F
:1020F0000BE00401E05102E1000E01D0010EDF6EA1
:10210000DF5002E0ACECD7F0DF50E552DFEF95F0A6
:102110000401E05105E0CCECB0F0ACECD7F0F8D71E
:102120001200D8EC95F0020EE126010EDB6AFC0EDF
:10213000DBCFF3FFDB06F35000094DE0FD0EDBCFF4
:10214000E9FFFE0EDBCFEAFFEF6A88D80009FDE069
:10215000AED8DF6E0D0EDF5C3EE00A0EDF5C3BE0CA
:10216000080EDF5C03E07F0EDF5C1DE1010EDB503B
:10217000DEE0010EDB06FD0EDB06FE0E01E2DB06F5
:1021800099DF0009FDE1080E54EC96F093DF000999
:10219000FDE1200E54EC96F08DDF0009FDE1080E04
:1021A00054EC96F0C4D7B9EC95F0C1E083DF000998
:1021B000FDE1DFCFE6FFC9D8E552010EDB2AFD0EB7
:1021C000DBCFE9FFDB2AFE0EDBCFEAFF01E3DB2AF0
:1021D000DFCFEFFFACD7010EDB50146E020EE15CD7
:1021E00002E2E16AE552E16E1450DFEF95F0A6ECF1
:1021F00096F00AE0030A05E0010A06E192EC96F087
:1022000010D0FE510EE005D092EC96F00301FE5185
:1022100008E07EDFE3EC95F06AECD7F0E55259EC8C
:1022200096F0DFEF95F0A6EC96F00AE0030A05E0E1
:10223000010A06E19BEC96F00FD0FE510DE005D0AF
:102240009BEC96F00301FE5107E062DFF1EC95F0A4
:102250003AECD7F059EC96F0DFEF95F096EC96F06B
:102260000FE0030A05E0010A0BE16FEC85F01AD0DC
:10227000FE5119E0FF510EE1F8EC95F014E00FD09B
:102280006FEC85F0DF6EDF500EE10301FE510BE0D5
:10229000FF5102E0010E06D0F8EC95F004E00301D6
:1022A000010EFF6FDF6EDF50E552DFEF95F0D8ECE7
:1022B00095F0E65242EC96F014E0030A06E0010ABB
:1022C00010E175EC85F0DF6E3CD0FE513AE0DF6A3C
:1022D000FF5104E0FFC1DFFFFF6B33D07BEC96F0D2
:1022E00030D075EC85F0DF6EB9EC95F018E10301A4
:1022F000FE5127E0DF6AFF5104E0FFC1DFFFFF6B03
:1023000002D07BEC96F0B9EC95F01BE00301010ED6
:10231000FD6F7E0EE66E310EE66E010E07D00301F4
:10232000FD6B6D0EE66E310EE66E010EE66EDD0E95
:10233000E66E060EE66EF3ECE4F01DEC96F054EC5F
:10234000D3F0DF50E552DFEF95F0A6EC96F00AE00F
:10235000030A05E0010A06E146EC96F015D0FE51AD
:1023600013E005D046EC96F00301FE510DE0010E9E
:10237000E66ED950FE0FE66EFF0EDA20E66E2EEC0A
:10238000D7F0E55259EC96F0DFEF95F0D8EC95F0E8
:10239000060EE126040EDB6ADB50146E156A040E8D
:1023A000145C000E15582CE2C7EC95F0D950FB0FC9
:1023B000146EFF0EDA20156E040EDB500F0114248C
:1023C000E96E000E1520EA6EEF50E66EE66A62ECEA
:1023D000A0F0DDEC95F0DBDB0DEC96F0040EDB50AD
:1023E000146E156A030E141802E1155009E06B0E05
:1023F000E66E310EE66E010EB8DB040EDB2ACCD79A
:10240000060EE15C02E2E16AE552E16ED8D3D0DB70
:102410002F0EE1260401D86B4B0ED96FDA6BDB6B04
:10242000080EDE6FDD6BDC6B4DEC96F0E8AE02D093
:10243000E73402D0E750005D03E36550020B04E08F
:102440008B920301FE6B04D08B820301010EFE6FA1
:10245000280EE66EE66A010EE66EE66A650EE66E28
:10246000310EE66E010EE66ED950250F33EC96F074
:10247000F3ECE4F0146E090EE15E1450CCECB0F015
:102480003B0EE66E310EE66E010E6FDBA7DD370EFA
:10249000E66E310EE66E010E68DB2A0EE66E310E38
:1024A000E66E010E62DBD950250FDDDBB6DB060ED2
:1024B000E66E310EE66E010E58DBF00EE66E300E63
:1024C000E66E010E52DB75C0E6FF76C0E6FF77C010
:1024D000E6FF78C0E6FF77EC96F0D50EE66E300E9C
:1024E000E66E010E42DB7DC0E6FF7EC0E6FF7FC0E8
:1024F000E6FF80C0E6FF77EC96F0BC0EE66E300E8D
:10250000E66E010E32DB6DC0E6FF6EC0E6FF6FC007
:10251000E6FF70C0E6FFEBDBA30EE66E300EE66E64
:10252000010E23DB71C0E6FF72C0E6FF73C0E6FF59
:1025300074C0E6FFDCDB8E0EE66E300EE66E010E3A
:1025400014DB79C0E6FF7AC0E6FF7BC0E6FF7CC003
:10255000E6FFCDDB780EE66E300EE66E010E05DB93
:1025600087DB5BDB620EE66E300EE66E010EFDDA97
:102570008AC0E6FF8BC0E6FF65DB4D0EE66E300ECF
:10258000E66E010EF2DA8CC0E6FF8DC0E6FF5ADB84
:10259000340EE66E300EE66E010EE7DA8EC0E6FF10
:1025A0008FC0E6FF4FDB1D0EE66E300EE66E010EAD
:1025B000DCDA90C0E6FF91C0E6FF44DB080EE66E71
:1025C000300EE66E010ED1DA92C0E6FF93C0E6FF50
:1025D00039DBF30EE66E2F0EE66E010EC6DA4DDB2A
:1025E0001CDBEA0EE66E2F0EE66E010E6DDB400B75
:1025F00006E0E60E146E2F0E156E010E05D0E30EEA
:10260000146E2F0E156E010E58DBC30EE66E2F0EE4
:10261000E66E010E59DB400B06E0BB0E146E2F0E6A
:10262000156E010E05D0B20E146E2F0E156E010E32
:1026300044DBA90EE66E2F0EE66E010E96DA9C0EB6
:10264000E66E2F0EE66E010E3FDB010B02E0A4DA10
:1026500001D0A8DA32DB790EE66E2F0EE66E010E9F
:1026600033DB010B02E09EDA01D096DA26DB700E36
:10267000E66E2F0EE66E010E78DA5E0EE66E2F0E17
:10268000E66E010E21DB020B02E086DA01D08ADA67
:1026900014DB3F0EE66E2F0EE66E010E15DB020B0D
:1026A00002E080DA01D078DA08DB360EE66E2F0E13
:1026B000E66E010E5ADA260EE66E2F0EE66E010E5B
:1026C00003DB040B02E068DA01D06CDAF6DA090EFB
:1026D000E66E2F0EE66E010EF7DA040B02E062DA08
:1026E00001D05ADAEADA000EE66E2F0EE66E010E1F
:1026F0003CDAF30EE66E2E0EE66E010EE5DA080BFE
:1027000002E04ADA01D04EDAD8DAD80EE66E2E0EA2
:10271000E66E010ED9DA080B02E044DA01D03CDAA9
:10272000CCDACF0EE66E2E0EE66E010ECDDA100B71
:1027300006E0E60E146E2F0E156E010E05D0E30EA8
:10274000146E2F0E156E010EB8DA9C0EE66E2E0E6C
:10275000E66E010EB9DA100B06E0BB0E146E2F0EFA
:10276000156E010E05D0B20E146E2F0E156E010EF1
:10277000A4DA850EE66E2E0EE66E010EF6D96A0E0E
:10278000E66E2E0EE66E010EF0D9520EE66E2E0E9D
:10279000E66E010EEAD962DD000916E17EDAE8AEE6
:1027A00002D0E73402D0E750005D03E36550020B2E
:1027B00004E08B920301FE6BEED78B82ACECD7F07A
:1027C0000301010EFE6FE7D74F0EE66E2E0EE66E8A
:1027D000010ECBD9200EDB6A6ADD210A01E1EBD0C4
:1027E000600A01E1C7D0740A01E1BBD0010A01E12E
:1027F000B5D0070A01E1AFD0010A01E1A9D0030A6F
:1028000001E1A3D0010A01E19DD0730A01E18AD060
:10281000110A01E17DD0030A71E01D0A65E0040A96
:1028200059E0030A4BE01F0A3FE01A0A31E01D0A93
:1028300025E0030A19E0170A0DE00E0A01E006D1AF
:10284000410EE66E2E0EE66E010E42DA750EEE6E4B
:10285000000E27D0360EE66E2E0EE66E010E38DA2A
:102860007D0EEE6E000E1DD02D0EE66E2E0EE66E67
:10287000010E2EDA6D0EEE6E000E13D0240EE66EF3
:102880002E0EE66E010E24DA710EEE6E000E09D0E9
:10289000190EE66E2E0EE66E010E1ADA790EEE6E47
:1028A000000EED6E010E49D00B0EE66E2E0EE66E9A
:1028B000010E47DA820EEE6E060E09D0FA0EE66EB3
:1028C0002D0EE66E010E3DDA970EEE6E000EED6EE9
:1028D000030E33D0ED0EE66E2D0EE66E010EFDD921
:1028E0008A0EEE6E000E27D0E10EE66E2D0EE66E1D
:1028F000010EF3D98C0EEE6E000E1DD0D00EE66EDA
:102900002D0EE66E010EE9D98E0EEE6E000E13D07E
:10291000C10EE66E2D0EE66E010EDFD9900EEE6E44
:10292000000E09D0B50EE66E2D0EE66E010ED5D95D
:10293000920EEE6E000EED6E020EF36E200EF3CFD1
:10294000DBFF84D00001817D81D0000181717ED0C8
:10295000000181737BD00001817578D000018177FF
:1029600075D0000181798151100B01E0010E000149
:10297000B86F6CD0610EE66E000EE66EACEC83F0C4
:10298000E552E552A00EE66E2D0EE66E010EE66EE5
:102990006FD95FECD9F051D99A0EE66E2D0EE66E26
:1029A000010EE66E6AD95FECD9F047D90001819932
:1029B0000001B86B4BD038EC85F0880EE66E2D0E1A
:1029C000E66E010ED2D82ED99CD906E2230EDB0684
:1029D000240EFAE2DB06F8D7010EE66E220EE66E52
:1029E000E66A4BD96AEC78F028D9E66A93D9240EC6
:1029F000E66EE66A42D924ECDCF0DFD87A0EE66EA9
:102A00002D0EE66E010EB1D80DD97BD906E2230E4C
:102A1000DB06240EFAE2DB06F8D7010EE66E3A0E6C
:102A2000E66EE66A25D96AEC78F007D9800EE66E84
:102A300071D93C0EE66EE66A1BD924ECDCF0BDD8F9
:102A40006D0EE66E2D0EE66E010E8FD8200EDB04A5
:102A50001DE148D9D950140F06D999D8E4EC9EF05D
:102A6000ACD8000956E0180EDBCFE9FF190EDBCF1A
:102A7000EAFF140EDBCFEEFF150EDBCFEEFF160ED6
:102A8000DBCFEEFF170EDBCFEEFFF8D4020E146E95
:102A9000200EDB50145C53E125D979D805ECE0F029
:102AA000E552E5521C0E06C0DBFF1D0E07C0DBFF22
:102AB0001E0E08C0DBFF1F0E09C0DBFFD9501C0F24
:102AC0008CD8D890030EEB50000A08E6000EEE5C9E
:102AD000000EEE58000EEE58000EEE581AE31C0ED3
:102AE000DBCF07F01D0EDBCF08F01E0EDBCF09F0A9
:102AF0001F0EDBCF0AF00A34000E0A1809E6D88050
:102B0000FF0E0754FF0E0854000E0954000E0A541D
:102B100009E25C0EE66E2D0EE66E010EE66EF7EC37
:102B200090F01FD01A0EDBCFE9FF1B0EDBCFEAFFC0
:102B30001C0EDBCFEEFF1D0EDBCFEDFF9FD4030E8F
:102B4000146E200EDB50145C01E098D4CBD81FD853
:102B5000210EDBCFE6FF220EDBCFE6FF3EECD9F005
:102B6000E552E552E552E55289D4E66EF7EC90F075
:102B7000F0D0DFCFE6FFE66ACDECE4F0E552E552B7
:102B8000F3CF14F0F4CF15F0F350F4101200D9CFB6
:102B9000E6FFDACFE6FF1200980E146E2F0E156EC8
:102BA000010E1200940E146E2F0E156E010E1200FF
:102BB000D9CFE6FFE1CFD9FF1200E552CAD0E552E6
:102BC000E7CFD9FF1200FC0EDBCFE6FFFD0EDBCF17
:102BD000E6FFFE0EDBCFE6FF1200E96EDACFEAFF7A
:102BE0001200FD0EDBCFE6FFFE0EDBCFE6FF12008C
